:020000040800F2
:10000000B85E002029020008A5AC00083999000854
:1000100085AA00080131000881CC0008000000001A
:1000200000000000000000000000000051B80008BF
:100030007548000800000000F1B10008EDB80008A4
:10004000430200084302000843020008430200087C
:1000500043020008430200087948000843020008F0
:1000600043020008430200088548000843020008D4
:100070007D460008430200084302000843020008CE
:10008000430200084302000843020008430200083C
:1000900005310008153100084302000891480008A6
:1000A000430200084302000843020008430200081C
:1000B000430200084302000843020008430200080C
:1000C00043020008430200084302000843020008FC
:1000D0004302000811CB00084302000821CB0008AE
:1000E00043020008430200084302000843020008DC
:1000F00043020008430200084302000843020008CC
:1001000043020008430200084302000843020008BB
:10011000430200084302000843020008D5B9000862
:10012000430200088D4600089D460008AD460008C1
:10013000430200084302000843020008430200088B
:100140002531000835310008430200084302000849
:10015000BD460008CD4600084302000865CC0008F3
:10016000430200084302000843020008430200085B
:100170004302000843020008430200080000000098
:10018000430200084302000800F002F800F03CF8C7
:100190000AA090E8000C82448344AAF10107DA45E2
:1001A00001D100F031F8AFF2090EBAE80F0013F0F8
:1001B000010F18BFFB1A43F0010318476843010001
:1001C00088430100103A24BF78C878C1FAD8520792
:1001D00024BF30C830C144BF04680C6070470000C1
:1001E0000023002400250026103A28BF78C1FBD840
:1001F000520728BF30C148BF0B6070471FB513F0CE
:10020000A6FF1FBD10B510BD00F062F91146FFF743
:10021000F5FF0CF0DDFF00F080F903B4FFF7F2FF0B
:1002200003BC00F083F900000948804709480047F3
:10023000FEE7FEE7FEE7FEE7FEE7FEE7FEE7FEE796
:10024000FEE7FEE704480549054A064B70470000F3
:10025000C1B9000889010008B8580020B85E002024
:10026000B85A0020B85A002053EA020C00F0698006
:100270002DE9F04B4FF00006002B1FBFB3FA83F5BA
:1002800003FA05F424FA05F65E4012BF1643B2FAEB
:1002900082F502FA05F4C5F120051EBF22FA05FC1D
:1002A00044EA0C04203556EA044C4FEA144418BFC3
:1002B000641C4FF000084FF00009904271EB030CF2
:1002C00039D3002919BFB1FA81F701FA07F6B0FA5C
:1002D00080F700FA07F6C7F120071EBF20FA07FCD7
:1002E00046EA0C062037B6FBF4FCA7EB0507103FE7
:1002F00007F01F0BCBF120062CFA06F60CFA0BFBCD
:1003000044BFB3460026202FA4BF5E464FF0000B2B
:100310005BEA060C08BF4FF0010B19EB0B0948EB29
:100320000608ABFB027C06FB02CC0BFB03CCC01B1C
:1003300071EB0C01C1E70B46024641464846BDE859
:10034000F08B13B5084318BF4FF0FF300146AFF3F1
:100350000080BDE81C407047032A40F2308010F056
:10036000030C00F0158011F8013BBCF1020F624450
:1003700098BF11F801CB00F8013B38BF11F8013BE1
:10038000A2F1040298BF00F801CB38BF00F8013B8E
:1003900011F0030300F06280083AC0F0088051F8C1
:1003A000043B083A51F804CBA0E80810F5E7121D09
:1003B0005CBF51F8043B40F8043BAFF30080D20728
:1003C00024BF11F8013B11F801CB48BF11F8012BF4
:1003D00024BF00F8013B00F801CB48BF00F8012B17
:1003E000704702F0FF0343EA032242EA024200F0B0
:1003F00002B84FF0000200B51346944696462039E5
:1004000022BFA0E80C50A0E80C50B1F12001BFF4CD
:10041000F7AF090728BFA0E80C5048BF0CC05DF833
:1004200004EB890028BF40F8042B08BF704748BF81
:1004300020F8022B11F0804F18BF00F8012B7047F5
:1004400070477047704710B500F03AF8006810BD6B
:1004500010B5044600F034F8046010BD10B5203A21
:10046000C0F00B80B1E81850A0E81850B1E818505F
:10047000A0E81850203ABFF4F5AF5FEA027C24BF31
:10048000B1E81850A0E8185044BF18C918C0BDE81A
:1004900010405FEA827C24BF51F8043B40F8043BE3
:1004A00008BF7047D20728BF31F8023B48BF11F898
:1004B000012B28BF20F8023B48BF00F8012B7047F2
:1004C00000487047080100200048704708010020DC
:1004D0007546FFF7F9FFAE4605006946534620F022
:1004E0000700854618B020B5FFF7ACFEBDE82040F8
:1004F0004FF000064FF000074FF000084FF0000BE0
:10050000AC46ACE8C009ACE8C009ACE8C009ACE84E
:10051000C00921F007018D46704710B50446AFF3BE
:1005200000802046BDE81040FFF777BE0149182043
:10053000ABBEFEE7260002007047000080B58AB01F
:1005400008900791089820B9FFE7FF208DF8270051
:100550009BE0079820B9FFE7FF208DF8270094E083
:10056000079890ED000A90ED013A90ED021A90ED97
:10057000032A20EE030A21EE021A30EE010A30EEC1
:10058000000A8DED060A079890ED010A90ED021A17
:1005900020EE000A21EE011A30EE010A30EE001AB8
:1005A000B7EE000A8DED010A30EE410A8DED050A25
:1005B0009DED060ADDED050A11F0B2FC9DED011A74
:1005C000089880ED010A079890ED000A90ED013A35
:1005D00090ED024A90ED032A20EE040A22EE032A4F
:1005E00030EE420A30EE000A8DED040A9DED040A59
:1005F000B0EEC00AB4EE410AF1EE10FA0ADBFFE7F2
:10060000DDED040A9FED230A0CF056FD089880EDFD
:10061000020A07E09DED040A11F080F9089880EDC8
:10062000020AFFE7079890ED000A90ED011A90ED9D
:10063000022A90ED033A20EE030A21EE021A30EE70
:10064000010A30EE000A8DED030A079890ED020AC8
:1006500090ED031A20EE000A21EE011A30EE010A95
:1006600030EE001AB7EE000A30EE410A8DED020AB4
:100670009DED030ADDED020A11F052FC089880EDB1
:10068000000A00208DF82700FFE79DF927000AB037
:1006900080BD00BFDB0FC93F80B58CB00A900991C7
:1006A0008DED080A0A9820B9FFE7FF208DF82F008A
:1006B00029E19DED081AB7EE000A80EE010A0A98BA
:1006C00080ED040A0A994FF07E5008600A990020D4
:1006D00048600A9988600A99C8600998002800F063
:1006E0000E81FFE7099801680091406813F064FCEF
:1006F0000246009801920A46019942EC101B8DEDCA
:10070000020B13F059FC9DED020B41EC110B11F0A3
:1007100007FB8DED040B9DF8170080F080008DF82D
:1007200017000498059912F05FFD0790099890ED65
:10073000000AB5EE400AF1EE10FA2BD1FFE7099856
:1007400090ED010AB5EE400AF1EE10FA22D1FFE772
:10075000099890ED020AB5EE400AF1EE10FA19D1AF
:10076000FFE70A9940F2C560C3F64D7008600A9928
:1007700044F62D20C3F60D4048600A994AF25640CF
:10078000CBF6393088600A9944F2AD70C3F619701F
:10079000C860B3E09DED070A9FED5D1AB4EE410A13
:1007A000F1EE10FA08DBFFE79DED070AB5EE400A0F
:1007B000F1EE10FA19DDFFE70A9945F66E10C3F65F
:1007C0007F7008600A9945F20C30C3F6B01048609B
:1007D0000A9948F6AB00CBF6BB3088600A9949F21B
:1007E0008550C3F69750C86087E09DED070A9FEDDE
:1007F000491AB4EE410AF1EE10FA0ADBFFE79DED6B
:10080000070A9FED431AB4EE410AF1EE10FA19DD22
:10081000FFE70A9940F2C560C3F64D7008600A9977
:1008200044F62D20C3F60D4048600A994AF256401E
:10083000CBF6393088600A9944F2AD70C3F619706E
:10084000C86059E09DED070A9FED331AB4EE410AE6
:10085000F1EE10FA0ADBFFE79DED070A9FED2D1A76
:10086000B4EE410AF1EE10FA19DDFFE70A9940F201
:10087000C560C3F64D7008600A9944F62D20C3F692
:100880000D4048600A994AF25640CBF639308860EC
:100890000A9944F2AD70C3F61970C8602BE09DED63
:1008A000070A9FED1D1AB4EE410AF1EE10FA08DBBB
:1008B000FFE79DED070AB5EE400AF1EE10FA19DDEB
:1008C000FFE70A9940F2C560C3F64D7008600A99C7
:1008D00044F62D20C3F60D4048600A994AF256406E
:1008E000CBF6393088600A9944F2AD70C3F61970BE
:1008F000C860FFE7FFE7FFE7FFE7FFE7FFE700204C
:100900008DF82F00FFE79DF92F000CB080BD00BFD0
:10091000DB0FC93FDB0F49400000B44280B52DED2D
:10092000048BB2B030902F912E922D93309828B92D
:10093000FFE7FF208DF8C70000F0F7BD2F9828B91A
:10094000FFE7FF208DF8C70000F0EFBD2E9828B913
:10095000FFE7FF208DF8C70000F0E7BD40F204017B
:10096000C2F200014EF69E70C3F6275008602D9823
:1009700048B9FFE730982F992E9A00F0DDFD8DF8E9
:10098000C70000F0D2BD2D98006809902D984068EE
:1009900008902D98806807909DED090AB5EE400AF1
:1009A000F1EE10FA19D1FFE79DED080AB5EE400A05
:1009B000F1EE10FA11D1FFE79DED070AB5EE400AFE
:1009C000F1EE10FA09D1FFE730982F992E9A00F036
:1009D000B3FD8DF8C70000F0A8BD2F980068069001
:1009E0002F98406805902F98806804902E98006892
:1009F00003902E98406802902E988068019030985D
:100A00009DED033A90ED010A90ED022A90ED031A54
:100A100020EE430A9DED023A22EE032A30EE420A0E
:100A20009DED012A21EE021A30EE410AB6EE001ABF
:100A300020EE010A8DED270A30989DED034A90EDD6
:100A4000000A90ED023A90ED032A20EE040A9DED93
:100A5000014A23EE043A30EE030A9DED023A22EEFB
:100A6000032A30EE420A20EE010A8DED260A309864
:100A70009DED024A90ED000A90ED013A90ED032AB7
:100A800020EE040A9DED014A23EE043A30EE430ABB
:100A90009DED033A22EE032A30EE020A20EE010A0F
:100AA0008DED250A30989DED014A90ED000A90EDFC
:100AB000013A90ED022A20EE040A9DED024A23EE4F
:100AC000043A30EE030A9DED033A22EE032A30EE9B
:100AD000420A20EE010A8DED240A9DED060AB5EECC
:100AE000400AF1EE10FA11D1FFE79DED050AB5EECF
:100AF000400AF1EE10FA09D1FFE79DED040AB5EEC8
:100B0000400AF1EE10FA00F09984FFE79DED060A25
:100B100020EE000A9DED051A21EE011A30EE010AC1
:100B20009DED041A21EE011A30EE010A08F006FFCD
:100B30008DED2C0A9DED2C1A9DED060A20EE010A82
:100B40008DED060A9DED2C1A9DED050A20EE010A99
:100B50008DED050A9DED2C1A9DED040A20EE010A8B
:100B60008DED040A9DED090A20EE000A9DED081A9C
:100B700021EE011A30EE010A9DED071A21EE011A4D
:100B800030EE010A08F0DAFE8DED2C0A9DED2C1AEC
:100B90009DED090A20EE010A8DED090A9DED2C1A42
:100BA0009DED080A20EE010A8DED080A9DED2C1A34
:100BB0009DED070A20EE010A8DED070A309890EDB1
:100BC000000A30EE000A9DED091A20EE010A8DEDB3
:100BD000210A309890ED000A30EE000A9DED081AC7
:100BE00020EE010A8DED200A309890ED000A30EEDB
:100BF000000A9DED071A20EE010A8DED1F0A3098BC
:100C000090ED010A30EE000A9DED091A20EE010A6E
:100C10008DED1E0A309890ED000A30EE000A8DED41
:100C2000190A309890ED010A30EE000A8DED180A8D
:100C3000309890ED020A30EE000A8DED170A3098D8
:100C400090ED030A30EE000A8DED160A309890ED13
:100C5000000A90ED021A30EE000A20EE010A8DED36
:100C6000150A309890ED020A90ED031A30EE000A52
:100C700020EE010A8DED140A309890ED000A20EE66
:100C8000000A8DED130A309890ED000A90ED011ADC
:100C900020EE010A8DED120A309890ED000A90EDD9
:100CA000021A20EE010A8DED110A309890ED000A2B
:100CB00090ED031A20EE010A8DED100A309890EDA8
:100CC000010A20EE000A8DED0F0A309890ED010A1E
:100CD00090ED021A20EE010A8DED0E0A309890ED8B
:100CE000010A90ED031A20EE010A8DED0D0A3098ED
:100CF00090ED020A20EE000A8DED0C0A309890ED7E
:100D0000020A90ED031A20EE010A8DED0B0A3098CD
:100D100090ED030A20EE000A8DED0A0A9DED091AF6
:100D20009DED130A21EE000A9DED202A309890EDEA
:100D3000025A90ED033A22EE032A30EE420A9DED6C
:100D40001F2A22EE052A30EE020A9DED0F2A21EE1F
:100D5000022A30EE020A9DED182A9DED084A22EE85
:100D6000044A24EE054A30EE040A9DED074A22EEBD
:100D7000042A22EE032A30EE020A9DED0C2A21EE0F
:100D8000022A30EE420A9DED0A2A21EE021A30EEC6
:100D9000410A8DED230A9DED210A309890ED015A0C
:100DA00090ED024A90ED033A20EE030A9DED081AF9
:100DB0009DED132A21EE022A30EE020A9DED1F2A34
:100DC00022EE052A30EE420A9DED1E2A22EE042A6A
:100DD00030EE020A9DED0F2A21EE022A30EE420A81
:100DE0009DED0C2A21EE022A30EE020A9DED172A13
:100DF0009DED074A22EE042A22EE032A30EE020A73
:100E00009DED0A2A21EE021A30EE410A8DED220AEA
:100E10009DED230A20EE000A9DED221A21EE011A13
:100E200030EE010A08F08AFDB7EE006A86EE000A8D
:100E30008DED1D0A9DED210A309890ED012A90ED6F
:100E4000021A90ED033A20EE011A9DED200A20EEE1
:100E5000020A30EE412A9DED071A9DED130A21EE9C
:100E6000000A30EE022A9DED1E0A20EE030A30EE43
:100E7000020A9DED0F2A21EE022A30EE420A9DED74
:100E8000172A9DED084A22EE042A22EE032A30EEAC
:100E9000020A9DED0C2A21EE022A30EE420A9DED57
:100EA0000A2A21EE021A30EE010A8DED1C0A9DED90
:100EB0001D0A30EE000A8DED1B0A9DED1C0A30EE76
:100EC000000A8DED1A0A9DED170ADDED0D0A30EED0
:100ED000A02A9DED151A31EE422A9DED061A31EE3B
:100EE000021A20EE010A9DED181ADDED123A33EEDA
:100EF000A32A9DED143A32EE032A9DED053A32EE17
:100F0000432A21EE021A70EE014A9DED1C3A3098F8
:100F100090ED011A90ED020AD0ED032A63EE001A5B
:100F20009DED1D2A9DED0C7AB6EE004A8DED004A2E
:100F300077EE445A9DED0A5A35EE255A62EE055A6F
:100F40009DED115A75EE606A63EE266A75EEA66A2B
:100F5000DDED095A75EEA65A61EEA51A71EEA41AD6
:100F600062EE222A23EE011A31EE621ADDED0E2A1C
:100F7000DDED104A72EEE42A62EE222ADDED0B4A24
:100F800073EEA43A63EE233A72EEA32ADDED083A3B
:100F900072EEE32A21EE221A31EE211A22EE000A25
:100FA00035EE205A22EE052A9DED0F5A34EE455AB1
:100FB00035EE475A23EE053A32EE032A9DED073A05
:100FC00032EE432A20EE020A30EE010A8DED2B0AA2
:100FD0009DED160ADDED0D2A32EEA21A9DED152AC1
:100FE00031EE421A9DED062A31EE421A20EE010A38
:100FF0009DED191ADDED126A36EEA62A9DED143A22
:1010000032EE032A9DED053A32EE432A21EE021A12
:1010100030EE011A3098D0ED005AD0ED014AD0EDF3
:10102000023A90ED032AB1EE000A24EE803A9DEDDB
:101030000F7A37EE075A75EE461ADDED0C0A30EEE0
:10104000A05A75EE211A9DED045A35EE215A23EE71
:10105000053A31EE031A9DED1C5A65EE027A9DEDBC
:101060001D3A74EE601A9DED0A8A71EEC81A23EEDD
:10107000218ADDED111A32EEE19A25EE099A38EE59
:10108000098A9DED099A38EE498A67EE887A31EE31
:10109000271A63EE233A65EE255A73EEA53ADDED85
:1010A0000E5ADDED107A75EEE75A63EE255ADDED46
:1010B0000B7A76EEA76A65EE266A75EEA65ADDED26
:1010C000086A75EEE65A63EEA53A31EE231A23EE6E
:1010D000022ADDED1A3A63EEA43A32EE632A71EE8B
:1010E000A21A23EE213A34EE477A37EE607A25EEE3
:1010F000075A33EE053A9DED075A33EE453A22EE94
:10110000032A31EE021A8DED2A1A9DED191ADDED32
:101110000D0A30EEA03A9DED152A32EE433A9DEDD0
:10112000062A32EE032A21EE021A9DED162ADDED83
:10113000124A34EEA43A9DED145A33EE053A9DED71
:10114000055A33EE453A22EE032A31EE022A309850
:1011500090ED001AD0ED011AD0ED022AD0ED033A3D
:1011600022EE800A9DED0F5A35EE053A33EE467AAF
:101170009DED0C6A36EE063A33EE077A9DED043AA1
:1011800033EE073A20EE030A70EE025A9DED1B0A79
:1011900020EE620A9DED1C3A23EE012A30EE420A4F
:1011A0009DED1D2A34EE467ADDED0A6A37EE667A49
:1011B00062EE076A9DED117A70EEC77A63EE277AC8
:1011C00076EEA76ADDED097A76EEE76A20EE260A6A
:1011D00030EE250A62EE211A63EE233A71EEA31A6D
:1011E000DDED0E3ADDED105A73EEE53A62EE233A8C
:1011F000DDED0B5A74EEA54A63EE244A73EEA43A71
:10120000DDED084A73EEE43A61EEA31A30EE210AEE
:1012100022EE011ADDED1A1A61EEA21A31EE611A00
:1012200037EE207A22EE072A34EE455A35EE465A3A
:1012300023EE053A32EE032A9DED073A32EE432AB9
:1012400021EE021A30EE010A8DED290A9DED180AF1
:101250009DED0D7A37EE071A9DED152A31EE421AF3
:101260009DED062A31EE421A20EE010A9DED171A75
:10127000DDED122A32EEA22A9DED143A32EE032A57
:101280009DED053A32EE432A21EE021A70EE013A44
:101290009DED1B1A3098D0ED001A90ED010AD0EDAB
:1012A000020A90ED032A21EE022A9DED1C3A23EE5C
:1012B000001A31EE421A9DED1D2A9DED0C5A34EEB6
:1012C000456ADDED0A4A36EE646A62EE064A9DED35
:1012D000116A77EE465A63EE255A74EEA54ADDEDA3
:1012E000095A74EEE54A21EE241A31EE231A62EE11
:1012F000211A63EE200A70EEE10ADDED0E1ADDED33
:10130000103A71EEE31A62EE211ADDED0B3A72EE3D
:10131000A32A63EE222A71EEA21ADDED082A71EEED
:10132000E21A60EEA10A31EE201A22EE000A36EE31
:10133000076A22EE062A9DED0F6A34EE464A34EE25
:10134000454A23EE043A32EE032A9DED073A32EE87
:10135000432A20EE020A30EE010A8DED280A9DEDA7
:101360002B0A20EE000A9DED2A1A21EE011A30EE1A
:10137000010A9DED291A21EE011A30EE010A9DEDB8
:10138000281A21EE011A30EE010A08F0D7FA8DED85
:101390002C0A9DED2C1A9DED2B0A20EE010A8DEDF5
:1013A0002B0A9DED2C1A9DED2A0A20EE010A8DEDE7
:1013B0002A0A9DED2C1A9DED290A20EE010A8DEDD9
:1013C000290A9DED2C1A9DED280A20EE010A8DEDCB
:1013D000280A40F20400C2F2000090ED000A9DEDE0
:1013E0002B1A20EE011A9DED270A30EE410A8DEDF1
:1013F000270A90ED000A9DED2A1A20EE011A9DEDB4
:10140000260A30EE410A8DED260A90ED000A9DED88
:10141000291A20EE011A9DED250A30EE410A8DEDC4
:10142000250A90ED000A9DED281A20EE011A9DED87
:10143000240A30EE410A8DED240AFFE79DED271ABC
:10144000309890ED000A90ED042A21EE021A30EE59
:10145000010A80ED000A9DED261A309890ED010AF0
:1014600090ED042A21EE021A30EE010A80ED010A05
:101470009DED251A309890ED020A90ED042A21EE98
:10148000021A30EE010A80ED020A9DED241A30980E
:1014900090ED030A90ED042A21EE021A30EE010AC3
:1014A00080ED030A309890ED000A90ED013A90ED3E
:1014B000022A90ED031A20EE000A23EE033A30EEE2
:1014C000030A22EE022A30EE020A21EE011A30EE61
:1014D000010A08F033FA8DED2C0A9DED2C1A309894
:1014E00090ED000A20EE010A80ED000A9DED2C1A15
:1014F000309890ED010A20EE010A80ED010A9DED81
:101500002C1A309890ED020A20EE010A80ED020AB2
:101510009DED2C1A309890ED030A20EE010A80ED23
:10152000030A00208DF8C700FFE79DF9C70032B01D
:10153000BDEC048B80BD000080B5A0B01E901D9155
:101540001C921E9820B9FFE7FF208DF87F00D3E2A0
:101550001D9820B9FFE7FF208DF87F00CCE21C9892
:1015600020B9FFE7FF208DF87F00C5E240F20401BB
:10157000C2F2000142F60230C3F6075008601D981F
:1015800000681B901D9840681A901D9880681990FB
:101590001C98006818901C98406817901C988068E8
:1015A00016901E989DED183A90ED010A90ED022AD2
:1015B00090ED031A20EE430A9DED173A22EE032A1E
:1015C00030EE420A9DED162A21EE021A30EE410A53
:1015D000B6EE001A20EE010A8DED100A1E989DED60
:1015E000184A90ED000A90ED023A90ED032A20EEA1
:1015F000040A9DED164A23EE043A30EE030A9DEDEF
:10160000173A22EE032A30EE420A20EE010A8DED4F
:101610000F0A1E989DED174A90ED000A90ED013AD1
:1016200090ED032A20EE040A9DED164A23EE043ABB
:1016300030EE430A9DED183A22EE032A30EE020AFC
:1016400020EE010A8DED0E0A1E989DED164A90EDD2
:10165000000A90ED013A90ED022A20EE040A9DED79
:10166000174A23EE043A30EE030A9DED183A22EEB3
:10167000032A30EE420A20EE010A8DED0D0A9DED9F
:101680001B0AB5EE400AF1EE10FA11D1FFE79DED0D
:101690001A0AB5EE400AF1EE10FA09D1FFE79DED06
:1016A000190AB5EE400AF1EE10FA00F0AE81FFE73C
:1016B0009DED1B0A20EE000A9DED1A1A21EE011A7B
:1016C00030EE010A9DED191A21EE011A30EE010AE1
:1016D00008F034F98DED150A9DED151A9DED1B0AE4
:1016E00020EE010A8DED1B0A9DED151A9DED1A0ADB
:1016F00020EE010A8DED1A0A9DED151A9DED190ACD
:1017000020EE010A8DED190A1E9890ED000A30EEC8
:10171000000A8DED0C0A1E9890ED010A30EE000AC9
:101720008DED0B0A1E9890ED020A30EE000A8DED49
:101730000A0A1E9890ED030A30EE000A8DED090AA0
:101740001E9890ED000AB1EE003A20EE030A8DEDEE
:10175000080A1E9890ED010A20EE030A8DED070A93
:101760001E9890ED020A20EE030A8DED060A1E98DF
:1017700090ED010AB2EE001A20EE010A8DED050A85
:101780001E9890ED020A20EE010A8DED040A1E98C3
:1017900090ED000A20EE000A8DED030A1E9890EDF0
:1017A000010A20EE000A8DED020A1E9890ED020A51
:1017B00020EE000A8DED010A1E9890ED030A20EE3E
:1017C000000A8DED000A9DED081A9DED010A21EE3B
:1017D000000A9DED0A2A9DED1B4A22EE042A30EEF6
:1017E000020A9DED022A21EE021A30EE010A9DED59
:1017F0000B1A9DED1A2A21EE021A30EE410A8DEDE8
:10180000140A9DED071A9DED000A21EE000A9DEDD8
:10181000092A9DED1B4A22EE042A30EE420A9DED74
:10182000032A22EE032A1E9890ED014A22EE042A92
:1018300030EE020A9DED0C2A9DED1A4A22EE042A92
:1018400030EE420A30EE410A9DED052A9DED024A36
:1018500022EE044A30EE040A9DED014A22EE042AEB
:1018600030EE020A9DED192A21EE021A30EE010A2D
:101870008DED130A9DED030A20EE030A1E9890EDEC
:10188000021A20EE010A9DED0C1A9DED1B2A21EE95
:10189000021A30EE010A9DED061A9DED002A21EE96
:1018A000022A30EE020A9DED092A9DED1A4A22EE27
:1018B000042A30EE420A30EE410A9DED042A9DEDE5
:1018C000024A22EE044A30EE040A9DED014A22EE5D
:1018D000042A30EE020A9DED192A21EE021A30EE9A
:1018E000010A8DED120A9DED020A20EE030A1E98F0
:1018F00090ED032A20EE020A9DED0B1A9DED1B4A86
:1019000021EE041A30EE410A9DED011A21EE031A70
:1019100021EE021A30EE010A9DED0A1A9DED1A2AF7
:1019200021EE021A30EE410A8DED110A9DED140AE6
:1019300020EE000A9DED131A21EE011A30EE010A85
:101940009DED121A21EE011A30EE010A9DED111AD9
:1019500021EE011A30EE010A07F0F0FF8DED150AB5
:101960009DED151A9DED140A20EE010A8DED140A65
:101970009DED151A9DED130A20EE010A8DED130A57
:101980009DED151A9DED120A20EE010A8DED120A49
:101990009DED151A9DED110A20EE010A8DED110A3B
:1019A00040F20400C2F2000090ED000A9DED141A0E
:1019B00020EE011A9DED100A30EE410A8DED100A5D
:1019C00090ED000A9DED131A20EE011A9DED0F0A0D
:1019D00030EE410A8DED0F0A90ED000A9DED121ACE
:1019E00020EE011A9DED0E0A30EE410A8DED0E0A31
:1019F00090ED000A9DED111A20EE011A9DED0D0AE1
:101A000030EE410A8DED0D0AFFE79DED101A1E988C
:101A100090ED000A90ED042A21EE021A30EE010A40
:101A200080ED000A9DED0F1A1E9890ED010A90EDD1
:101A3000042A21EE021A30EE010A80ED010A9DED22
:101A40000E1A1E9890ED020A90ED042A21EE021A59
:101A500030EE010A80ED020A9DED0D1A1E9890ED00
:101A6000030A90ED042A21EE021A30EE010A80EDFD
:101A7000030A1E9890ED000A90ED013A90ED022ABB
:101A800090ED031A20EE000A23EE033A30EE030A2B
:101A900022EE022A30EE020A21EE011A30EE010A8D
:101AA00007F04CFF8DED150A9DED151A1E9890ED6F
:101AB000000A20EE010A80ED000A9DED151A1E981D
:101AC00090ED010A20EE010A80ED010A9DED151A44
:101AD0001E9890ED020A20EE010A80ED020A9DEDAB
:101AE000151A1E9890ED030A20EE010A80ED030AF4
:101AF00000208DF87F00FFE79DF97F0020B080BDBA
:101B000084B08DED030ACDED020A9DED030A9DED33
:101B1000021AB1EE411AB4EE410AF1EE10FA07DAF8
:101B2000FFE79DED020AB1EE400A8DED010A18E0D3
:101B30009DED030A9DED021AB4EE410AF1EE10FA92
:101B400005DDFFE79DED020A8DED000A04E09DED45
:101B5000030A8DED000AFFE79DED000A8DED010AF5
:101B6000FFE79DED010A04B07047000080B541F227
:101B7000D040C2F20000006808210BF033FF80BDA6
:101B800080B582B040F2D822C2F20002002001905B
:101B90001221132300F02CFA019802B080BD00003E
:101BA00080B5022001214FF0FF320BF06DFF80BDA8
:101BB00081B000909FED010A01B070470000C8435A
:101BC00080B541F2D040C2F20000006810210BF055
:101BD00009FF80BD80B540F2D820C2F20000C21DCE
:101BE00001200221062300F003FA002080BD00003E
:101BF00080B5042001214FF0FF320BF045FF80BD7E
:101C000080B58AB008900791089820B9FFE7FE20B8
:101C10008DF82700B4E0079820B9FFE7FE208DF883
:101C20002700ADE040F60560C2F200000078C00772
:101C300020B1FFE7FD208DF82700A1E00BF0B2FFF7
:101C400041F2D041C2F20001086020B9FFE7FE2056
:101C50008DF8270094E007980899C8620020069044
:101C60007E21B622049200F059FA049A0120142130
:101C700000F054FA1E20059001F06EF905990698BF
:101C800000F0F2F90699084600F0EEF91E2804D09B
:101C9000FFE7FC208DF8270072E00120002100F012
:101CA000E3F90F2804D0FFE7FC208DF8270067E058
:101CB0000320019000F0E6FE0420029000F0E2FE16
:101CC00041F69572C0F600020020039001210091B8
:101CD00001F0E0F8019841F66D31C0F6000100F026
:101CE0004BFF029841F6C131C0F6000100F044FFFD
:101CF00003984021AA2200F011FA009A039841218A
:101D000000F00CFA03985321082200F007FA029A17
:101D10000398582100F002FA029A03987D2100F0FE
:101D2000FDF9322001F018F9009A0F21104600F059
:101D3000F5F90098019A102100F0F0F90098039A43
:101D4000162100F0EBF9009A1821104600F0E6F990
:101D500000981521802200F0E1F90A2001F0FCF83A
:101D60000099019840F60562C2F20002117000F07D
:101D7000B3FE029800F0B0FE03988DF82700FFE74D
:101D80009DF927000AB080BD84B00290029820B966
:101D9000FFE7FE208DF80F006AE040F2D821C2F282
:101DA0000001B1F80100ADF80600B1F80300ADF88C
:101DB0000400B1F80500ADF80200BDF9060000EE20
:101DC000100AB8EEC00A029880ED040ABDF90400BA
:101DD00000EE100AB8EEC00A029880ED050ABDF9BF
:101DE000020000EE100AB8EEC00A029880ED060A62
:101DF000029890ED040A9FED201A80EE010A80ED12
:101E0000040A029890ED050A80EE010A80ED050AA9
:101E1000029890ED060A80EE010A80ED060A487CE1
:101E2000897CC00040EA5110ADF80000BDF9000007
:101E3000B0F5806F07DBFFE7BDF80000A0F500609C
:101E4000ADF80000FFE7BDF9000000EE100AB8EEA3
:101E5000C00AB4EE001A20EE010AB3EE071A30EE03
:101E6000010A029880ED0A0A00208DF80F00FFE7B2
:101E70009DF90F0004B0704700A0AA4584B00290FD
:101E8000029820B9FFE7FE208DF80F007AE040F2BB
:101E9000D820C2F20000B0F80710ADF80610B0F874
:101EA0000910ADF80410B0F80B00ADF80200BDF950
:101EB000060000EE100AB8EEC00A029880ED070A8C
:101EC000BDF9040000EE100AB8EEC00A029880EDD9
:101ED000080ABDF9020000EE100AB8EEC00A029826
:101EE00080ED090A029890ED070A9FED281A80EE0E
:101EF000010A80ED070A029890ED080A80EE010AB7
:101F000080ED080A029890ED090A80EE010A80ED42
:101F1000090A029890ED070A9FED1D1A20EE010AAA
:101F200080ED070A029890ED080A20EE010A80ED84
:101F3000080A029890ED090A20EE010A80ED090ACC
:101F40000298C16A91ED001A90ED070A30EE410A3D
:101F500080ED070A0298C16A91ED011A90ED080A16
:101F600030EE410A80ED080A0298C16A91ED021A2A
:101F700090ED090A30EE410A80ED090AFE208DF845
:101F80000F00FFE79DF90F0004B070476F12034286
:101F900035FA8E3C80B5012000F0C8FD68B9FFE736
:101FA0000121084600F030FE41F2D040C2F20000AC
:101FB000006802210BF016FDFFE7022000F0B6FDDD
:101FC00068B9FFE70220012100F01EFE41F2D04077
:101FD000C2F20000006804210BF004FDFFE780BDA1
:101FE00080B5182001214FF0FF320BF04DFD80BD70
:101FF00080B586B08DF817008DF8161004928DF814
:102000000F30049808B9FFE72BE09DF81700014650
:10201000029120B1FFE70298012805D009E00120D4
:10202000002100F0F1FD04E00220002100F0ECFDB1
:10203000FFE79DF8160040F0800040F2EB21C2F26D
:10204000000108700122009200230193184600F05D
:1020500043FF009B019804999DF80F2000F0DAFEE1
:10206000FFE706B080BD000080B586B08DF8160091
:102070008DF81510012000F06FFF9DF81600014645
:10208000049120B1FFE70498012805D009E0012060
:10209000002100F0B9FD04E00220002100F0B4FDB1
:1020A000FFE79DF8150040F0800040F2EB21C2F2FE
:1020B000000101910870012200230293184600F0EC
:1020C0000BFF0199029B0222184600F0A3FE9DF827
:1020D00016000146039120B1FFE7039801280CD0B8
:1020E00017E00121084600F08FFD40F2EB20C2F21C
:1020F000000040788DF817000BE00220012100F06D
:1021000083FD40F2EB20C2F2000000788DF817004A
:10211000FFE79DF8170006B080BD000080B584B0D1
:102120008DF80F008DF80E108DF80D209DF80E0023
:1021300000F07F0040F2EB21C2F2000108709DF830
:102140000D004870012000F007FF9DF80F000146C8
:10215000029120B1FFE70298012805D009E0012093
:10216000002100F051FD04E00220002100F04CFDB0
:10217000FFE740F2EB21C2F20001022200231846E1
:1021800000F0AAFE9DF80F000146019120B1FFE783
:102190000198012805D009E00121084600F034FD2E
:1021A00004E00220012100F02FFDFFE704B080BD14
:1021B00080B586B08DF8160004918DF80F209DF83B
:1021C0000F0020B9FFE70A208DF80F00FFE741F26A
:1021D000D030C2F20000006864210BF0DFFA20B1B9
:1021E000FFE7FB208DF8170070E041F2CC30C2F21F
:1021F000000000680290FFE70298E0B1FFE7029854
:1022000000789DF81610884211D1FFE702984068C7
:10221000049988420BD1FFE741F2D030C2F20000AE
:1022200000680BF09FFBFF208DF817004EE002982E
:1022300000690290E0E7142000F00EFD0190019883
:1022400058B9FFE741F2D030C2F2000000680BF04D
:1022500089FBFE208DF8170038E09DF80F001C2147
:1022600000220BF099F9019988600198806870B993
:10227000FFE7019800F0FEFB41F2D030C2F200000F
:1022800000680BF06FFBFF208DF817001EE09DF833
:102290001600019908700498019948609DF80F0094
:1022A0000199087341F2CC31C2F200010868019A29
:1022B00010610198086041F2D030C2F2000000685D
:1022C0000BF050FB00208DF81700FFE79DF9170079
:1022D00006B080BD82B001908DF80310019802B065
:1022E0007047000084B08DF80B00019141F2CC30B2
:1022F000C2F2000000680090FFE70098A8B1FFE775
:10230000009800789DF80B1088420AD1FFE70098EA
:1023100040680199884204D1FFE7009880680390E3
:1023200006E0009800690090E7E700200390FFE7CF
:10233000039804B07047000082B000900098C06815
:10234000022809D1FFE7009881680220042908BF0C
:1023500003208DF8070008E0009880680438B0FA80
:1023600080F040098DF80700FFE79DF8070002B0F4
:102370007047000083B08DF807009DF80700022821
:1023800003DBFFE70020029018E09DF807000146FC
:10239000009120B1FFE70098012806D00BE040F63D
:1023A0002010C2F20000029008E040F64810C2F28D
:1023B0000000029002E000200290FFE7029803B0C4
:1023C0007047000080B586B08DF816000491039226
:1023D000029340F60460C2F200000078C00720B902
:1023E000FFE7FD208DF8170037E0039820B9FFE7DD
:1023F000FE208DF8170030E041F2D030C2F200002C
:10240000006864210BF0CAF920B1FFE7FB208DF8CA
:10241000170022E09DF816000499FFF763FF019072
:1024200041F2D030C2F2000000680BF09BFA019834
:1024300020B9FFE7FC208DF817000EE00198039902
:10244000029B00220BF048F800900098002818BF6B
:102450004FF0FF308DF81700FFE79DF9170006B029
:1024600080BD000080B592B040F60460C2F200006A
:102470000078C00720B1FFE7FD208DF8470074E029
:1024800040F26810C2F200006821FDF7B2FF40F68A
:10249000B851C2F2000142F2D520C0F60000086037
:1024A00000200BF0CBF9014641F2D030C2F200001F
:1024B0000160006820B9FFE7FF208DF8470054E075
:1024C00040F60461C2F200010491012005900870F9
:1024D00007A802902821FDF78CFF0299059A002099
:1024E00006900C90079008900D900E9209900A901B
:1024F0000F920E22019210920B9040F62010C2F221
:102500000000009002F0A4FA009803F08DF90698FC
:1025100042F28162C0F60002062100F04DF80098F8
:10252000032102F0BFF9019A029905980C920B90D1
:1025300040F64810C2F20000039002F089FA0398B6
:1025400003F072F9059842F26572C0F600020821A4
:1025500000F032F80398102102F0A4F9049A0599CA
:10256000069811708DF84700FFE79DF9470012B0FB
:1025700080BD000080B584B002908DF8071040F651
:10258000B850C2F20000006858B1FFE740F6B850FA
:10259000C2F20000026802989DF80710904703906D
:1025A00006E002989DF80710FFF794FE0390FFE7FE
:1025B000039804B080BD000082B08DF806008DF84D
:1025C0000510009240F60460C2F200000078C007D7
:1025D00020B9FFE7FD208DF807002AE0009820B918
:1025E000FFE7FE208DF8070023E09DF80600022893
:1025F00004DBFFE7FF208DF807001AE09DF80500D7
:102600000D2804DBFFE7FF208DF8070011E000989C
:102610009DF8061040F26813C2F20003342211FB49
:1026200002319DF8052041F8220000208DF80700B6
:10263000FFE79DF9070002B07047000080B584B045
:102640008DF80E0002918DF8072040F60460C2F26A
:1026500000000078C00720B9FFE7FD208DF80F00CB
:1026600009E09DF80E0002999DF80720FFF7A0FDF4
:102670008DF80F00FFE79DF90F0004B080BD00004A
:1026800080B598B000200E90FFE70E98012867DC17
:10269000FFE79DF83800FFF76DFE0D900D9808B923
:1026A000FFE759E0FFE70D98002102F0C9FA002882
:1026B00051D0FFE70D98002111AA0FAB02F0EAFA02
:1026C000002847D1FFE7139818B9FFE71198019048
:1026D00002E012980190FFE701980C9011A8FFF713
:1026E0002BFE8DF82F000C989DF82F10FFF742FF5E
:1026F0000A909DF838000A99FFF7F4FD09900998AF
:1027000038B3FFE7002008900790069005900490EA
:10271000039002909DF82F008DF808000C9803900C
:102720000A98049015988DF81400149838B9FFE7AA
:1027300002A80D30159A0FA9FDF70EFEFFE703F072
:102740008FFF0890099802A900231A460AF0A4FFF7
:10275000FFE7FFE7A7E7FFE70E9801300E9094E749
:1027600018B080BD80B598B000200E90FFE70E989D
:10277000012867DCFFE79DF83800FFF7FBFD0D90AF
:102780000D9808B9FFE759E0FFE70D98012102F025
:1027900057FA002851D0FFE70D98012111AA0FAB7D
:1027A00002F078FA002847D1FFE7139818B9FFE73D
:1027B0001198019002E012980190FFE701980C90A7
:1027C00011A8FFF7B9FD8DF82F000C989DF82F1078
:1027D000FFF7D0FE0A909DF838000A99FFF782FDB6
:1027E0000990099838B3FFE70020089007900690F9
:1027F00005900490039002909DF82F008DF808003A
:102800000C9803900A98049015988DF81400149869
:1028100038B9FFE702A80D30159A0FA9FDF79CFD06
:10282000FFE703F01DFF0890099802A900231A464C
:102830000AF032FFFFE7FFE7A7E7FFE70E98013056
:102840000E9094E718B080BD80B58EB08446109885
:102850008DF836C08DF835100C920B938DF82B0047
:1028600040F60460C2F200000078C00720B9FFE71C
:10287000FD208DF8370079E09DF83600022804DB52
:10288000FFE7FF208DF8370070E00B9870B9FFE785
:102890009DF83500022809D0FFE79DF83500032890
:1028A00004D0FFE7FE208DF837005FE09DF82B0095
:1028B000092804DBFFE7FF208DF8370056E09DF87C
:1028C0003600FFF757FD0990099820B9FFE7FE2071
:1028D0008DF837004AE00020089007900690059098
:1028E000049003909DF835000146009103281FD8FD
:1028F0000099DFE801F002080F160C980390002001
:102900000590069018E00C98049004200590002093
:10291000069011E00C98039000200590022006908C
:102920000AE00C980490042005900220069003E031
:10293000FF208DF8370019E09DF82B00079000204C
:102940008DF8200009980B9A03A902AB01F0D4FF7F
:102950008DF807009DF8070020B1FFE7FF208DF8F4
:10296000370003E000208DF83700FFE79DF93700BE
:102970000EB080BD80B584B08DF80E000291029833
:1029800020B9FFE7FE208DF80F000EE09DF80E0045
:1029900002990A684B1D0979EC46CCF80010002119
:1029A000FFF752FF8DF80F00FFE79DF90F0004B00D
:1029B00080BD000080B588B08DF81E00069140F6FD
:1029C0000460C2F200000078C00720B9FFE7FD20D4
:1029D0008DF81F004AE09DF81E00022804DBFFE787
:1029E000FF208DF81F0041E09DF81E00FFF7C2FC9C
:1029F0000590059820B9FFE7FE208DF81F0035E00F
:102A000003F02EFE0490069868B9FFE7059802F0DF
:102A10004BFA039003996FF00400002918BF0020BF
:102A20008DF81F0022E0FFE7059802F03DFA0290C2
:102A3000029820B1FFE700208DF81F0016E00698ED
:102A4000013078B1FFE703F00BFE0499401A0190C2
:102A500001980699884204D3FFE7FB208DF81F00F8
:102A600004E0FFE701200AF0FDFBDDE79DF91F0010
:102A700008B080BD80B582B0019001980CF0F4FCE4
:102A800002B080BD80B582B08DF806009DF80600CA
:102A90000146009140B1FFE70098032808D0FFE706
:102AA0000098042808D00BE0062003F06DFE0BE030
:102AB0000A2003F069FE07E0172003F065FE03E03B
:102AC000FF208DF8070003E000208DF80700FFE7E6
:102AD0009DF9070002B080BD80B582B08DF8060078
:102AE0009DF806000146009140B1FFE700980328D9
:102AF00008D0FFE70098042808D00BE0062003F078
:102B00004DFE0BE00A2003F049FE07E0172003F01A
:102B100045FE03E0FF208DF8070003E000208DF85C
:102B20000700FFE79DF9070002B080BD80B582B0C5
:102B30008DF806009DF80600082804DBFFE700205A
:102B40008DF8070013E09DF8062044F28031C0F6AE
:102B5000010101EBC200406831F8321003F050FD72
:102B60000138B0FA80F040098DF80700FFE79DF8C2
:102B7000070002B080BD000083B08DF80A0001910B
:102B8000019820B9FFE7FE208DF80B0038E09DF892
:102B90000A00082804DBFFE7FF208DF80B002FE078
:102BA0009DF80A1044F28030C0F6010030F8310080
:102BB000ADF8020000208DF80100FFE79DF801004C
:102BC0000F2819DCFFE7BDF802009DF80110C8408E
:102BD000C00750B1FFE701989DF8012040F2D011E5
:102BE000C2F2000141F8220006E0FFE79DF8010073
:102BF00001308DF80100E1E700208DF80B00FFE7C0
:102C00009DF90B0003B0704780B582B08DF80600C7
:102C10008DF805109DF80600082804DBFFE7FF206B
:102C20008DF8070014E09DF8062044F28031C0F6CC
:102C3000010101EBC200406831F832109DF8052017
:102C400002F0010203F0F4FC00208DF80700FFE71A
:102C50009DF9070002B080BD80B582B00190019857
:102C60000CF002F802B080BD86B08DF816008DED34
:102C7000040A9DF81600022804DBFFE7FF208DF808
:102C800017008CE09DED040AB7EE001AB4EE410A7D
:102C9000F1EE10FA04DDFFE74FF07E500490FFE7FD
:102CA0009DED040AB5EE400AF1EE10FA03DAFFE7F3
:102CB00000200490FFE79DF8161044F2C030C0F6E3
:102CC000010050F831100968C96A03919DED040AAA
:102CD0000399013101EE101AB8EE411A20EE010AF3
:102CE000BCEEC00A8DED020A9DF8161000EBC10083
:102CF000808860B9FFE702989DF8162044F2C03141
:102D0000C0F6010151F832100968486343E09DF8AC
:102D1000161044F2C030C0F6010000EBC1008088FC
:102D200004280DD1FFE702989DF8162044F2C03127
:102D3000C0F6010151F8321009688863019028E05B
:102D40009DF8161044F2C030C0F6010000EBC1003F
:102D5000808808280DD1FFE702989DF8162044F2DC
:102D6000C031C0F6010151F832100968C863009003
:102D70000CE002989DF8162044F2C031C0F6010123
:102D800051F83210096808640090FFE7009801903C
:102D9000FFE70198FFE700208DF81700FFE79DF996
:102DA000170006B07047000080B582B08DF80600AD
:102DB0009DF80600022804DBFFE7FF208DF80700DE
:102DC00010E09DF8062044F2C030C0F6010000EB90
:102DD000C20150F83200898806F002F800208DF810
:102DE0000700FFE79DF9070002B080BD82B08DF8B3
:102DF00003009DF8030030B9FFE740F6B030C2F29F
:102E00000000019002E000200190FFE7019802B06D
:102E10007047000080B584B08DF80E000291ADF8C7
:102E200006208DF805309DF80E00012804DBFFE731
:102E3000FF208DF80F0029E09DF80E00FFF7D6FF68
:102E40000090009820B9FFE7FF208DF80F001DE0EB
:102E50009DF80500C00760B1FFE700980299BDF832
:102E6000062004F093FC002818BF01208DF80F0005
:102E70000CE000980299BDF80620142304F05EFBD4
:102E8000002818BF01208DF80F00FFE79DF90F0003
:102E900004B080BD82B08DF806008DF80510009258
:102EA000009820B9FFE7FE208DF8070010E0009899
:102EB0009DF8062040F21821C2F2000101EB4211F8
:102EC0009DF8052041F8220000208DF80700FFE75B
:102ED0009DF9070002B0704780B584B08DF80E00F0
:102EE0000291ADF806208DF805309DF80E000128FE
:102EF00004DBFFE7FF208DF80F0029E09DF80E00AE
:102F0000FFF774FF0090009820B9FFE7FF208DF8CD
:102F10000F001DE09DF80500C00760B1FFE70098B5
:102F20000299BDF8062005F07FF9002818BF01209E
:102F30008DF80F000CE000980299BDF806201423CC
:102F400004F044FD002818BF01208DF80F00FFE7B2
:102F50009DF90F0004B080BD80B586B004900AF0E2
:102F600005FA01464FF47A70B0FBF1F00390049833
:102F70000399B0FBF1F002900AF0BAF90146481C3F
:102F8000019198B1FFE70198022820D3FFE701984B
:102F900002280FD0FFE701980338022806D3FFE785
:102FA00001986FF00041884215D1FFE7FF208DF8AE
:102FB000170014E0029818B1FFE70298009002E0B1
:102FC00001200090FFE700980AF04CF903E0049814
:102FD00003F0C8F8FFE700208DF81700FFE79DF920
:102FE000170006B080BD000080B58AB00AF0BEF9B7
:102FF00007900EF033F8079A4FF47A710191B1FB04
:10300000F2F1484306904EF21800CEF20000029012
:10301000006805900EF022F8019A01460298079B7D
:10302000B2FBF3F2514304910068039006980499AF
:10303000884215D1FFE704984FF47A7250430599FE
:1030400051434EF21402CEF2000212680132B1FB7B
:10305000F2F1401A00F57A7000210991089014E00D
:1030600004984FF47A725043039951434EF214027C
:10307000CEF2000212680132B1FBF2F1401A00F503
:103080007A70002109910890FFE7089809990AB021
:1030900080BD000080B582B0019001980068006892
:1030A000C00600282AD5FFE7FFE70020009001981E
:1030B00000680068009001980068406800900098DF
:1030C000FFE7019809F064FB00EBC00140F23820F3
:1030D000C2F2000000EB8100006A70B1FFE70198C6
:1030E00009F056FB00EBC00140F23820C2F20000AC
:1030F00000EB8100006A8047FFE7FFE702B080BD78
:10310000FFE7FEE780B540F62010C2F2000001F0B4
:1031100003FF80BD80B540F62010C2F2000001F030
:10312000FBFE80BD80B540F64810C2F2000001F001
:10313000F3FE80BD80B540F64810C2F2000001F0F9
:10314000EBFE80BD82B00090009820B9FFE703201D
:103150008DF807001DE00098006846F20041C4F2B7
:103160000001884204D1FFE700208DF8070010E03D
:103170000098006846F60001C4F20001884204D1BC
:10318000FFE701208DF8070003E003208DF807001A
:10319000FFE79DF8070002B07047000080B588B0D7
:1031A00006900591069818B1FFE7059820B9FFE74A
:1031B000FE208DF81F0014E1FFF716FF069A039218
:1031C00013685268C01A914110F04BFF01460398F2
:1031D00000EE101A9FED851A80EE010A80ED020ABA
:1031E000FFF702FF0A4606994A60086006980599AB
:1031F00000F000F920B1FFE7FD208DF81F00F0E09E
:103200000698007B0146029120B1FFE70298012851
:1032100008D026E0069900200861069948610699C1
:10322000886122E0059890ED020A90ED051A20EEE3
:10323000010A069880ED040A059890ED030A90EDC6
:10324000051A20EE010A069880ED050A059890ED12
:10325000040A90ED051A20EE010A069880ED060A90
:1032600003E0FD208DF81F00BBE0069901F24C4001
:1032700091ED040A06F09EFB069880ED040A06997B
:1032800001F26C4091ED050A06F094FB069880ED82
:10329000050A069901F28C4091ED060A06F08AFBB8
:1032A000069880ED060A0698059900F021F900209D
:1032B0000490FFE70498032800F38F80FFE7069847
:1032C000049900EB8101086D08660699049AC2EB27
:1032D000021001EB800000F5807001EB820292ED9C
:1032E000180AD2ED340AD1ED021A9FED411A8DED84
:1032F000011A07F00FFD9DED011A049840F6F00346
:10330000C2F2000303EB800080ED000A0699049AE4
:10331000C2EB021001EB800000F5F87003EB8203B2
:1033200093ED000A01EB8202D2ED300AD1ED021AD0
:1033300007F0F0FC0698049900EB810080ED200A6C
:103340000699049A01EB421000F22C5001EB820125
:1033500091ED200A06F02EFB9DED011A06980499C6
:1033600000EB810000F2CC5080ED000A0698049931
:1033700000EB8101086B08670699049AC2EB021002
:1033800001EB800000F5387001EB820292ED1C0A1F
:10339000D2ED280AD1ED021A07F0BCFC0698049978
:1033A00000EB810080ED240A0699049A01EB42109B
:1033B00000F2AC4001EB820191ED240A06F0FAFA2A
:1033C0000698049900EB810000F2BC5080ED000AE1
:1033D000FFE70498013004906CE700208DF81F008F
:1033E000FFE79DF91F0008B080BD00BF00247449AD
:1033F0000000000080B584B002900191029820B9CD
:10340000FFE7FE208DF80F0031E000200090FFE77D
:103410000098032823DCFFE702980099C1EB011113
:1034200000EB810000F5387007F0B8FE02980099B3
:10343000C1EB011100EB810000F5F87007F0AEFE62
:1034400002980099C1EB011100EB810000F580703A
:1034500007F0A4FEFFE7009801300090D8E701983C
:1034600000790299087300208DF80F00FFE79DF99D
:103470000F0004B080BD000080B582B00190002034
:103480000090FFE70098032823DCFFE70199D1F8BB
:103490002804009A00EBC200603001EB820101F2C7
:1034A000BC5191ED000A06F06DFE0199D1F8280497
:1034B000009A00EBC200803001EB820101F2CC5196
:1034C00091ED000A06F05EFEFFE7009801300090E3
:1034D000D8E70198D0F82804603006F01FFC019866
:1034E000D0F82804803006F019FC02B080BD00003E
:1034F00080B5ADF53C7DBB90BA91BB98007B0128AF
:103500007ED1FFE7BB98006910F056FD41EC100B2F
:103510009FED531B50EC111BC20F51EC100B62F3CB
:10352000DF7141EC100B51EC100B9FED4F0B53EC86
:10353000102B10F081FD002862D1FFE7BB98406995
:1035400010F03AFD41EC100B9FED451B50EC111BA8
:10355000C20F51EC100B62F3DF7141EC100B51EC18
:10356000100B9FED410B53EC102B10F065FD002864
:1035700046D1FFE7BB98806910F01EFD41EC100BAF
:103580009FED371B50EC111BC20F51EC100B62F377
:10359000DF7141EC100B51EC100B9FED330B53EC32
:1035A000102B10F049FD58BBFFE7BB9890F8D003F3
:1035B00028B9FFE7BB99012081F8D003FFE700207D
:1035C0008DF8E702FFE79DF8E702032816DCFFE726
:1035D000BB989DF8E71200EB8101D1F8AC050864B7
:1035E000BB989DF8E71200EB810100200862FFE71D
:1035F0009DF8E70201308DF8E702E4E700F0EABD4C
:10360000BB99002081F8D0038DF8E602FFE79DF812
:10361000E60203280FDCFFE7BB989DF8E61200EBFB
:103620008101086CC1F8AC05FFE79DF8E6020130A6
:103630008DF8E602EBE7BB98007B0146B5910028C8
:1036400000F08985FFE7B598012815D0FFE7B59808
:10365000022800F0A28500F0BCBD00BF00BF00BF83
:1036600000000000000000009A9999999999B93FCB
:10367000000000000000F03FBB980090006910F0CF
:103680009BFC0246009801920A46019942EC101BED
:103690008DED040B806910F08FFC41EC100B8DED6B
:1036A000020B1FED0D0B8DEDAA0B0EF0CDF90EF0F8
:1036B0001FFF9DED021B51EC110B53EC102B10F072
:1036C0000FF99DED040B41EC110B53EC112B51EC58
:1036D000100B0FF0BBFD41EC100B8DED0C0BBB99EB
:1036E00008698969069110F067FC024606980792FE
:1036F0000A46079942EC101B8DED0A0B10F05CFC9A
:103700009DEDAA0B41EC110B8DED081B0EF09CF901
:103710000EF0EEFE9DED081B51EC110B53EC102B3F
:1037200010F0DEF89DED0A0B41EC110B53EC112B60
:1037300051EC100B0FF08AFD9DED0C1B41EC100BB2
:1037400051EC110B53EC102B10F0CAF841EC100B9C
:103750008DED1C0BBB99486989690E9110F02CFC0A
:1037600002460E980F920A460F9942EC101B8DEDFF
:10377000120B10F021FC9DEDAA0B41EC110B8DED0D
:10378000101B0EF061F90EF023FD9DED101B51ECA6
:10379000110B53EC102B10F0A3F89DED120B41EC24
:1037A000110B53EC112B51EC100B0FF04FFD41ECB2
:1037B000100B8DED1A0BBB9948698969149110F0B3
:1037C000FBFB0246149815920A46159942EC101B11
:1037D0008DED180B10F0F0FB9DEDAA0B41EC110BD9
:1037E0008DED161B0EF030F90EF0F2FC9DED161B60
:1037F00051EC110B53EC102B10F072F89DED180BDF
:1038000041EC110B53EC112B51EC100B0FF01EFD82
:103810009DED1A1B41EC100B51EC110B53EC102BCE
:1038200010F05EF89DED1C1B41EC100B51EC110BE0
:1038300053EC102B0FF00AFD41EC100B0EF0BCFE08
:1038400051EC100B0FF0D0FCBB990862BB990869D2
:1038500089691E9110F0B0FB02461E981F920A461D
:103860001F9942EC101B8DED220B10F0A5FB9DED76
:10387000AA0B41EC110B8DED201B0EF0E5F80EF0BC
:1038800037FE9DED201B51EC110B53EC102B10F06B
:1038900027F89DED220B41EC110B53EC112B51EC51
:1038A000100B0FF0D3FC41EC100B8DED2A0BBB99E4
:1038B00008698969249110F07FFB024624982592BB
:1038C0000A46259942EC101B8DED280B10F074FB75
:1038D0009DEDAA0B41EC110B8DED261B0EF0B4F8FB
:1038E0000EF006FE9DED261B51EC110B53EC102B38
:1038F0000FF0F6FF9DED280B41EC110B53EC112B53
:1039000051EC100B0FF0A2FC9DED2A1B41EC100BAB
:1039100051EC110B53EC102B0FF0E2FF41EC100BAC
:103920008DED3A0BBB99486989692C9110F044FBE5
:1039300002462C982D920A462D9942EC101B8DEDD3
:10394000300B10F039FB9DEDAA0B41EC110B8DED06
:103950002E1B0EF079F80EF03BFC9DED2E1B51EC6A
:10396000110B53EC102B0FF0BBFF9DED300B41EC16
:10397000110B53EC112B51EC100B10F02FFA41EC02
:10398000100B8DED380BBB9948698969329110F0A5
:1039900013FB0246329833920A46339942EC101BCD
:1039A0008DED360B10F008FB9DEDAA0B41EC110BD1
:1039B0008DED341B0EF048F80EF00AFC9DED341B23
:1039C00051EC110B53EC102B0FF08AFF9DED360BD1
:1039D00041EC110B53EC112B51EC100B10F0FEF9D4
:1039E0009DED381B41EC100B51EC110B53EC102BDF
:1039F0000FF076FF9DED3A1B41EC100B51EC110BD3
:103A000053EC102B0FF022FC41EC100B0EF0D4FD08
:103A100051EC100B0FF0E8FBBB994862BB990869A9
:103A200089693C9110F0C8FA02463C983D920A46DA
:103A30003D9942EC101B8DED400B10F0BDFA9DED51
:103A4000AA0B41EC110B8DED3E1B0DF0FDFF0EF0AE
:103A50004FFD9DED3E1B51EC110B53EC102B0FF065
:103A60003FFF9DED400B41EC110B53EC112B51EC42
:103A7000100B10F0B3F941EC100B8DED480BBB9916
:103A800008698969429110F097FA02464298439278
:103A90000A46439942EC101B8DED460B10F08CFA50
:103AA0009DEDAA0B41EC110B8DED441B0DF0CCFFED
:103AB0000EF01EFD9DED441B51EC110B53EC102B31
:103AC0000FF00EFF9DED460B41EC110B53EC112B4B
:103AD00051EC100B10F082F99DED481B41EC100BDE
:103AE00051EC110B53EC102B0FF0FAFE41EC100BC4
:103AF0008DED580BBB99486989694A9110F05CFAC1
:103B000002464A984B920A464B9942EC101B8DEDA7
:103B10004E0B10F051FA9DEDAA0B41EC110B8DEDFF
:103B20004C1B0DF091FF0EF053FB9DED4C1B51EC27
:103B3000110B53EC102B0FF0D3FE9DED4E0B41EC0F
:103B4000110B53EC112B51EC100B10F047F941EC19
:103B5000100B8DED560BBB9948698969509110F097
:103B60002BFA0246509851920A46519942EC101B8A
:103B70008DED540B10F020FA9DEDAA0B41EC110BCA
:103B80008DED521B0DF060FF0EF022FB9DED521BE0
:103B900051EC110B53EC102B0FF0A2FE9DED540BCA
:103BA00041EC110B53EC112B51EC100B10F016F9EA
:103BB0009DED561B41EC100B51EC110B53EC102BEF
:103BC0000FF08EFE9DED581B41EC100B51EC110BCC
:103BD00053EC102B0FF03AFB41EC100B0EF0ECFC09
:103BE00051EC100B0FF000FBBB998862BB99086980
:103BF00089695A9110F0E0F902465A985B920A4698
:103C00005B9942EC101B8DED5E0B10F0D5F99DED2C
:103C1000AA0B41EC110B8DED5C1B0DF015FF0EF0A6
:103C200067FC9DED5C1B51EC110B53EC102B0FF05E
:103C300057FE9DED5E0B41EC110B53EC112B51EC3B
:103C4000100B10F0CBF841EC100B8DED660BBB990F
:103C500008698969609110F0AFF902466098619235
:103C60000A46619942EC101B8DED640B10F0A4F92B
:103C70009DEDAA0B41EC110B8DED621B0DF0E4FEE6
:103C80000EF036FC9DED621B51EC110B53EC102B2A
:103C90000FF026FE9DED640B41EC110B53EC112B44
:103CA00051EC100B10F09AF89DED661B41EC100BD7
:103CB00051EC110B53EC102B0FF012FE41EC100BDA
:103CC0008DED760BBB9948698969689110F074F99C
:103CD0000246689869920A46699942EC101B8DED7C
:103CE0006C0B10F069F99DEDAA0B41EC110B8DEDF9
:103CF0006A1B0DF0A9FE0EF06BFA9DED6A1B51ECEC
:103D0000110B53EC102B0FF0EBFD9DED6C0B41EC08
:103D1000110B53EC112B51EC100B0FF097FA41ECF7
:103D2000100B8DED740BBB99486989696E9110F089
:103D300043F902466E986F920A466F9942EC101B47
:103D40008DED720B10F038F99DEDAA0B41EC110BC3
:103D50008DED701B0DF078FE0EF03AFA9DED701BA4
:103D600051EC110B53EC102B0FF0BAFD9DED720BC3
:103D700041EC110B53EC112B51EC100B0FF066FAC8
:103D80009DED741B41EC100B51EC110B53EC102BFF
:103D90000FF0A6FD9DED761B41EC100B51EC110BC5
:103DA00053EC102B0FF052FA41EC100B0EF004FC08
:103DB00051EC100B0FF018FABB99C862BB99486917
:103DC0008969789110F0F8F80246789879920A4655
:103DD000799942EC101B8DED7C0B10F0EDF89DED08
:103DE000AA0B41EC110B8DED7A1B0DF02DFE0EF0A0
:103DF000EFF99DED7A1B51EC110B53EC102B0FF0EA
:103E00006FFD9DED7C0B41EC110B53EC112B51EC34
:103E1000100B0FF01BFA41EC100B8DED840BBB99CE
:103E2000086989697E9110F0C7F802467E987F92F2
:103E30000A467F9942EC101B8DED820B10F0BCF806
:103E40009DEDAA0B41EC110B8DED801B0DF0FCFDDF
:103E50000EF04EFB9DED801B51EC110B53EC102B23
:103E60000FF03EFD9DED820B41EC110B53EC112B3D
:103E700051EC100B0FF0EAF99DED840B41EC110BA6
:103E80000DF04EFF51EC100B9FEDED0B53EC102B92
:103E9000B493B3920FF024FD41EC100B51EC100BD6
:103EA0000FF0A2F9BB990864BB99486989698691AA
:103EB00010F082F80246869887920A46879942EC6B
:103EC000101B8DED8A0B10F077F89DEDAA0B41ECDD
:103ED000110B8DED881B0DF0B7FD0EF079F99DEDFE
:103EE000881B51EC110B53EC102B0FF0F9FC9DEDDE
:103EF0008A0B41EC110B53EC112B51EC100B0FF012
:103F00006DFF41EC100B8DED920BBB99086989692F
:103F10008C9110F051F802468C988D920A468D993A
:103F200042EC101B8DED900B10F046F89DEDAA0BA6
:103F300041EC110B8DED8E1B0DF086FD0EF0D8FAC5
:103F40009DED8E1B51EC110B53EC102B0FF0C8FCA8
:103F50009DED900B41EC110B53EC112B51EC100B20
:103F60000FF074F99DED920B41EC110B0DF0D8FEA2
:103F7000B39AB49B51EC100B0FF0B2FC41EC100B58
:103F800051EC100B0FF030F9BB994864BB994869AC
:103F90008969949110F010F80246949895920A4617
:103FA000959942EC101B8DED980B10F005F89DEDE6
:103FB000AA0B41EC110B8DED961B0DF045FD0EF09B
:103FC00007F99DED961B51EC110B53EC102B0FF0E4
:103FD00087FC9DED980B41EC110B53EC112B51EC30
:103FE000100B0FF0FBFE41EC100B8DEDA00BBB99FD
:103FF000086989699A910FF0DFFF02469A989B92AF
:104000000A469B9942EC101B8DED9E0B0FF0D4FFDE
:104010009DEDAA0B41EC110B8DED9C1B0DF014FDD9
:104020000EF066FA9DED9C1B51EC110B53EC102B1E
:104030000FF056FC9DED9E0B41EC110B53EC112B38
:1040400051EC100B0FF0CAFE9DEDA00B41EC110BD3
:104050000DF066FEB39AB49B51EC100B0FF040FCD0
:1040600041EC100B51EC100B0FF0BEF8BB998864BB
:10407000BB9948698969A2910FF09EFF0246A298F8
:10408000A3920A46A39942EC101B8DEDA60B0FF0EC
:1040900093FF9DEDAA0B41EC110B8DEDA41B0DF0D0
:1040A000D3FC0EF095F89DEDA41B51EC110B53ECD5
:1040B000102B0FF015FC9DEDA60B41EC110B53ECF2
:1040C000112B51EC100B0FF0C1F841EC100B8DEDE2
:1040D000B00BBB9908698969A8910FF06DFF024682
:1040E000A898A9920A46A99942EC101B8DEDAE0B37
:1040F0000FF062FF9DEDAA0B41EC110B8DEDAC1B97
:104100000DF0A2FC0EF0F4F99DEDAC1B51EC110B7F
:1041100053EC102B0FF0E4FB9DEDAE0B41EC110BBB
:1041200053EC112B51EC100B0FF058FE9DEDB00B22
:1041300041EC110B0DF0F4FDB39AB49B51EC100B54
:104140000FF0CEFB41EC100B51EC100B0FF04CF8C4
:10415000BB99C8643DE00020B890FFE7B8980328F9
:104160000BDCFFE7BB98B89900EB810100200862E7
:10417000FFE7B8980130B890F0E7BB9848F200012B
:10418000C4F29D310164BB9A0020C4F23420506413
:10419000BB9A9164BB99C8641BE00020B790FFE70D
:1041A000B79803280BDCFFE7BB98B79900EB8101B8
:1041B00000200862FFE7B7980130B790F0E7BB999D
:1041C00000200864BB994864BB998864BB99C864A3
:1041D000FFE7FFE700208DF8DB02FFE79DF8DB0239
:1041E000032822DCFFE7BB989DF8DB1200EB81007F
:1041F00090ED100AB5EE400AF1EE10FA0EDAFFE784
:10420000BB989DF8DB1200EB810090ED100A9FED4A
:10421000981A30EE010A80ED100AFFE7FFE79DF8DB
:10422000DB0201308DF8DB02D8E700208DF8DA02DE
:10423000FFE79DF8DA02032800F30E8104E000BFD7
:1042400000000000DCA54C40BB989DF8DA1200EBA2
:10425000810090ED100A90ED341A30EE410A40F2E0
:104260009420C2F2000000EB810080ED000AFFE71D
:104270009DF8DA1240F29420C2F2000000EB8100B7
:1042800090ED000A9FED761AB4EE410AF1EE10FAB5
:1042900011DDFFE79DF8DA1240F29420C2F200002F
:1042A00000EB810090ED000A9FED721A30EE010ADA
:1042B00080ED000ADCE7FFE79DF8DA1240F2942077
:1042C000C2F2000000EB810090ED000A9FED651A3C
:1042D000B4EE410AF1EE10FA11DAFFE79DF8DA12B6
:1042E00040F29420C2F2000000EB810090ED000A41
:1042F0009FED5F1A30EE010A80ED000ADCE79DF8C1
:10430000DA1240F29420C2F2000000EB810090ED3E
:10431000000A9FED551AB4EE410AF1EE10FA31DDB4
:10432000FFE79DF8DA1240F29420C2F2000000EBA1
:10433000810090ED000A9FED4A1AB4EE410AF1EEB9
:1043400010FA1FDCFFE7BB989DF8DA1200EB810141
:10435000086A0863BB989DF8DA2200EB820090EDB2
:10436000340A40F29421C2F2000101EB820191ED86
:10437000001A30EE010A9FED3B1A30EE010A80ED83
:10438000140A62E09DF8DA1240F29420C2F20000B2
:1043900000EB810090ED000A9FED341AB4EE410A63
:1043A000F1EE10FA31DAFFE79DF8DA1240F29420CC
:1043B000C2F2000000EB810090ED000A9FED291A87
:1043C000B4EE410AF1EE10FA1FDBFFE7BB989DF84F
:1043D000DA1200EB8101086A0863BB989DF8DA22C3
:1043E00000EB820090ED340A40F29421C2F2000109
:1043F00001EB820191ED001A30EE010A9FED181ACF
:1044000030EE010A80ED140A1EE0BB989DF8DA1226
:1044100000EB810090ED080AB1EE400A80ED0C0A35
:10442000BB989DF8DA2200EB820090ED340A40F24E
:104430009421C2F2000101EB820191ED001A30EEED
:10444000010A80ED140AFFE7FFE7FFE79DF8DA02B3
:1044500001308DF8DA02ECE60DF53C7D80BD00BF41
:1044600000003443000034C30000B4420000B4C272
:104470000000B4430000B4C380B584B00290029839
:1044800020B9FFE7FE208DF80F0091E005F08AFFCC
:1044900000200190FFE70198032800F38580FFE7E3
:1044A0000298D0F82804019900EBC100803005F093
:1044B00075FD183005F0C2FB9FED411A80EE010A30
:1044C0009FED401A20EE010A0298019900EB81004D
:1044D00080ED340A0298D0F82804019900EBC1005D
:1044E000803005F05BFD183005F0BAFB9FED361A01
:1044F00080EE010A0298019900EB810080ED300AFC
:104500000298D0F82804019900EBC100603005F052
:1045100045FD183005F0A4FB9FED2C1A80EE010A32
:104520000298019900EB810080ED280A0298019918
:1045300000EB810090ED340A00F5836090ED001AE5
:1045400030EE410A10EE100A0FF036FD41EC100B70
:104550009FED191B0DF048FF51EC100B0EF044FEBF
:104560000299019A01EB8201C1F8D00002980199E9
:1045700000EB810090ED340AB5EE400AF1EE10FA3E
:104580000DDAFFE70298019900EB810090ED340A03
:104590009FED0F1A30EE010A80ED340AFFE7FFE7C6
:1045A00001980130019076E700208DF80F00FFE7B9
:1045B0009DF90F0004B080BD00000000008076402F
:1045C000DB0F4940000034430000A04300401C467C
:1045D0000000B44385B08DED040ACDED030A8DEDE6
:1045E000021A9DED040A9DED031A30EE410A8DED8D
:1045F000010A9DED020AB5EE400AF1EE10FA32DD35
:10460000FFE79DED020AB0EE001A80EE010A8DED83
:10461000000A9DED010A9DED001AB4EE410AF1EE8B
:1046200010FA09DDFFE79DED021A9DED010A30EE5B
:10463000410A8DED010A15E09DED010A9DED001A7C
:10464000B1EE411AB4EE410AF1EE10FA09DAFFE7D1
:104650009DED021A9DED010A30EE010A8DED010A71
:10466000FFE7FFE7FFE79DED010A05B07047000097
:1046700040F20800C2F200007047000080B540F62A
:104680009020C2F2000001F0C3FA80BD80B540F670
:10469000F020C2F2000001F0BBFA80BD80B540F608
:1046A0007010C2F2000001F0B3FA80BD80B540F690
:1046B000D010C2F2000001F0ABFA80BD80B540F628
:1046C0003020C2F2000001F0A3FA80BD80B540F6B0
:1046D0005030C2F2000001F09BFA80BD82B0019020
:1046E0000198007810384AF6AB21CAF6AA21A0FB3F
:1046F000011000090090009944F27830C0F60100E2
:10470000405C0199C8650098042807D3FFE7019928
:104710000868042262F30900886506E001990868C8
:1047200040F2FF3290438865FFE70198806D02B048
:104730007047000086B0059000208DF813000598A2
:10474000806A03900598806910BBFFE70398029088
:1047500003281BD80299DFE801F0020D0218059822
:1047600090F82F00C00720B1FFE701208DF813005B
:10477000FFE70CE00598C06AB0F1C07F04D1FFE705
:1047800001208DF81300FFE701E000E0FFE745E0BE
:1047900005988069B0F5005F25D1FFE70398019087
:1047A00003281ED80199DFE801F00206021101205A
:1047B0008DF8130016E0059890F82F00C00720B17F
:1047C000FFE701208DF81300FFE70BE00598C06AB2
:1047D000B0F1C07F04D1FFE701208DF81300FFE79F
:1047E00000E0FFE719E003980090032804D3FFE7F7
:1047F0000098032804D00EE001208DF813000BE090
:10480000059890F82F00C00720B1FFE701208DF830
:104810001300FFE700E0FFE7FFE7FFE79DF8130065
:1048200006B0704784B00390029101920093039800
:104830000168086820F480200860009803990968DE
:10484000486003988068402809D1FFE701980399E0
:1048500009688860029803990968C86008E00298AE
:10486000039909688860019803990968C860FFE79F
:1048700004B070477047000080B5012001F0C8FC0B
:1048800080BD000080B5102001F0C2FC80BD00009A
:1048900080B5202001F0BCFC80BD000072B6FFE7AF
:1048A000FEE7000084B002900191029890F8200089
:1048B0008DF803009DF80300012805D0FFE79DF85F
:1048C000030002280AD1FFE7019A029801684869AB
:1048D0001043486100208DF80F0008E00299486AF3
:1048E00040F48020486201208DF80F00FFE79DF81A
:1048F0000F0004B07047000088B006900591049244
:104900000393069890F820008DF807000698006839
:10491000806800900598806808B9FFE700E0FFE72D
:104920009DF80700012806D0FFE79DF80700022840
:1049300040F08080FFE79DF80300400700280CD47A
:10494000FFE79DF803000007002806D4FFE79DF865
:104950000300C006002864D5FFE70098C0F301609B
:1049600002900299012088400399086005988068A8
:1049700068B9FFE705980168C06840EA41500699A8
:104980000968029A01EB0211C1F880010EE0059955
:104990004A688868C96840EAC200084306990968FD
:1049A000029A01EB0211C1F88001FFE70598006946
:1049B00006990968029A01EB0211C1F88401059871
:1049C000007D01280CD1FFE706980068029900EBF2
:1049D0000111D1F8840140F48070C1F88401FFE72F
:1049E0000498406806990968029A01EB0211C1F81F
:1049F0008C010498006806990968029A01EB02117B
:104A0000C1F8880106980068029900EB0111D1F8FD
:104A1000800140F00100C1F8800100208DF81F00E6
:104A200011E00699486A40F40010486201208DF8B0
:104A30001F0008E00699486A40F48020486201207F
:104A40008DF81F00FFE79DF81F0008B070470000B9
:104A500086B004900391049890F820008DF803002C
:104A60009DF80300012806D0FFE79DF80300022807
:104A700040F0B080FFE746F20040C4F20000019031
:104A80000199D1F8000240F00100C1F8000201993B
:104A9000D1F8000220F47C50C1F800020398426A69
:104AA0000199D1F8000240EA0220C1F800020398FF
:104AB000406900F01F01012088400290029A01998C
:104AC000D1F81C029043C1F81C020398C069F0B9E8
:104AD000FFE7029A0199D1F80C029043C1F80C0249
:104AE000039A9088D168526940EA0140019901EB2C
:104AF000C201C1F84002039A10889168526940EAE5
:104B00000140019901EBC201C1F84402FFE703989B
:104B1000C06901281ED1FFE7029A0199D1F80C0261
:104B20001043C1F80C02039A90881168526940EA58
:104B30000140019901EBC201C1F84002039A90893A
:104B40009168526940EA0140019901EBC201C1F844
:104B50004402FFE70398806940B9FFE7029A019990
:104B6000D1F804029043C1F8040207E0029A0199C7
:104B7000D1F804021043C1F80402FFE7039800696A
:104B800040B9FFE7029A0199D1F814029043C1F8A5
:104B9000140207E0029A0199D1F814021043C1F8F7
:104BA0001402FFE70398006A012808D1FFE7029A80
:104BB0000199D1F81C021043C1F81C02FFE70199CA
:104BC000D1F8000220F00100C1F8000200208DF8A9
:104BD000170008E00499486A40F4802048620120E8
:104BE0008DF81700FFE79DF8170006B0704700002A
:104BF00080B582B001900198FEF7A4FA8DF8030009
:104C00009DF80300032819D0FFE79DF8030040F248
:104C10006812C2F20002342110FB0120006B60B167
:104C2000FFE79DF8030040F26812C2F2000234214F
:104C300010FB0120006B8047FFE7FFE702B080BD5B
:104C400084B00390029100200190039890F8200016
:104C50008DF803009DF80300012805D0FFE79DF8BB
:104C60000300022812D1FFE7029838B9FFE7039842
:104C70000068C06800F00300019006E00398006837
:104C8000006900F003000190FFE7FFE7019804B01E
:104C90007047000086B0049003910292019304983B
:104CA00090F820008DF803009DF80300012806D03D
:104CB000FFE79DF80300022840F0E880FFE7039833
:104CC00080B9FFE704980068C068800748B9FFE72B
:104CD0000499486A40F40010486201208DF81700DA
:104CE000DDE00FE0049800680069800748B9FFE73D
:104CF0000499486A40F40010486201208DF81700BA
:104D0000CDE0FFE704980068039900EB0110D0F8AC
:104D1000B00100F00400029988600298806858B9D8
:104D2000FFE704980068039900EB0110D0F8B00188
:104D3000400D029908600AE004980068039900EBAE
:104D40000110D0F8B001C00802994860FFE704984C
:104D50000068039900EB0110D0F8B00100F00200E8
:104D60000299C86004980068039900EB0110D0F81C
:104D7000B40100F00F00082804D3FFE702990820CF
:104D800008610BE004980068039900EB0110D0F86B
:104D9000B40100F00F0002990861FFE70498006871
:104DA000039900EB0110D0F8B40180B2000A029917
:104DB000886104980068039900EB0110D0F8B401F1
:104DC000000C0299486104980068039900EB0110F7
:104DD000D0F8B8010199087004980068039900EBB5
:104DE0000110D0F8B801000A0199487004980068D1
:104DF000039900EB0110D0F8B801000C01998870FC
:104E000004980068039900EB0110D0F8B801000E77
:104E10000199C87004980068039900EB0110D0F85C
:104E2000BC010199087104980068039900EB011016
:104E3000D0F8BC01000A01994871049800680399F0
:104E400000EB0110D0F8BC01000C019988710498A6
:104E50000068039900EB0110D0F8BC01000E019925
:104E6000C871039838B9FFE704980168C86840F032
:104E70002000C86006E004980168086940F020003E
:104E80000861FFE700208DF8170008E00499486AE0
:104E900040F48020486201208DF81700FFE79DF85C
:104EA000170006B07047000083B002900020019008
:104EB000029890F820008DF803009DF80300012867
:104EC00005D0FFE79DF80300022822D1FFE70298F2
:104ED000006880684001002804D5FFE70198013090
:104EE0000190FFE70298006880680001002804D55F
:104EF000FFE7019801300190FFE7029800688068A1
:104F0000C000002804D5FFE7019801300190FFE7B9
:104F1000FFE7019803B0704780B58AB00990002080
:104F200008900998006840690790099800684068EF
:104F30000690099800688068059009980068C06824
:104F400004900998006800690390099800688069D6
:104F500002909DF81C00C007002800F09480FFE735
:104F60009DF81400C00758B3FFE7099801680120B5
:104F700088609DF814008007002804D5FFE7099891
:104F800000F0C0FC1BE09DF814004007002805D588
:104F9000FFE7089840F4006008900FE09DF81400C7
:104FA0000007002805D5FFE7089840F480500890D6
:104FB00003E0099800F07EFCFFE7FFE7FFE7FFE76B
:104FC0009DF81500C00760B3FFE7099801684FF42A
:104FD000807088609DF815008007002804D5FFE7E1
:104FE000099800F0DDFC1BE09DF815004007002843
:104FF00005D5FFE7089840F4005008900FE09DF8B1
:1050000015000007002805D5FFE7089840F4804008
:10501000089003E0099800F09BFCFFE7FFE7FFE73B
:10502000FFE79DF81600C00760B3FFE70998016825
:105030004FF4803088609DF816008007002804D562
:10504000FFE7099800F0FCFC1BE09DF81600400704
:10505000002805D5FFE7089840F4004008900FE0CD
:105060009DF816000007002805D5FFE7089840F4D2
:105070008030089003E0099800F0BAFCFFE7FFE7F2
:10508000FFE7FFE7FFE79DF81C000007002810D5A9
:10509000FFE79DF81000C006002809D5FFE7089833
:1050A00040F400700890099801681020C860FFE77C
:1050B000FFE79DF81C00400700280FD5FFE79DF88B
:1050C00010000007002808D5FFE7099801680820AC
:1050D000C860099800F0E0FAFFE7FFE79DF81C00C0
:1050E000800700280BD5FFE709980068C068800793
:1050F00020B1FFE7099800F0F7FAFFE7FFE79DF816
:105100001C004006002810D5FFE79DF80C00C006E3
:10511000002809D5FFE7089840F4806008900998B6
:10512000016810200861FFE7FFE79DF81C0080067A
:1051300000280FD5FFE79DF80C000007002808D5D0
:10514000FFE70998016808200861099800F0F4FA5F
:10515000FFE7FFE79DF81C00C00600280BD5FFE71E
:10516000099800680069800720B1FFE7099800F0FE
:105170000BFBFFE7FFE79DF81E00800700280FD517
:10518000FFE79DF81800C006002808D5FFE709983A
:10519000016810204860099800F01EFBFFE7FFE758
:1051A0009DF81E00C00778B1FFE79DF818000007C2
:1051B000002808D5FFE70998016808204860099889
:1051C00000F066FCFFE7FFE79DF81D0000060028E1
:1051D00040F18D80FFE79DF818004007002840F15E
:1051E0008180FFE79DF81D00C00750B1FFE79DF8E3
:1051F0000800C00728B1FFE7089840F001000890B8
:10520000FFE79DF81D00800700280BD5FFE79DF8FC
:1052100008008007002805D5FFE7089840F0020045
:105220000890FFE79DF81D00400700280BD5FFE719
:105230009DF808004007002805D5FFE7089840F0D2
:1052400004000890FFE79DF81D000007002848D5DE
:10525000FFE79DF8080010F0700F42D0FFE70298BA
:1052600000F0700001460191102814D0FFE701986A
:10527000202815D0FFE70198302816D0FFE70198C5
:10528000402817D0FFE70198502818D0FFE7019871
:10529000602819D01DE0089840F00800089019E037
:1052A000089840F01000089014E0089840F02000A2
:1052B00008900FE0089840F0400008900AE0089835
:1052C00040F08000089005E0089840F48070089055
:1052D00000E0FFE709980168886920F070008861A4
:1052E000FFE7FFE70998016804204860FFE7089896
:1052F00048B1FFE7089A0999486A1043486209983B
:10530000FFF776FCFFE70AB080BD000080B584B0EF
:105310000290029820B9FFE701208DF80F00E0E02D
:10532000029890F8200020B9FFE7029800F0DEF81C
:10533000FFE702980168086840F00100086001F08A
:105340008FF90190FFE7029800684068C007A8B98C
:10535000FFE701F085F90199401A0B280DD3FFE70B
:105360000299486A40F4003048620299052081F8A9
:10537000200001208DF80F00B3E0E4E702980168F7
:10538000086820F00200086001F06AF90190FFE768
:105390000298006840688007002815D5FFE701F0F3
:1053A0005FF90199401A0B280DD3FFE70299486A6B
:1053B00040F4003048620299052081F82000012065
:1053C0008DF80F008DE0E3E70298007E012807D1F9
:1053D000FFE702980168086840F08000086006E076
:1053E00002980168086820F080000860FFE70298D2
:1053F000407E012807D1FFE702980168086840F065
:105400004000086006E002980168086820F040004B
:105410000860FFE70298807E012807D1FFE7029825
:105420000168086840F02000086006E00298016802
:10543000086820F020000860FFE70298C07E01287D
:1054400007D1FFE702980168086820F010000860A3
:1054500006E002980168086840F010000860FFE765
:105460000298007F012807D1FFE7029801680868C9
:1054700040F00800086006E002980168086820F023
:1054800008000860FFE70298407F012807D1FFE786
:1054900002980168086840F00400086006E002987D
:1054A0000168086820F004000860FFE7029B1968A3
:1054B0005A689868D3F80CC040EA0C00D3F810C0C2
:1054C00040EA0C005B691843013A1043C861029935
:1054D00000204862029A012182F820108DF80F0006
:1054E000FFE79DF80F0004B080BD000080B594B0C8
:1054F000139000201290119010900F900E9013981E
:10550000006846F20041C4F20001884253D1FFE72F
:1055100040F21020C2F20000016801310160006811
:10552000012812D1FFE7FFE700200D9043F640006D
:10553000C4F20200016841F000710160006800F0EF
:1055400000700D900D98FFE7FFE7FFE700200C903B
:1055500043F63000C4F20200016841F00801016026
:10556000006800F008000C900C98FFE703200E90F4
:1055700002210F91002107911091119009201290A2
:1055800040F60040C4F202000EA900F05DFE079A4A
:10559000142005900521069101F00AF9059801F003
:1055A000FDF80699079A1520089001F001F908986E
:1055B00001F0F4F86EE01398006846F60001C4F2BA
:1055C0000001884265D1FFE7FFE700200B9043F61A
:1055D0004000C4F20200016841F08061016000688F
:1055E00000F080600B900B98FFE740F21020C2F2B1
:1055F00000000168013101600068012812D1FFE755
:10560000FFE700200A9043F64000C4F20200016860
:1056100041F000710160006800F000700A900A9883
:10562000FFE7FFE7FFE70020099043F63000C4F2F0
:105630000200016841F002010160006800F0020010
:1056400009900998FFE760200E9002200F9000203B
:1056500003901090032011900920129040F2004016
:10566000C4F202000EA900F0EFFD039A4020019061
:105670000521029101F09CF8019801F08FF8029940
:10568000039A4120049001F093F8049801F086F801
:10569000FFE7FFE714B080BD80B582B001900198AC
:1056A000FDF750FD8DF803009DF80300032819D085
:1056B000FFE79DF8030040F26812C2F200023421B5
:1056C00010FB0120C06960B1FFE79DF8030040F2C4
:1056D0006812C2F20002342110FB0120C069804729
:1056E000FFE7FFE702B080BD80B582B0019001986E
:1056F000FDF728FD8DF803009DF80300032819D05D
:10570000FFE79DF8030040F26812C2F20002342164
:1057100010FB0120806960B1FFE79DF8030040F2B3
:105720006812C2F20002342110FB01208069804718
:10573000FFE7FFE702B080BD80B582B0019001981D
:10574000FDF700FD8DF803009DF80300032819D034
:10575000FFE79DF8030040F26812C2F20002342114
:1057600010FB0120406A60B1FFE79DF8030040F2A2
:105770006812C2F20002342110FB0120406A804707
:10578000FFE7FFE702B080BD80B582B001900198CD
:10579000FDF7D8FC8DF803009DF80300032819D00D
:1057A000FFE79DF8030040F26812C2F200023421C4
:1057B00010FB0120006A60B1FFE79DF8030040F292
:1057C0006812C2F20002342110FB0120006A8047F7
:1057D000FFE7FFE702B080BD80B582B0019001987D
:1057E000FDF7B0FC8DF803009DF80300032819D0E5
:1057F000FFE79DF8030040F26812C2F20002342174
:1058000010FB0120806A60B1FFE79DF8030040F2C1
:105810006812C2F20002342110FB0120806A804726
:10582000FFE7FFE702B080BD80B584B00290029828
:1058300090F8200001282FD1FFE70299022081F87B
:10584000200002980168086820F00100086000F05C
:1058500007FF0190FFE7029800684068C007A8B101
:10586000FFE700F0FDFE0199401A0B280DD3FFE77A
:105870000299486A40F4003048620299052081F894
:10588000200001208DF80F000FE0E4E702990020CE
:1058900048628DF80F0008E00299486A40F4002041
:1058A000486201208DF80F00FFE79DF80F0004B05B
:1058B00080BD000080B582B001900198FDF742FCE8
:1058C0008DF803009DF80300032819D0FFE79DF829
:1058D000030040F26812C2F20002342110FB0120E2
:1058E000C06860B1FFE79DF8030040F26812C2F2A1
:1058F0000002342110FB0120C0688047FFE7FFE76A
:1059000002B080BD80B582B001900198FDF71AFC0D
:105910008DF803009DF80300032817D0FFE79DF8DA
:1059200003003421414340F26810C2F200004058A5
:1059300058B1FFE79DF803003421414340F268105D
:10594000C2F2000040588047FFE7FFE702B080BD89
:1059500080B582B001900198FDF7F4FB8DF803004B
:105960009DF80300032819D0FFE79DF8030040F2DB
:105970006812C2F20002342110FB0120006960B1FC
:10598000FFE79DF8030040F26812C2F200023421E2
:1059900010FB012000698047FFE7FFE702B080BDF0
:1059A00080B582B001900198FDF7CCFB8DF8030023
:1059B0009DF80300032819D0FFE79DF8030040F28B
:1059C0006812C2F20002342110FB0120406860B16D
:1059D000FFE79DF8030040F26812C2F20002342192
:1059E00010FB012040688047FFE7FFE702B080BD61
:1059F00080B582B001900198FDF7A4FB8DF80300FB
:105A00009DF80300032819D0FFE79DF8030040F23A
:105A10006812C2F20002342110FB0120406960B11B
:105A2000FFE79DF8030040F26812C2F20002342141
:105A300010FB012040698047FFE7FFE702B080BD0F
:105A400080B582B001900198FDF77CFB8DF80300D2
:105A50009DF80300032819D0FFE79DF8030040F2EA
:105A60006812C2F20002342110FB0120806860B18C
:105A7000FFE79DF8030040F26812C2F200023421F1
:105A800010FB012080688047FFE7FFE702B080BD80
:105A900080B582B001900198FDF754FB8DF80300AA
:105AA0009DF80300032819D0FFE79DF8030040F29A
:105AB0006812C2F20002342110FB0120C06A60B1FA
:105AC000FFE79DF8030040F26812C2F200023421A1
:105AD00010FB0120C06A8047FFE7FFE702B080BDEE
:105AE00080B584B002900298806D019000F0B8FDFE
:105AF0000090029890F8350002280DD0FFE7029937
:105B000080204865FFE70299002081F83400FFE714
:105B100001208DF80F0055E002980168086820F018
:105B20001600086002980168486920F0800048610A
:105B30000298006C20B9FFE70298806C38B1FFE74B
:105B400002980168086820F008000860FFE70298E2
:105B50000168086820F001000860FFE7029800680B
:105B60000068C007C8B1FFE700F07AFD0099401A4D
:105B7000062811D3FFE702992020486502990320E7
:105B800081F83500FFE70299002081F83400FFE733
:105B900003208DF80F0015E0E0E70298C16D3F206B
:105BA0008840019988600299012081F83500FFE75B
:105BB0000299002081F83400FFE7FFE700208DF80C
:105BC0000F00FFE79DF80F0004B080BD82B0009089
:105BD000009890F83500022807D0FFE70099802050
:105BE000486501208DF807000EE00099052081F836
:105BF000350000980168086820F001000860FFE7A0
:105C000000208DF80700FFE79DF8070002B07047FD
:105C100080B586B005900020039040F20000C2F2EB
:105C20000000006848F2B511C1F64E31A0FB01102A
:105C3000800A02900598806D019001980068049098
:105C400004980599C96DC840000700281AD5FFE7D8
:105C50000598006800684007002812D5FFE70598FE
:105C60000168086820F0040008600598C16D0820EC
:105C70008840019988600599486D40F001004865A9
:105C8000FFE7FFE704980599C96DC840C007A0B1B8
:105C9000FFE7059800684069000600280CD5FFE77B
:105CA0000598C16D01208840019988600599486D6B
:105CB00040F002004865FFE7FFE704980599C96DC9
:105CC000C8404007002814D5FFE705980068006821
:105CD000800700280CD5FFE70598C16D0420884097
:105CE000019988600599486D40F004004865FFE718
:105CF000FFE704980599C96DC840C006002847D53C
:105D0000FFE7059800680068000700283FD5FFE717
:105D10000598C16D10208840019988600598006839
:105D20000068400300281AD5FFE70598006800685E
:105D30000003002809D4FFE70598006C20B1FFE7B5
:105D40000598016C8847FFE708E00598806C20B152
:105D5000FFE70598816C8847FFE7FFE716E00598A5
:105D600000680068C005002807D4FFE705980168AF
:105D7000086820F008000860FFE70598006C20B173
:105D8000FFE70598016C8847FFE7FFE7FFE7FFE7BC
:105D900004980599C96DC8408006002840F18D809F
:105DA000FFE7059800680068C006002840F184807D
:105DB000FFE70598C16D202088400199886005980B
:105DC00090F83500052834D1FFE705980168086888
:105DD00020F01600086005980168486920F08000EE
:105DE00048610598006C20B9FFE70598806C38B1D0
:105DF000FFE705980168086820F008000860FFE7E1
:105E00000598C16D3F20884001998860059901205F
:105E100081F83500FFE70599002081F83400FFE79D
:105E20000598006D20B1FFE70598016D8847FFE7F1
:105E30007BE0059800680068400300281AD5FFE75A
:105E40000598006800680003002809D4FFE705985A
:105E5000406C20B1FFE70598416C8847FFE708E0F8
:105E60000598C06B20B1FFE70598C16B8847FFE735
:105E7000FFE720E0059800680068C005002811D4FD
:105E8000FFE705980168086820F010000860059990
:105E9000012081F83500FFE70599002081F83400E2
:105EA000FFE7FFE70598C06B20B1FFE70598C16BDE
:105EB0008847FFE7FFE7FFE7FFE70598406DA0B3DE
:105EC000FFE70598406DC00730B3FFE7059905204F
:105ED00081F8350005980168086820F00100086025
:105EE000FFE70398013003900299884201D9FFE748
:105EF00007E0FFE7059800680068C0070028F0D1B8
:105F0000FFE70599012081F83500FFE7059900209A
:105F100081F83400FFE7FFE70598C06C20B1FFE788
:105F20000598C16C8847FFE7FFE706B080BD000019
:105F300080B586B004900020039000F091FB0290A1
:105F4000049820B9FFE701208DF81700A3E004981A
:105F5000406A08B1FFE7FFE70499022081F83500A5
:105F6000FFE70499002081F83400FFE704980168F6
:105F7000086820F001000860FFE7049800680068E6
:105F8000C00790B1FFE700F06BFB0299401A0628AA
:105F90000AD3FFE70499202048650499032081F87B
:105FA00035008DF8170076E0E7E704980068006890
:105FB0000390039848F23F01CFF21001084003908C
:105FC000049900914868D1F808C0CB680A6940EA92
:105FD0000C00184310434A6910438A691043CA6988
:105FE0001043096A01430398084303900498406AE8
:105FF000042808D1FFE70499C86A096B0143039894
:1060000008430390FFE7039804990968086004981F
:10601000006840690390039820F0070003900498FB
:10602000416A0398084303900498406A04281AD1EF
:10603000FFE70498816A0398084303900498C06AB4
:1060400080B1FFE70498FEF775FB50B1FFE70499B4
:10605000402048650499012081F835008DF817002B
:1060600019E0FFE7FFE7039804990968486104987D
:10607000FEF734FB01900498C16D3F2088400199E0
:106080008860049900204865049A012182F835103F
:106090008DF81700FFE79DF8170006B080BD0000DF
:1060A00080B588B0069005910492039300208DF886
:1060B0000B000698806D0190FFE7069890F8340079
:1060C000012804D1FFE702208DF81F0045E0069962
:1060D000012081F83400FFE7FFE7069890F83500CB
:1060E00001282BD1FFE70699022081F83500069997
:1060F0000020486506980599049A039BFEF792FBD9
:106100000698C16D3F208840019988600698016813
:10611000086840F0160008600698006C38B1FFE788
:1061200006980168086840F008000860FFE70698D4
:106130000168086840F00100086009E0FFE706997F
:10614000002081F83400FFE702208DF80B00FFE704
:106150009DF80B008DF81F00FFE79DF81F0008B0A9
:1061600080BD000080B584B0039000F079FA029001
:10617000039801900198013048B1FFE740F2F80020
:10618000C2F200000178019808440190FFE7FFE7A0
:1061900000F066FA0299401A0199884201D2FFE79D
:1061A000F6E704B080BD000080B582B0ADF806000F
:1061B00000208DF80500FFE79DF805000F2824DC7E
:1061C000FFE7BDF806009DF80510C840C007A8B15C
:1061D000FFE79DF8051040F2D010C2F2000050F821
:1061E000210050B1FFE79DF8051040F2D010C2F237
:1061F000000050F821008047FFE7FFE7FFE79DF828
:10620000050001308DF80500D6E702B080BD000022
:1062100080B582B0ADF8060043F61440C4F2010028
:106220000068BDF8061008420CD0FFE7BDF8060074
:1062300043F61441C4F201010860BDF80600FFF7FF
:10624000B3FFFFE702B080BD8EB00D900C9100202F
:106250000A90099008900B90FFE70B980F2800F226
:10626000CC81FFE70B99012088400A900C980068C8
:106270000A990840099009980A99884240F0B88123
:10628000FFE70C98406800F00300012807D0FFE703
:106290000C98406800F0030002282FD1FFE70D980A
:1062A000806808900B984100032000FA01F10898DB
:1062B000884308900C98C0680B99490000FA01F1D6
:1062C00008980843089008980D9988600D984068D0
:1062D00008900B99012000FA01F108988843089072
:1062E0000C984068C0F300100B9900FA01F108986F
:1062F0000843089008980D994860FFE70C9840689B
:1063000000F00300032818D0FFE70D98C06808903C
:106310000B984100032000FA01F108988843089087
:106320000C9880680B99490000FA01F1089808431D
:10633000089008980D99C860FFE70C98406800F035
:106340000300022826D1FFE70D980B996FF0030296
:1063500002EA51010844006A08900B9800F0070017
:1063600081000F2000FA01F10898884308900C98EA
:1063700000690B9901F00701890000FA01F1089802
:106380000843089008980D990B9B02EA53021144A8
:106390000862FFE70D98006808900B984100032001
:1063A00000FA01F10898884308900C98406800F0C2
:1063B00003000B99490000FA01F10898084308907E
:1063C00008980D9908600C9880798007002800F0E3
:1063D0000E81FFE7FFE70020079043F64400C4F278
:1063E0000200016841F480410160006800F48040CF
:1063F00007900798FFE70B9820F0030043F6080189
:10640000C4F20101405808900B9800F0030081008D
:106410000F2000FA01F10898884308900D98002198
:10642000C4F20201884203D1FFE7002006905EE03B
:106430000D9840F20041C4F20201884203D1FFE707
:106440000120059050E00D9840F60001C4F20201D1
:10645000884203D1FFE70220049042E00D9840F605
:106460000041C4F20201884203D1FFE703200390F8
:1064700034E00D9841F20001C4F20201884203D1D8
:10648000FFE70420029026E00D9841F20041C4F29B
:106490000201884203D1FFE70520019018E00D9822
:1064A00041F60001C4F20201884203D1FFE7062051
:1064B00000900AE00D9941F60042C4F20202082061
:1064C000914208BF07200090FFE700980190FFE786
:1064D00001980290FFE702980390FFE70398049069
:1064E000FFE704980590FFE705980690FFE70698F8
:1064F000C0B20B9901F00301890000FA01F108987C
:106500000843089008980B9921F0030143F608020C
:10651000C4F20102885043F60840C4F2010000684A
:10652000089009990898884308900C988079C006CB
:10653000002805D5FFE70999089808430890FFE768
:10654000089843F60841C4F20101086043F60C4084
:10655000C4F20100006808900999089888430890DF
:106560000C9880798006002805D5FFE709990898DE
:1065700008430890FFE7089843F60C41C4F2010174
:10658000086043F60440C4F20100006808900999CD
:106590000898884308900C9880798007002805D5D2
:1065A000FFE70999089808430890FFE7089843F621
:1065B0000441C4F20101086043F60040C4F2010046
:1065C0000068089009990898884308900C98807989
:1065D000C00728B1FFE70999089808430890FFE72A
:1065E000089843F60041C4F201010860FFE7FFE7A5
:1065F000FFE70B9801300B902FE60EB070470000BC
:1066000082B00190ADF8021001980069BDF8021047
:10661000084204D0FFE701208DF8010003E00020CC
:106620008DF80100FFE79DF8010002B070470000FF
:1066300082B00190ADF802108DF801209DF80100A4
:1066400028B1FFE7BDF802000199886105E0BDF8B7
:106650000200000401998861FFE702B07047000062
:1066600045F2DC00C2F200000068704740F2F8001A
:10667000C2F20000027845F2DC01C2F200010868B3
:10668000104408607047000080B543F60041C4F232
:106690000201086840F400700860086840F48060F7
:1066A0000860086840F480700860032000F09AF8E1
:1066B0000F2000F005F800F03BF8002080BD00003E
:1066C00080B582B0009040F20000C2F20000006885
:1066D00040F2F801C2F200010A784FF47A71B1FB7E
:1066E000F2F1B0FBF1F001F0F7FE20B1FFE701207D
:1066F0008DF8070018E000980F280DD8FFE70099E3
:106700004FF0FF30002200F053F8009840F2FC01F7
:10671000C2F20001086003E001208DF8070003E0E9
:1067200000208DF80700FFE79DF8070002B080BD4C
:1067300080B582B0FFE70020019043F64400C4F228
:106740000200016841F480410160006800F480406B
:1067500001900198FFE7FFE70020009043F640001A
:10676000C4F20200016841F080510160006800F04D
:10677000805000900098FFE76FF001000F21002289
:1067800000F016F802B080BD80B582B08DF8070029
:106790009DF9070006F0D6FA02B080BD80B582B040
:1067A0008DF807009DF9070006F0E8FA02B080BDF9
:1067B00080B586B08DF817000491039200200290F6
:1067C00006F0F4FA02909DF91700019002980499DE
:1067D000039A04F069FA0146019806F0EFFA06B050
:1067E00080BD000080B582B00190019806F02AFBC0
:1067F00002B080BD80B584B002900191029820B9AA
:10680000FFE701208DF80F0021E1019843F60041D8
:10681000C4F20201096801F00701884212D9FFE7BA
:10682000019943F60040C4F202000170006800F0D4
:1068300007000199884204D0FFE701208DF80F007E
:1068400005E1FFE702980078800700282AD5FFE7D6
:10685000029800784007002809D5FFE743F60801B1
:10686000C4F20201086840F4E0500860FFE70298B3
:1068700000780007002809D5FFE743F60801C4F2B5
:106880000201086840F460400860FFE743F6080131
:10689000C4F20201086820F0F000029A92681043E6
:1068A0000860FFE702980078C00700286ED0FFE775
:1068B00002984068012811D1FFE743F60000C4F2B6
:1068C0000200006800F400310020B0EB514F04D109
:1068D000FFE701208DF80F00B9E02CE00298406836
:1068E000022805D0FFE702984068032811D1FFE78E
:1068F00043F60000C4F20200006800F000710020BE
:10690000B0EB516F04D1FFE701208DF80F009EE03E
:1069100010E043F60000C4F20200006800F002013B
:106920000020B0EB510F04D1FFE701208DF80F00DC
:106930008DE0FFE7FFE743F60801C4F202010868B3
:1069400020F00300029A526810430860FFF788FEA7
:106950000090FFE743F60800C4F20200006800F070
:106960000C0002994968B0EB810F0ED0FFE7FFF7EA
:1069700077FE0099401A41F28931884204D3FFE73B
:1069800003208DF80F0062E0E4E7FFE7019843F68B
:106990000041C4F20201096801F00701884212D2E5
:1069A000FFE7019943F60040C4F20200017000685D
:1069B00000F007000199884204D0FFE701208DF81C
:1069C0000F0044E0FFE702980078400700280CD54C
:1069D000FFE743F60801C4F20201086820F4E05022
:1069E000029AD26810430860FFE702980078000717
:1069F00000280DD5FFE743F60801C4F2020108683C
:106A000020F46040029A126940EAC2000860FFE781
:106A100000F04CF843F60801C4F202010968C9B25B
:106A20000A0944F26031C0F60101895CC84040F2B5
:106A30000001C2F20001086040F2FC00C2F2000056
:106A40000068FFF73DFE00208DF80F00FFE79DF87E
:106A50000F0004B080BD000040F20000C2F2000050
:106A60000068704780B5FFF7F7FF43F60801C4F2EE
:106A700002010968C1F3822244F27031C0F60101BB
:106A8000895CC84080BD000080B5FFF7E5FF43F694
:106A90000801C4F20201096889B24A0B44F270315C
:106AA000C0F60101895CC84080BD000080B586B099
:106AB0000020059004900390029043F60800C4F271
:106AC0000200006800F00C000146019140B1FFE7B0
:106AD000019804280AD0FFE7019808280CD04FE05D
:106AE00042F20040C0F2F40002904FE041F6003064
:106AF000C0F2B700029049E043F60400C4F202007D
:106B0000016801F03F01059100684002002813D59B
:106B1000FFE743F60400C4F202000068C0F38810E7
:106B200041F60031C0F2B701A0FB0101059A002334
:106B3000F9F79AFB049012E043F60400C4F2020055
:106B40000068C0F3881042F20041C0F2F401A0FBDB
:106B50000101059A0023F9F787FB0490FFE743F64C
:106B60000400C4F20200006800F44031022000EB8F
:106B7000D130039004980399B0FBF1F0029005E046
:106B800042F20040C0F2F4000290FFE7029806B023
:106B900080BD000080B586B00490049820B9FFE75E
:106BA00001208DF8170050E304980078C0070028F2
:106BB00000F0A580FFE743F60800C4F20200006879
:106BC00000F00C00042813D0FFE743F60800C4F2DD
:106BD0000200006800F00C0008281ED1FFE743F611
:106BE0000400C4F2020000684002002815D5FFE747
:106BF00043F60000C4F20200006800F400310020F7
:106C0000B0EB514F08D0FFE70498406820B9FFE788
:106C100001208DF8170018E370E0FFE70498406842
:106C2000B0F5803F09D1FFE743F60001C4F202014D
:106C3000086840F48030086020E004984068B0F5AF
:106C4000A02F0DD1FFE743F60001C4F2020108684E
:106C500040F480200860086840F4803008600CE050
:106C600043F60001C4F20201086820F48030086095
:106C7000086820F480200860FFE7FFE7FFE704983A
:106C80004068E8B1FFE7FFF7EBFC0390FFE743F64E
:106C90000000C4F20200006800F400310020B0EBF4
:106CA000514F0CD1FFE7FFF7DBFC0399401A652831
:106CB00004D3FFE703208DF81700C6E2E7E71CE0E6
:106CC000FFF7CEFC0390FFE743F60000C4F202009A
:106CD000006800F400310020B0EB514F0CD0FFE70A
:106CE000FFF7BEFC0399401A652804D3FFE7032091
:106CF0008DF81700A9E2E7E7FFE7FFE7FFE7049851
:106D000000788007002840F19680FFE743F60800EE
:106D1000C4F20200006810F00C0F13D0FFE743F636
:106D20000800C4F20200006800F00C0008282CD112
:106D3000FFE743F60400C4F20200006840020028A6
:106D400023D4FFE743F60000C4F20200006800F01D
:106D500002010020B0EB510F09D0FFE70498C06892
:106D6000012804D0FFE701208DF817006DE243F6FB
:106D70000001C4F20201086820F0F800049A1269C8
:106D800040EAC2000860FFE754E00498C06870B3AE
:106D9000FFE70021C4F2472101200860FFF760FCF3
:106DA0000390FFE743F60000C4F20200006800F021
:106DB00002010020B0EB510F0CD1FFE7FFF750FCB0
:106DC0000399401A032804D3FFE703208DF8170026
:106DD0003BE2E7E743F60001C4F20201086820F055
:106DE000F800049A126940EAC200086021E000211C
:106DF000C4F2472100200860FFF732FC0390FFE750
:106E000043F60000C4F20200006800F00201002016
:106E1000B0EB510F0CD0FFE7FFF722FC0399401AAB
:106E2000032804D3FFE703208DF817000DE2E7E7FE
:106E3000FFE7FFE7FFE704980078000700284BD53D
:106E4000FFE70498406918B3FFE740F68061C4F299
:106E5000472101200860FFF703FC0390FFE743F69A
:106E60007400C4F20200006800F002010020B0EBE0
:106E7000510F0CD1FFE7FFF7F3FB0399401A0328EA
:106E800004D3FFE703208DF81700DEE1E7E722E0F7
:106E900040F68061C4F2472100200860FFF7E0FB64
:106EA0000390FFE743F67400C4F20200006800F0AC
:106EB00002010020B0EB510F0CD0FFE7FFF7D0FB31
:106EC0000399401A032804D3FFE703208DF8170025
:106ED000BBE1E7E7FFE7FFE70498007840070028F9
:106EE00040F1CE80FFE700208DF8070043F6400018
:106EF000C4F202000068C000002815D4FFE7FFE7D5
:106F00000020009043F64000C4F20200016841F006
:106F100080510160006800F0805000900098FFE709
:106F200001208DF80700FFE747F20000C4F20000DF
:106F30000068C005002822D4FFE747F20001C4F230
:106F40000001086840F480700860FFF789FB039037
:106F5000FFE747F20000C4F200000068C005002807
:106F60000CD4FFE7FFF77CFB0399401A032804D3F6
:106F7000FFE703208DF8170067E1EAE7FFE7FFE787
:106F800004988068012809D1FFE743F67001C4F234
:106F90000201086840F0010008601FE00498806862
:106FA00005280DD1FFE743F67001C4F2020108681D
:106FB00040F004000860086840F0010008600CE040
:106FC00043F67001C4F20201086820F00100086075
:106FD000086820F004000860FFE7FFE7FFE7049877
:106FE0008068F8B1FFE7FFF73BFB0390FFE743F64C
:106FF0007000C4F20200006800F002010020B0EB53
:10700000510F0ED1FFE7FFF72BFB0399401A41F216
:107010008931884204D3FFE703208DF8170014E17B
:10702000E5E71EE0FFF71CFB0390FFE743F6700067
:10703000C4F20200006800F002010020B0EB510F22
:107040000ED0FFE7FFF70CFB0399401A41F289319C
:10705000884204D3FFE703208DF81700F5E0E5E749
:10706000FFE79DF80700012809D1FFE743F640013B
:10707000C4F20201086820F080500860FFE7FFE7D3
:1070800004988069002800F0DC80FFE743F60800E0
:10709000C4F20200006800F00C00082800F08580AF
:1070A000FFE70498806902285CD1FFE76021C4F201
:1070B000472100200860FFF7D3FA0390FFE743F66B
:1070C0000000C4F20200006800F000710020B0EB84
:1070D000516F0CD0FFE7FFF7C3FA0399401A03285A
:1070E00004D3FFE703208DF81700AEE0E7E704992B
:1070F000C869D1F820C04B6A8A6A40EA0C0040EAAD
:107100008310D2034FF6FF739A43A2F580321043E7
:10711000C96A40EA016043F60401C4F20201086052
:107120006021C4F2472101200860FFF799FA03901B
:10713000FFE743F60000C4F20200006800F00071AF
:107140000020B0EB516F0CD1FFE7FFF789FA0399EC
:10715000401A032804D3FFE703208DF8170074E0DA
:10716000E7E721E06021C4F2472100200860FFF733
:1071700077FA0390FFE743F60000C4F202000068CC
:1071800000F000710020B0EB516F0CD0FFE7FFF76B
:1071900067FA0399401A032804D3FFE703208DF808
:1071A000170052E0E7E7FFE74AE00498806901280A
:1071B00004D1FFE701208DF8170046E043F60400F4
:1071C000C4F202000068029004988069012831D05E
:1071D000FFE7029800F480000499C969884229D128
:1071E000FFE7029800F03F000499096A884221D124
:1071F000FFE7029847F6C07108400499496AB0EB6E
:10720000811F17D1FFE7029800F440300499896A82
:10721000C9034FF6FF729143A1F58031884209D12D
:10722000FFE7029800F070600499C96AB0EB016F43
:1072300004D0FFE701208DF8170006E0FFE7FFE725
:10724000FFE700208DF81700FFE79DF8170006B054
:1072500080BD000080B582B00190019804F04AFA28
:107260008DF803009DF8030002281BD0FFE701986A
:1072700004F040FA014640F21820C2F2000000EB90
:107280004110806968B1FFE7019804F033FA0146C4
:1072900040F21820C2F2000000EB411080698047E4
:1072A000FFE7FFE702B080BD80B584B0029002988E
:1072B00020B9FFE701208DF80F0071E00298406AC5
:1072C00060B9FFE702984068B0F5827F01D1FFE71F
:1072D00003E002990020C861FFE705E00299002061
:1072E000086102994861FFE70299002088620298CC
:1072F00090F8510040B9FFE70299002081F8500052
:10730000029800F051F8FFE70299022081F851003D
:1073100002980168086820F040000860029A019213
:1073200011685068D2F808C0D36800F482700CF479
:10733000044C604403F400631844136903F002032F
:107340001844536903F001031844936903F400736C
:107350001844D36903F038031844136A03F0800318
:107360001843926A02F4005210430860029A508B4C
:1073700000F004001168526A02F0100210444860E4
:1073800002980168C86920F40060C8610299002071
:107390004865029A012182F851108DF80F00FFE72D
:1073A0009DF80F0004B080BD80B590B00F90002014
:1073B0000E900D900C900B900A900F98006843F27D
:1073C0000001C4F20101884240F0B680FFE7FFE708
:1073D0000020099043F64400C4F20200016841F421
:1073E00080510160006800F4805009900998FFE71F
:1073F000FFE70020089043F63000C4F20200016865
:1074000041F002010160006800F002000890089855
:10741000FFE7FFE70020079043F63000C4F20200C8
:10742000016841F001010160006800F0010007906F
:107430000798FFE718200A90022001900B90002087
:1074400005900C90032002900D90052003900E9063
:1074500040F20040C4F202000AA90491FEF7F4FED3
:10746000DDF804C0029A03980499059B4FF0800E42
:10747000CDF828E0CDF82CC00C930D920E90002092
:10748000C4F20200FEF7E0FE059940F67010C2F269
:107490000000069046F24042C4F2020202604FF041
:1074A000C06242608160C1604FF4806202614161EC
:1074B0008161C1614FF4403202624162FEF738FDE2
:1074C00018B1FFE7FDF7EAF9FFE7FFE70F9840F68D
:1074D0007011C2F20001C1640F988863FFE740F6A3
:1074E000D010C2F20000009046F25841C4F20201EE
:1074F00001604FF0C0614160402181600021C160A6
:107500004FF48062026141618161C1614FF40032D8
:1075100002624162FEF70CFD18B1FFE7FDF7BEF90C
:10752000FFE7FFE70F9840F6D011C2F20001816437
:107530000F988863FFE7FFE710B080BD80B588B083
:1075400006900591ADF812200393069890F851002B
:10755000012804D0FFE702208DF81F0011E10598F3
:1075600020B1FFE7BDF8120020B9FFE701208DF838
:107570001F0006E106984068B0F5827F16D1FFE74C
:107580000698806890B9FFE70699042081F85100B9
:107590000698059ABDF812300399EC46CCF8001015
:1075A000114600F065FB8DF81F00EAE0FFF758F880
:1075B0000290FFE7069890F85000012804D1FFE7F9
:1075C00002208DF81F00DCE00699012081F85000B0
:1075D000FFE7FFE70699042081F851000699002093
:1075E00048650599069A9163BDF81210069A91872D
:1075F000BDF81210069AD187069908630699888605
:107600000699C886069908640699486406988068B1
:10761000B0F5004F0DD1FFE706980168086820F02B
:107620004000086006980168086820F480400860FF
:10763000FFE706980068006800F04000402807D087
:10764000FFE706980168086840F040000860FFE71F
:107650000698C068D0BBFFE7FFE70698C08FA0B3CD
:10766000FFE7069800688068C00778B1FFE70698D2
:107670000068007B0699896B08700699886B013059
:1076800088630699C88F0138C8871DE0FEF7E8FFB8
:107690000299401A0399884204D3FFE70398013006
:1076A00018B9FFE7039870B9FFE70699012081F840
:1076B0005100FFE70699002081F85000FFE7032002
:1076C0008DF81F005DE0FFE7C7E739E0FFE70698A8
:1076D000C08FA0B3FFE7069800688068C00778B144
:1076E000FFE706980068C0680699896B08800699CC
:1076F000886B023088630699C88F0138C8871DE0FF
:10770000FEF7AEFF0299401A0399884204D3FFE7BF
:107710000398013018B9FFE7039870B9FFE706999D
:10772000012081F85100FFE70699002081F8500000
:10773000FFE703208DF81F0023E0FFE7C7E7FFE71F
:1077400006980399029A03F0FDFE20B1FFE706991F
:1077500020204865FFE70699012081F85100FFE7E6
:107760000699002081F85000FFE70698406D20B18F
:10777000FFE701208DF81F0003E000208DF81F00B7
:10778000FFE79DF81F0008B080BD000080B584B001
:1077900002900191ADF80220029890F85100012862
:1077A00004D0FFE702208DF80F00B7E0019820B168
:1077B000FFE7BDF8020020B9FFE701208DF80F00B8
:1077C000ACE002988068A0B9FFE702984068B0F585
:1077D000827F0ED1FFE70299042081F851000298C0
:1077E000019ABDF80230114600F014FC8DF80F002C
:1077F00094E0FFE7029890F85000012804D1FFE7D9
:1078000002208DF80F0089E00299012081F85000D4
:10781000FFE7FFE70299042081F851000299002058
:1078200048650199029A9163BDF80210029A918706
:10783000BDF80210029AD18702990864029948643F
:10784000029988860299C88602988068B0F5004F30
:107850000DD1FFE702980168086820F04000086039
:1078600002980168086820F480400860FFE70298E9
:10787000C16C4BF22930C0F6000008640298C16C5C
:107880004BF27130C0F60000C8630298C16C4BF235
:10789000F520C0F60000C8640298C16C002008659D
:1078A000029B19689A6BD86C0C31DB8FFEF7F8FBE2
:1078B00078B1FFE70299486D40F010004865FFE796
:1078C0000299002081F85000FFE701208DF80F0099
:1078D00024E002980068006800F04000402807D0CB
:1078E000FFE702980168086840F040000860FFE781
:1078F000FFE70299002081F85000FFE70298016835
:10790000486840F02000486002980168486840F0EC
:107910000100486000208DF80F00FFE79DF80F0080
:1079200004B080BD80B582B00190019803F0E2FE02
:107930008DF803009DF8030002281BD0FFE7019893
:1079400003F0D8FE014640F21820C2F2000000EB1E
:107950004110406868B1FFE7019803F0CBFE014693
:1079600040F21820C2F2000000EB4110406880474E
:10797000FFE7FFE702B080BD80B582B001900198BB
:1079800003F0B8FE8DF803009DF8030002281BD019
:10799000FFE7019803F0AEFE014640F21820C2F264
:1079A000000000EB4110006968B1FFE7019803F0A7
:1079B000A1FE014640F21820C2F2000000EB411087
:1079C00000698047FFE7FFE702B080BD80B588B05F
:1079D00006900591ADF812200393FEF741FE029048
:1079E000BDF81200ADF80600069890F85100012885
:1079F00004D0FFE702208DF81F0034E1059820B184
:107A0000FFE7BDF8120020B9FFE701208DF81F0045
:107A100029E1FFE7069890F85000012804D1FFE71C
:107A200002208DF81F001EE10699012081F8500008
:107A3000FFE7FFE70699032081F85100069900202F
:107A400048650599069A1163BDF81210069A918649
:107A5000BDF81210069AD186069988630699888720
:107A60000699C8870699486406990864069880684C
:107A7000B0F5004F0DD1FFE706980168086820F0C7
:107A80004000086006980168086840F4804008607B
:107A9000FFE706980068006800F04000402807D023
:107AA000FFE706980168086840F040000860FFE7BB
:107AB0000698C068B0F5006F51D1FFE7069840689E
:107AC00028B1FFE7BDF8060001280ED1FFE70698B0
:107AD0000168006B0088C8600699086B0230086373
:107AE0000699C88E0138C886FFE7FFE70698C08E62
:107AF000A0B3FFE7069800688068800700280ED5CD
:107B0000FFE706980168006B0088C8600699086B5B
:107B1000023008630699C88E0138C8861DE0FEF75A
:107B20009FFD0299401A0399884204D3FFE7039806
:107B3000013018B9FFE7039870B9FFE706990120F3
:107B400081F85100FFE70699002081F85000FFE717
:107B500003208DF81F0086E0FFE7C7E750E0069896
:107B6000406828B1FFE7BDF8060001280ED1FFE705
:107B700006980168006B007808730699086B01305D
:107B800008630699C88E0138C886FFE7FFE70698A4
:107B9000C08EA0B3FFE706980068806880070028C1
:107BA0000ED5FFE706980168006B00780873069908
:107BB000086B013008630699C88E0138C8861DE03D
:107BC000FEF74EFD0299401A0399884204D3FFE75D
:107BD0000398013018B9FFE7039870B9FFE70699D9
:107BE000012081F85100FFE70699002081F850003C
:107BF000FFE703208DF81F0035E0FFE7C7E7FFE749
:107C000006980399029A03F00FFD20B1FFE7069949
:107C100020204865FFE70698806870B9FFE7FFE716
:107C20000020009006980068C068009006980068E0
:107C3000806800900098FFE7FFE70699012081F82F
:107C40005100FFE70699002081F85000FFE70698F1
:107C5000406D20B1FFE701208DF81F0003E00020F8
:107C60008DF81F00FFE79DF81F0008B080BD0000E1
:107C700080B58CB0DDF838C00A9009910892ADF853
:107C80001E3001200390FEF7EBFC04900A9890F858
:107C900051008DF817000A9840680690BDF81E0044
:107CA000ADF81C009DF81700012812D0FFE70698D8
:107CB000B0F5827F09D1FFE70A98806828B9FFE70D
:107CC0009DF81700042804D0FFE702208DF82F004C
:107CD0009BE1099838B1FFE7089820B1FFE7BDF8AC
:107CE0001E0020B9FFE701208DF82F008DE1FFE78E
:107CF0000A9890F85000012804D1FFE702208DF87F
:107D00002F0082E10A99012081F85000FFE7FFE788
:107D10000A9890F85100042805D0FFE70A99052039
:107D200081F85100FFE70A990020486508990A9AEE
:107D30009163BDF81E100A9AD187BDF81E100A9AE9
:107D4000918709990A9A1163BDF81E100A9AD18683
:107D5000BDF81E100A9A91860A9908640A99486427
:107D60000A980068006800F04000402807D0FFE74C
:107D70000A980168086840F040000860FFE70A9828
:107D8000C068B0F5006F40F08180FFE70A98406856
:107D900028B1FFE7BDF81C0001280ED1FFE70A98C3
:107DA0000168006B0088C8600A99086B023008639C
:107DB0000A99C88E0138C886FFE7FFE70A98C18E86
:107DC0000120019039B9FFE70A98C08F002818BF39
:107DD00001200190FFE70198C007002855D0FFE778
:107DE0000A98006880688007002818D5FFE70A987D
:107DF000C08EA0B1FFE70398012810D1FFE70A98D1
:107E00000168006B0088C8600A99086B023008633B
:107E10000A99C88E0138C88600200390FFE70A98A7
:107E200000688068C007A8B1FFE70A98C08F88B1D2
:107E3000FFE70A980068C0680A99896B08800A9968
:107E4000886B023088630A99C88F0138C88701207F
:107E50000390FFE7FEF704FC0499401A0E9988424C
:107E600012D3FFE70E98013070B1FFE70A990120A5
:107E700081F85100FFE70A99002081F85000FFE7E0
:107E800003208DF82F00C0E098E782E00A98406850
:107E900028B1FFE7BDF81C0001280ED1FFE70A98C2
:107EA0000168006B007808730A99086B0130086359
:107EB0000A99C88E0138C886FFE7FFE70A98C18E85
:107EC0000120009039B9FFE70A98C08F002818BF39
:107ED00001200090FFE70098C007002858D0FFE776
:107EE0000A98006880688007002818D5FFE70A987C
:107EF000C08EA0B1FFE70398012810D1FFE70A98D0
:107F00000168006B007808730A99086B01300863F8
:107F10000A99C88E0138C88600200390FFE70A98A6
:107F200000688068C007A8B1FFE70A98C08F88B1D1
:107F3000FFE70A980068C0680A99896B08700A9977
:107F4000886B013088630A99C88F0138C88701207F
:107F50000390FFE7FEF784FB0499401A0E998842CC
:107F600004D3FFE70E98013018B9FFE70E9870B9F7
:107F7000FFE70A99012081F85100FFE70A990020E4
:107F800081F85000FFE703208DF82F003DE095E7D2
:107F9000FFE70A980E99049A03F046FB68B1FFE7E1
:107FA0000A9920204865FFE70A99002081F85000CF
:107FB000FFE701208DF82F0027E00A98806870B94C
:107FC000FFE7FFE7002002900A980068C06802906F
:107FD0000A980068806802900298FFE7FFE70A9914
:107FE000012081F85100FFE70A99002081F8500034
:107FF000FFE70A98406D20B1FFE701208DF82F00C0
:1080000003E000208DF82F00FFE79DF82F000CB053
:1080100080BD000080B588B0069005910492ADF84F
:108020000E30069890F851008DF8070006984068C9
:1080300002909DF80700012812D0FFE70298B0F5E2
:10804000827F09D1FFE70698806828B9FFE79DF88D
:108050000700042804D0FFE702208DF81F00DFE0AE
:10806000059838B1FFE7049820B1FFE7BDF80E008E
:1080700020B9FFE701208DF81F00D1E0FFE7069847
:1080800090F85000012804D1FFE702208DF81F006E
:10809000C6E00699012081F85000FFE7FFE7069847
:1080A00090F85100042805D0FFE70699052081F8D3
:1080B0005100FFE70699002048650599069A11636B
:1080C000BDF80E10069A9186BDF80E10069AD1865C
:1080D0000499069A9163BDF80E10069A9187BDF82F
:1080E0000E10069AD1870699086406994864069886
:1080F00090F8510004280FD1FFE70698C16C4BF2AD
:108100002930C0F6000008640698C16C4BF271304B
:10811000C0F60000C8630EE00698C16C4BF25930FF
:10812000C0F6000008640698C16C4BF2BD40C0F672
:108130000000C863FFE70698C16C4BF2F520C0F65B
:108140000000C8640698C16C00200865069B196889
:108150009A6BD86C0C31DB8FFDF7A2FF78B1FFE78B
:108160000699486D40F010004865FFE70699002029
:1081700081F85000FFE701208DF81F0050E00698BD
:108180000168486840F0010048600698816C002052
:1081900008640699896CC8630699896CC864069955
:1081A000896C0865069B1A68196B986C0C32DB8E1B
:1081B000FDF776FF78B1FFE70699486D40F01000B3
:1081C0004865FFE70699002081F85000FFE701208D
:1081D0008DF81F0024E006980068006800F0400059
:1081E000402807D0FFE706980168086840F0400083
:1081F0000860FFE7FFE70699002081F85000FFE7DD
:1082000006980168486840F02000486006980168B8
:10821000486840F00200486000208DF81F00FFE72A
:108220009DF81F0008B080BD80B584B00290019118
:10823000ADF80220029890F85100012804D0FFE721
:1082400002208DF80F00A1E0019820B1FFE7BDF8F2
:10825000020020B9FFE701208DF80F0096E0FFE74C
:10826000029890F85000012804D1FFE702208DF811
:108270000F008BE00299012081F85000FFE7FFE733
:108280000299032081F85100029900204865019964
:10829000029A1163BDF80210029A9186BDF802108D
:1082A000029AD18602998863029948640299086407
:1082B000029988870299C88702988068B0F5004FB4
:1082C0000DD1FFE702980168086820F040000860BF
:1082D00002980168086840F480400860FFE702984F
:1082E000816C4BF24130C0F6000008640298816C4A
:1082F0004BF21540C0F60000C8630298816C4BF247
:10830000F520C0F60000C8640298816C0020086562
:10831000029B1A68196B986C0C32DB8EFDF7C0FE5D
:1083200078B1FFE70299486D40F010004865FFE71B
:108330000299002081F85000FFE701208DF80F001E
:1083400024E002980068006800F04000402807D050
:10835000FFE702980168086840F040000860FFE706
:10836000FFE70299002081F85000FFE702980168BA
:10837000486840F02000486002980168486840F072
:108380000200486000208DF80F00FFE79DF80F0005
:1083900004B080BD80B582B00190019803F0AAF9C5
:1083A0008DF803009DF80300022815D0FFE79DF823
:1083B0000300410140F21820C2F20000405850B1C1
:1083C000FFE79DF80300410140F21820C2F20000CF
:1083D00040588047FFE7FFE702B080BD80B582B01C
:1083E0000190019803F086F98DF803009DF80300D1
:1083F00002281BD0FFE7019803F07CF9014640F208
:108400001820C2F2000000EB4110C06868B1FFE71D
:10841000019803F06FF9014640F21820C2F2000003
:1084200000EB4110C0688047FFE7FFE702B080BD66
:1084300080B582B00190019803F05CF98DF80300DB
:108440009DF8030002281BD0FFE7019803F052F9C2
:10845000014640F21820C2F2000000EB4110806893
:1084600068B1FFE7019803F045F9014640F2182092
:10847000C2F2000000EB411080688047FFE7FFE791
:1084800002B080BD80B582B00190019803F032F94E
:108490008DF803009DF8030002281BD0FFE7019828
:1084A00003F028F9014640F21820C2F2000000EB68
:1084B0004110406968B1FFE7019803F01BF90146DC
:1084C00040F21820C2F2000000EB411040698047E2
:1084D000FFE7FFE702B080BD80B582B00190019850
:1084E00003F0DAF902B080BD81B0009001B07047AE
:1084F00081B0009001B0704785B003900291FFE712
:10850000039890F83C00012804D1FFE702208DF881
:1085100013007EE00399012081F83C00FFE7FFE7AC
:108520000399022081F83D0003980068406801909B
:108530000398006880680090019820F07000019016
:10854000029801680198084301900198039909680D
:108550004860039800680021C4F2010188423CD0C1
:10856000FFE703980068B0F1804F36D0FFE703982B
:10857000006840F20041C4F2000188422DD0FFE7BC
:108580000398006840F60001C4F20001884224D03C
:10859000FFE70398006840F60041C4F200018842FA
:1085A0001BD0FFE70398006840F20041C4F20101CC
:1085B000884212D0FFE70398006844F20001C4F239
:1085C0000101884209D0FFE70398006841F60001E5
:1085D000C4F2000188420ED1FFE7009820F080002D
:1085E0000090029841680098084300900098039911
:1085F00009688860FFE70399012081F83D00FFE7E3
:108600000399002081F83C00FFE700208DF813005B
:10861000FFE79DF8130005B07047000080B582B0F9
:108620000090009820B9FFE701208DF807003FE097
:10863000009890F83D0040B9FFE70099002081F8CC
:108640003C00009800F038F8FFE70099022081F81C
:108650003D00009951F8040B03F0C4F90099012082
:1086600081F84600FFE70099012081F83E0000995B
:1086700081F83F00009981F84000009981F841009D
:10868000FFE7FFE70099012081F84200009981F897
:108690004300009981F84400009981F84500FFE704
:1086A0000099012081F83D0000208DF80700FFE7C8
:1086B0009DF8070002B080BD80B586B00590059892
:1086C000006840F60001C4F20001884212D1FFE7C1
:1086D000FFE70020049043F64000C4F20200016866
:1086E00041F004010160006800F004000490049867
:1086F000FFE740E00598006841F20041C4F2000144
:1087000088421BD1FFE7FFE70020039043F64000BB
:10871000C4F20200016841F020010160006800F02D
:10872000200003900398FFE73720019005210022E5
:10873000FEF73EF80198FEF731F81BE00598006857
:1087400044F20041C4F20101884212D1FFE7FFE781
:108750000020029043F64400C4F20200016841F494
:1087600000310160006800F4003002900298FFE7D9
:10877000FFE7FFE7FFE706B080BD000080B586B0E9
:108780000490039100208DF80B00FFE7049890F807
:108790003C00012804D1FFE702208DF81700ABE070
:1087A0000499012081F83C00FFE7FFE704990220CB
:1087B00081F83D000498006880680190019820F0DD
:1087C00077000190019820F47F400190019804996E
:1087D00009688860039800680090002872D0FFE75D
:1087E000009810286ED0FFE7009820286AD0FFE795
:1087F0000098302866D0FFE70098402855D0FFE762
:108800000098502837D0FFE70098602840D0FFE755
:10881000009870280BD0FFE70098B0F5805F05D076
:10882000FFE70098B0F5005F16D052E055E00498DD
:108830000068039B5A689968DB6803F0C1F90498E3
:10884000006880680190019840F0770001900198DD
:1088500004990968886040E004980068039B5A689E
:108860009968DB6803F0ACF904980168886840F403
:108870008040886031E004980068039A5168D268AB
:1088800003F08AFB04980068502103F0B3F924E058
:1088900004980068039A5168D26803F0A5FB049815
:1088A0000068602103F0A6F917E004980068039AB5
:1088B0005168D26803F070FB04980068402103F00F
:1088C00099F90AE0049800680399096803F092F99D
:1088D00003E001208DF80B00FFE70499012081F8E7
:1088E0003D00FFE70499002081F83C00FFE79DF878
:1088F0000B008DF81700FFE79DF8170006B080BD4C
:1089000081B0009001B0704780B584B003900398A7
:108910000068C068029003980068006901909DF8A3
:1089200004008007002824D5FFE79DF80800800791
:1089300000281DD5FFE7039801686FF00200086169
:10894000039901200877039800688069800720B1A7
:10895000FFE70398FFF7D4FF06E0039800F044F91F
:10896000039800F039FAFFE7039900200877FFE742
:10897000FFE79DF804004007002825D5FFE79DF894
:108980000800400700281ED5FFE7039801686FF034
:108990000400086103990220087703980068806941
:1089A00010F4407F04D0FFE70398FFF7A9FF06E02B
:1089B000039800F019F9039800F00EFAFFE7039905
:1089C00000200877FFE7FFE79DF804000007002874
:1089D00024D5FFE79DF80800000700281DD5FFE714
:1089E000039801686FF00800086103990420087774
:1089F00003980068C069800720B1FFE70398FFF77C
:108A00007FFF06E0039800F0EFF8039800F0E4F928
:108A1000FFE7039900200877FFE7FFE79DF80400D0
:108A2000C006002825D5FFE79DF80800C0060028ED
:108A30001ED5FFE7039801686FF0100008610399E5
:108A40000820087703980068C06910F4407F04D0BC
:108A5000FFE70398FFF754FF06E0039800F0C4F81F
:108A6000039800F0B9F9FFE7039900200877FFE7C2
:108A7000FFE79DF80400C00778B1FFE79DF8080004
:108A8000C00748B1FFE7039801686FF00100086173
:108A9000039800F08BFAFFE7FFE79DF8040000065B
:108AA000002810D5FFE79DF808000006002809D52A
:108AB000FFE7039801686FF0800008610398FFF7F3
:108AC00013FDFFE7FFE79DF804004006002810D5DE
:108AD000FFE79DF808004006002809D5FFE7039846
:108AE00001686FF040000861039800F063FAFFE747
:108AF000FFE79DF804008006002810D5FFE79DF8E9
:108B000008008006002809D5FFE7039801686FF088
:108B1000200008610398FFF7EBFCFFE7FFE704B0D4
:108B200080BD000080B588B00790002006900590B9
:108B30000490039002900798006840F60001C4F288
:108B40000001884222D1FFE7FFE70020019043F6B1
:108B50003000C4F20200016841F0080101600068C1
:108B600000F0080001900198FFE74FF48040029068
:108B700002200390002104910591069040F60040E8
:108B8000C4F2020002A9FDF75FFB2BE00798006822
:108B900044F20041C4F20101884222D1FFE7FFE71D
:108BA0000020009043F63000C4F20200016841F05A
:108BB00020010160006800F0200000900098FFE7AD
:108BC0004020029002200390002104910590032090
:108BD000069041F20040C4F2020002A9FDF734FB06
:108BE000FFE7FFE708B080BD81B0009001B070479B
:108BF00080B586B004900391029200208DF80700A2
:108C0000FFE7049890F83C00012804D1FFE7022018
:108C10008DF8170089E00499012081F83C00FFE7F6
:108C2000FFE7029800900C2800F270800099DFE8BE
:108C300001F0076D6D6D206D6D6D3A6D6D6D5300BA
:108C400004980068039902F0EBFF049801688869B2
:108C500040F00800886104980168886920F00400E9
:108C600088610398026904980168886910438861E3
:108C700050E004980068039903F048F804980168EC
:108C8000886940F40060886104980168886920F46C
:108C9000806088610398026904980168886940EAE5
:108CA0000220886136E004980068039903F0A8F870
:108CB00004980168C86940F00800C8610498016818
:108CC000C86920F00400C86103980269049801682B
:108CD000C8691043C8611DE004980068039903F057
:108CE00009F904980168C86940F40060C8610498F3
:108CF0000168C86920F48060C8610398026904981B
:108D00000168C86940EA0220C86103E001208DF8CB
:108D10000700FFE7FFE70499002081F83C00FFE728
:108D20009DF807008DF81700FFE79DF8170006B0C3
:108D300080BD000080B582B00090009820B9FFE7A8
:108D400001208DF807003FE0009890F83D0040B901
:108D5000FFE70099002081F83C00009800F038F807
:108D6000FFE70099022081F83D00009951F8040BBB
:108D700002F038FE0099012081F84600FFE70099D3
:108D8000012081F83E00009981F83F00009981F8A8
:108D90004000009981F84100FFE7FFE700990120BA
:108DA00081F84200009981F84300009981F844005D
:108DB000009981F84500FFE70099012081F83D0006
:108DC00000208DF80700FFE79DF8070002B080BD86
:108DD00081B0009001B0704781B0009001B0704741
:108DE00080B58CB00A900991099828B9FFE70A98D4
:108DF00090F83E0007901CE00998042805D1FFE791
:108E00000A9890F83F00069010E00998082805D1CC
:108E1000FFE70A9890F84000059004E00A9890F85F
:108E200041000590FFE705980690FFE70698079038
:108E3000FFE70798012804D0FFE701208DF82F00F5
:108E4000AFE0099828B9FFE70A99022081F83E00AF
:108E50001EE00998042806D1FFE70A99022081F84C
:108E60003F00049012E00998082806D1FFE70A990C
:108E7000022081F84000039005E00A99022081F861
:108E800041000390FFE703980490FFE70498FFE791
:108E90000A98006809990122019202F075FE019872
:108EA0000A9909680022C4F20102914202900CD092
:108EB000FFE70A9800684FF60041CBF6FE710844C0
:108EC000B0FA80F040090290FFE70298C00738B17D
:108ED000FFE70A980168486C40F400404864FFE7E7
:108EE0000A9800680021C4F2010188423CD0FFE7E3
:108EF0000A980068B0F1804F36D0FFE70A98006802
:108F000040F20041C4F2000188422DD0FFE70A98E8
:108F1000006840F60001C4F20001884224D0FFE757
:108F20000A98006840F60041C4F2000188421BD054
:108F3000FFE70A98006840F20041C4F2010188424C
:108F400012D0FFE70A98006844F20001C4F2010160
:108F5000884209D0FFE70A98006841F60001C4F290
:108F60000001884212D1FFE70A980068806800F08B
:108F7000070008900898062807D0FFE70A980168BC
:108F8000086840F001000860FFE706E00A98016801
:108F9000086840F001000860FFE700208DF82F000E
:108FA000FFE79DF82F000CB080BD000081B000905D
:108FB00001B0704781B0009001B0704782B001905D
:108FC000ADF8021002B0704780B582B001900198F0
:108FD00003F0DEFB8DF803009DF8030003281BD08F
:108FE000FFE79DF8030000EBC00140F23820C2F219
:108FF000000000EB8100006968B1FFE79DF8030005
:1090000000EBC00140F23820C2F2000000EB81000A
:1090100000698047FFE7FFE702B080BD80B592B0EE
:109020001190119800680068109011980068C0684D
:109030000F901198006840690E9000200D900C90E0
:10904000109800F00F000D900D9888B9FFE79DF87B
:109050004000800600280AD5FFE79DF83C00800606
:10906000002804D5FFE7119803F0B6FB02E2FFE702
:109070000D98002800F0C280FFE79DF83800C00777
:1090800038B9FFE7BDF83C0010F4907F00F0B680DF
:10909000FFE79DF84000C00758B1FFE79DF83D008D
:1090A000C00730B1FFE71199486C40F001004864F7
:1090B000FFE79DF84000400700280BD5FFE79DF82B
:1090C0003800C00730B1FFE71199486C40F002004A
:1090D0004864FFE79DF84000800700280BD5FFE7B4
:1090E0009DF83800C00730B1FFE71199486C40F097
:1090F00004004864FFE79DF840000007002811D5F0
:10910000FFE79DF83C008006002805D4FFE79DF8A6
:109110003800C00730B1FFE71199486C40F00800F3
:109120004864FFE71198406C002866D0FFE79DF87F
:109130004000800600280AD5FFE79DF83C00800625
:10914000002804D5FFE7119803F046FBFFE71198CC
:1091500000684069C0F380100C901198406C0007C3
:10916000002804D4FFE70C9800283ED0FFE71198B0
:1091700003F0B0FA119800684069400600282FD526
:10918000FFE7FFE7FFE71198006850E8050F20F0C0
:1091900040000B90FFE70B991198026842E8051018
:1091A0000028F0D1FFE7FFE71198C06B98B1FFE707
:1091B0001198C16B4CF2B960C0F6000008651198B7
:1091C000C06BFCF703FD28B1FFE71198C06B016D80
:1091D0008847FFE703E01198FFF7F6FEFFE703E09B
:1091E0001198FFF7F1FEFFE706E01198FFF7ECFE9C
:1091F000119900204864FFE7FFE73BE11198006BFD
:10920000012840F01781FFE79DF84000C0060028C4
:1092100040F11081FFE79DF83C00C006002840F1B6
:109220000981FFE7FFE700200A90119800680068B5
:109230000A901198006840680A900A98FFE7119810
:10924000006840694006002840F19A80FFE71198C5
:10925000C06B00684068ADF82600BDF82600002805
:1092600075D0FFE7BDF826001199898D88426EDA26
:10927000FFE7BDF826001199C8851198C06BC06939
:10928000B0F5807F58D0FFE7FFE7FFE7119800684F
:1092900050E8030F20F480700890FFE708991198B8
:1092A000026842E803100028F0D1FFE7FFE7FFE77C
:1092B000FFE71198006850E8050F20F001000790C3
:1092C000FFE707991198026842E805100028F0D1DD
:1092D000FFE7FFE7FFE7FFE71198006850E8050F99
:1092E00020F040000690FFE706991198026842E8D6
:1092F00005100028F0D1FFE7FFE71199202081F841
:109300004200119900200863FFE7FFE71198006809
:1093100050E8030F20F010000590FFE70599119821
:10932000026842E803100028F0D1FFE7FFE7119838
:10933000C06BFCF7D5FBFFE7119902204863119839
:10934000818DC28D891A89B2FFF738FE17E0BDF80A
:1093500026001199898D884210D1FFE71198C06BC2
:10936000C069B0F5807F08D1FFE7119902204863FA
:109370001198818DFFF722FEFFE7FFE7FFE779E015
:109380001199888DC98D401AADF812001198C08DC1
:1093900000284ED0FFE7BDF81200002849D0FFE7B3
:1093A000FFE7FFE71198006850E8030F20F4907082
:1093B0000390FFE703991198026842E80310002820
:1093C000F0D1FFE7FFE7FFE7FFE71198006850E8FB
:1093D000050F20F001000290FFE702991198026842
:1093E00042E805100028F0D1FFE7FFE7119920209F
:1093F00081F84200119900200863FFE7FFE7119808
:10940000006850E8030F20F010000190FFE7019979
:109410001198026842E803100028F0D1FFE7FFE747
:109420001199022048631198BDF81210FFF7C6FD8C
:10943000FFE71FE09DF84000000600280AD5FFE77F
:109440009DF83C000006002804D5FFE7119803F0C2
:1094500015FB0FE09DF84000400600280AD5FFE705
:109460009DF83C004006002804D5FFE7119803F062
:109470007BF9FFE712B080BD80B582B00090009804
:1094800020B9FFE701208DF8070040E000988069CF
:1094900008B1FFE700E0FFE7009890F8410040B90D
:1094A000FFE70099002081F84000009800F034F8B0
:1094B000FFE70099242081F8410000980168C868FE
:1094C00020F40050C860009803F03AFA0098016850
:1094D000086920F49040086100980168486920F00C
:1094E0002A00486100980168C86840F40050C860CC
:1094F000009900204864009A202182F84110009AC7
:1095000082F84210009948638DF80700FFE79DF844
:10951000070002B080BD000080B59CB01B90002009
:109520001A9019901890179016901B98006841F2A5
:109530000001C4F20101884240F09380FFE7FFE799
:109540000020159043F64400C4F20200016841F087
:1095500010010160006800F0100015901598FFE7F9
:10956000FFE70020149043F63000C4F202000168C7
:1095700041F002010160006800F0020014901498AC
:10958000FFE7FFE70020139043F63000C4F202002B
:10959000016841F001010160006800F001001390D2
:1095A0001398FFE780201690022009901790002062
:1095B0000D90189003200A90199007200B901A9094
:1095C00040F20040C4F2020016A90C91FCF73CFEE8
:1095D000DDF824C00A9A0B980C990D9B4FF4007E7D
:1095E000CDF858E0CDF85CC0189319921A9000207D
:1095F000C4F20200FCF728FE0D9940F63020C2F2BA
:1096000000000E9046F28842C4F2020202604FF05F
:10961000006242608160C1604FF48062026141611A
:109620008161C1614FF4403202624162FCF780FC0B
:1096300018B1FFE7FBF732F9FFE7FFE71B9840F6A9
:109640003021C2F20001C1631B988863FFE7252027
:10965000089005210022FDF7ABF80898FDF79EF869
:1096600014E11B98006844F60001C4F2000188422E
:109670006AD1FFE7FFE70020129043F64000C4F2F2
:109680000200016841F480210160006800F480203C
:1096900012901298FFE7FFE70020119043F6300088
:1096A000C4F20200016841F004010160006800F0AA
:1096B000040011901198FFE74FF4406016900220CB
:1096C00017900020069018900320199007201A90F8
:1096D00040F60000C4F2020016A9FCF7B5FD069999
:1096E00040F69020C2F20000079046F22802C4F231
:1096F000020202604FF0006242608160C1604FF47C
:109700008062026141618161C1614FF40032026295
:109710004162FCF70DFC18B1FFE7FBF7BFF8FFE76C
:10972000FFE71B9840F69021C2F20001C1631B982D
:109730008863FFE72720059005210022FDF738F810
:109740000598FDF72BF8A0E01B98006841F2004156
:10975000C4F20101884240F09780FFE7FFE7002054
:10976000109043F64400C4F20200016841F0200169
:109770000160006800F0200010901098FFE7FFE7FC
:1097800000200F9043F63000C4F20200016841F05F
:1097900040010160006800F040000F900F98FFE763
:1097A0004FF48440169002201790002003901890E8
:1097B0000320199008201A9041F60000C4F202001C
:1097C00016A9FCF741FD039940F6F020C2F2000013
:1097D000049046F22842C4F2020202604FF0206276
:1097E00042608160C1604FF48062026141618161C9
:1097F000C1614FF4803202624162FCF799FB18B1FB
:10980000FFE7FBF74BF8FFE7FFE71B9840F6F02177
:10981000C2F20001C1631B988863FFE740F6503035
:10982000C2F20000029046F2A041C4F202010160BF
:109830004FF020614160402181600021C1604FF400
:109840008062026141618161C1614FF480320262D4
:109850004162FCF76DFB18B1FFE7FBF71FF8FFE76C
:10986000FFE71B9840F65031C2F2000181631B985C
:109870008863FFE74720019005210022FCF798FF4D
:109880000198FCF78BFFFFE7FFE7FFE71CB080BD07
:1098900080B582B00190019802F07AFF8DF8030044
:1098A0009DF8030003281BD0FFE79DF8030000EBA1
:1098B000C00140F23820C2F2000000EB8100C06815
:1098C00068B1FFE79DF8030000EBC00140F23820CB
:1098D000C2F2000000EB8100C0688047FFE7FFE7AD
:1098E00002B080BD80B582B00190019802F050FFB7
:1098F0008DF803009DF8030003281BD0FFE79DF8B7
:10990000030000EBC00140F23820C2F2000000EB7F
:109910008100406868B1FFE79DF8030000EBC001DB
:1099200040F23820C2F2000000EB8100406880471E
:10993000FFE7FFE702B080BDFFE7FEE784B08DEDF3
:10994000030A9DED030AB6EE001A20EE010A8DED22
:10995000020A0398019001980090009945F6DF10E3
:10996000C5F63770A0EB61000090009801909DED66
:10997000010A9DED021A21EE001A21EE002AB7EE2F
:10998000081A31EE422A20EE020A8DED010A9DED01
:10999000010A9DED022A22EE002A22EE002A31EE73
:1099A000421A20EE010A8DED010A9DED010A04B074
:1099B0007047000080B586B004908DED030A0498CE
:1099C00018B9FFE7002005904CE09DED030A0498CC
:1099D00090ED014A90ED022A90ED063A90ED071ABB
:1099E00023EE043A30EE430A21EE021A30EE410A29
:1099F0008DED020A002028B9FFE7029803F094F9E0
:109A000058B90DE002980AF0D7FA41EC100B51EC6E
:109A1000100B03F06FF918B1FFE703980290FFE70E
:109A20009DED020A049890ED034A90ED043A90ED02
:109A3000052A90ED061A20EE040A21EE031A30EEF4
:109A4000010A90ED071A21EE021A30EE010A8DED9F
:109A5000010A04998869C86102980499886101988B
:109A60000590FFE79DED050A06B080BD80B588B082
:109A700007908DED060ACDED050A079808B9FFE7B6
:109A80008BE005980799086007990020886107997D
:109A9000C861079890ED000AB5EE400AF1EE10FAA1
:109AA0000EDCFFE707994FF07E50C8600799002051
:109AB00008610799486107994860079988606CE0D8
:109AC0009DED060A079890ED001A80EE010A8DEDD3
:109AD000040A9DED041A9FED320A80EE010A08F097
:109AE000A9FD8DED030A9FED2F0A8DED000A08F008
:109AF000D3FBB0EE401A9DED000A31EE011A9DED48
:109B0000033A21EE031AB7EE002A8DED012A31EE59
:109B1000021A23EE033A31EE031A8DED021A9DED7F
:109B2000031A21EE011A9DED023A81EE031A0798FD
:109B300080ED031A079890ED031A31EE011A80EDBB
:109B4000041A0799C86848619DED031A21EE011AAD
:109B500031EE421A31EE011A9DED022A81EE021A0F
:109B6000079880ED011A08F097FBB0EE401A9DEDC2
:109B7000010A31EE012A9DED031A22EE012A30EE90
:109B8000420A21EE011A30EE010A9DED021A80EE22
:109B9000010A079880ED020AFFE708B080BD00BF08
:109BA000DB0F4940DB0F493F80B584B002908DED5B
:109BB000010A029818B9FFE70020039039E09DEDF3
:109BC000010A029890ED031A90ED043A90ED052AEF
:109BD00031EE031A31EE021A80EE010A8DED000A11
:109BE000002028B9FFE7009803F06CF858B911E09D
:109BF00000980AF0E1F941EC100B51EC100B03F066
:109C000041F838B1FFE700980299886100980299FD
:109C1000C86106E001980299886101980299C861BB
:109C2000FFE702989DED010AFFF7C4FE8DED030AE0
:109C3000FFE79DED030A04B080BD000082B00090F4
:109C4000009820B9FFE74FF04040019003E00098F2
:109C500040690190FFE79DED010A02B070470000E6
:109C600082B00090009820B9FFE74FF0404001908B
:109C700003E0009880690190FFE79DED010A02B0C2
:109C80007047000080B582B08DF806009DF8060090
:109C9000022804DBFFE7FF208DF8070039E09DF87C
:109CA000061040F20830C2F2000050F8210020B146
:109CB000FFE700208DF807002BE04820F8F7CCFFE5
:109CC00001469DF8062040F20830C2F2000040F83C
:109CD00022109DF8061050F8210020B9FFE7FF2060
:109CE0008DF8070015E09DF8061040F20830C2F22A
:109CF0000000009050F821004821F6F77AFB009907
:109D00009DF8060051F82010087000208DF807001B
:109D1000FFE79DF9070002B080BD000080B58EB05E
:109D20000C900C9820B9FFE7FE208DF83700AEE0CC
:109D30000C98007800F0B0F80B900B9820B9FFE772
:109D4000FC208DF83700A2E00B9802300A900C98A6
:109D50004088ADF81600BDF81610A1F2012001915F
:109D600004280CD3FFE70198A0F20520042829D38A
:109D7000FFE70198A0F20920032849D372E04FF4CD
:109D80000070069008208DF81C0000200490FFE76A
:109D90000498032815DCFFE70A98049A00EB4200B8
:109DA000407806A9053101F812000A98049A30F8A3
:109DB000120001EB42014870FFE704980130049063
:109DC000E6E753E040F2FF10069008208DF81C00F3
:109DD00004200390FFE70398072818DCFFE70A98A0
:109DE000039A00EB4200407806A9053101EB4202DC
:109DF00002F8080C0A98039A30F8120001EB4201AD
:109E000001F8070CFFE7039801300390E3E72DE02A
:109E100040F2FF20069008208DF81C000290FFE71A
:109E200002980A2818DCFFE70A98029A00EB420021
:109E3000407806A9053101EB420202F8100C0A989D
:109E4000029A30F8120001EB420101F80F0CFFE713
:109E5000029801300290E3E700208DF823008DF88E
:109E6000240003E0FF208DF8370010E00C98007804
:109E70000121F8F79FFD0C98007806A9F8F77AFD04
:109E8000002818BF4FF0FF308DF83700FFE79DF92D
:109E900037000EB080BD000082B08DF803009DF841
:109EA0000300022803DBFFE70020019009E09DF892
:109EB000031040F20830C2F2000050F82100019077
:109EC000FFE7019802B0704782B08DF805009DF859
:109ED00005000146009140B1FFE70098012809D034
:109EE000FFE7009802280AD00EE042F21070ADF8A9
:109EF00006000EE04FF48040ADF8060009E047F29E
:109F00003050ADF8060004E04FF6FF70ADF80600E3
:109F1000FFE7BDF9060002B07047000083B0ADF85E
:109F200008008DF807109DF80700014600910228EF
:109F300004D3FFE70098022813D026E0BDF80800FC
:109F4000B0F5007F0CDDFFE7BDF80800B0F5027F3B
:109F500006DAFFE7BDF8080001388DF80B0019E0BC
:109F600014E0BDF80800B0F5017F0DDDFFE7BDF896
:109F7000080040F20A21884206DCFFE7BDF808002D
:109F800001388DF80B0005E000E0FFE7FF208DF8B9
:109F90000B00FFE79DF90B0003B0704780B586B05A
:109FA0000490049818B9FFE7002005902FE004986A
:109FB0000078FFF771FF0390039818B9FFE70020BE
:109FC000059024E000200290FFE70298039991F8A1
:109FD0004410884218DAFFE70398029900EB8100E9
:109FE00080690190019850B1FFE701984088049979
:109FF0004988884203D1FFE70198059007E0FFE711
:10A00000029801300290E0E700200590FFE70598F4
:10A0100006B080BD83B08DF807009DF807000146AB
:10A02000009140B1FFE70098012809D0FFE70098B0
:10A0300002280AD00DE00020C4F2102002900CE0AB
:10A040000020C4F29810029007E04FF07E5002907A
:10A0500003E04FF07E500290FFE79DED020A03B04F
:10A060007047000080B586B00490049820B9FFE7DF
:10A07000FE208DF8170081E004980078FFF702FEBB
:10A0800020B1FFE7FF208DF8170077E004980078F3
:10A09000FFF702FF0390039820B9FFE7FF208DF838
:10A0A00017006BE000200290FFE70298039991F8F7
:10A0B000441088421BDAFFE70398029900EB810005
:10A0C000806978B1FFE70398029900EB810080690D
:10A0D000408804994988884204D1FFE7FD208DF823
:10A0E00017004BE0FFE7029801300290DDE703988C
:10A0F00090F844000B2804DBFFE7FF208DF81700E1
:10A100003CE05020F8F7A8FD0190019820B9FFE746
:10A11000FF208DF8170031E00199049A1068526809
:10A120004A600860019818302821F6F762F904980F
:10A130004079019900F0010081F82800049908781D
:10A1400049880322F8F77AFA38B1FFE70198F8F75F
:10A1500091FCFF208DF8170010E00198039991F809
:10A16000442001EB82018861039991F84400013099
:10A1700081F8440000208DF81700FFE79DF91700D3
:10A1800006B080BD80B58AB007A90191014601984B
:10A19000089180ED000A089820B9FFE7FE208DF8AD
:10A1A000270078E008980078FFF776FE069006987A
:10A1B00020B9FFE7FC208DF827006CE0019890EDB6
:10A1C000000AB7EE001AB4EE410AF1EE10FA04DD0F
:10A1D000FFE74FF07E500790FFE7019890ED000AEF
:10A1E000BFEE001AB4EE410AF1EE10FA05DAFFE70D
:10A1F0000020CBF680700790FFE708984079C007F1
:10A2000040B1FFE7019890ED000AB1EE400A80ED01
:10A21000000AFFE70898FFF7C1FE0590059820B9EE
:10A22000FFE7FC208DF8270035E008994888097978
:10A23000FFF774FE8DF813009DF91300B0F1FF3F96
:10A2400004DCFFE7FF208DF8270024E00198069941
:10A250000231039190ED000A8DED000A0898007913
:10A26000FFF732FE9DED000A01EE100AB8EEC11AAA
:10A2700020EE010ABDEEC00A10EE100AADF80A0089
:10A28000BDF80A0003999DF9132021F8120000205F
:10A290008DF82700FFE79DF927000AB080BD000078
:10A2A00080B590B00E900E9820B9FFE7FE208DF893
:10A2B0003F0072E00E980078FFF7EEFD0D900D98CC
:10A2C00020B9FFE7FC208DF83F0066E000200C90ED
:10A2D000FFE70C980D9991F84410884259DAFFE78E
:10A2E0000D980C9900EB810080690B900B98002869
:10A2F0004AD0FFE70B9840880E994988884243D19D
:10A30000FFE70E990878498804AA0023F8F75AF85D
:10A31000E8B1FFE7F8F768FE03910290029903980D
:10A320000B9A136A526AC91A904140F2E932891AAB
:10A3300070F1000007D3FFE70B9900200876FC209E
:10A340008DF83F0029E0FF208DF83F0025E00B99B4
:10A3500001200876F8F748FE0A460B994A6208621F
:10A360000B9804A900F090FB0B9901918868CA68CA
:10A370000B69D1F814C0C1F838C04B630A63C862D6
:10A3800000208DF83F0008E0FFE70C9801300C90AA
:10A390009FE7FC208DF83F00FFE79DF93F0010B0DC
:10A3A00080BD000080B586B000208DF817000490B5
:10A3B000FFE70498012830DCFFE79DF81000FFF765
:10A3C0006BFD0390039808B9FFE722E0002002909C
:10A3D000FFE70298039991F84410884218DAFFE7E2
:10A3E0000398029900EB810080690190019850B1B7
:10A3F000FFE70198FFF754FF20B1FFE7FF208DF83A
:10A400001700FFE7FFE7FFE7029801300290E0E75F
:10A41000FFE7049801300490CBE79DF9170006B0E0
:10A4200080BD000080B582B040F62010C2F200006E
:10A43000009046F20041C4F2000101600321416036
:10A44000002101918160C1604FF4A02202614FF4AC
:10A45000C0024261017641768176C176017741770B
:10A46000FAF754FF18B1FFE7FAF718FAFFE702B05E
:10A4700080BD000080B582B040F64810C2F20000F6
:10A48000009046F60001C4F2000101600321416022
:10A49000002101918160C1604FF4C02202614FF43C
:10A4A000A0024261017641768176C17601774177DB
:10A4B000FAF72CFF18B1FFE7FAF7F0F9FFE702B05F
:10A4C00080BD000080B58AB0FFE70020099043F608
:10A4D0003000C4F20200016841F40011016000681C
:10A4E00000F4001009900998FFE7FFE700200890AA
:10A4F00043F63000C4F20200016841F480010160BB
:10A50000006800F4800008900898FFE70C20009095
:10A510000521059100220692FCF74AF90098FCF704
:10A520003DF90599069A39200190FCF741F9019807
:10A53000FCF734F90599069A3A200290FCF738F9AD
:10A540000298FCF72BF90599069A3B200390FCF73B
:10A550002FF90398FCF722F90599069A44200490F4
:10A56000FCF726F90498FCF719F90599069A452095
:10A570000790FCF71DF90798FCF710F90AB080BDA9
:10A5800080B582B04BF68500C0F6000044F2B842B8
:10A59000C0F601020021019103F00CFB019940F685
:10A5A0001C12C2F2000210604CF23D00C0F6000026
:10A5B00044F28442C0F6010203F0FCFA02B080BD0E
:10A5C00080B59AB0002019901890179016901590A9
:10A5D000FFE70020149043F63000C4F20200016847
:10A5E00041F002010160006800F00200149014982C
:10A5F000FFE7FFE70020139043F63000C4F20200AB
:10A60000016841F040010160006800F040001390D3
:10A610001398FFE7FFE70020129043F63000C4F2E2
:10A620000200016841F001010160006800F00100D2
:10A6300012901298FFE7FFE70020119043F63000D8
:10A64000C4F20200016841F008010160006800F0F6
:10A65000080011901198FFE7FFE70020109043F6E3
:10A660003000C4F20200016841F00401016000689A
:10A6700000F0040010901098FFE7FFE700200F9013
:10A6800043F63000C4F20200016841F0800101602D
:10A69000006800F080000F900F98FFE7FFE70020B0
:10A6A0000E9043F63000C4F20200016841F0200130
:10A6B0000160006800F020000E900E98FFE741F660
:10A6C0000040C4F2020002904FF4E05101910022D8
:10A6D0000C92FBF7ADFF0020C4F2020004901021A1
:10A6E000039101220692FBF7A3FF069A40F2004075
:10A6F000C4F2020007901146FBF79AFF019B0298F3
:10A70000069A0C991593169217910221189115A982
:10A710000891FBF799FD0498069A089915924FF451
:10A720008813059316931792FBF78EFD039B0498ED
:10A73000069A08991593169217921892FBF784FDC2
:10A74000059A06980899302315931692179040F6AB
:10A750000000C4F20200FBF777FD069A07980899FB
:10A760001592169217921892FBF76EFD0C9A06201E
:10A77000099005210B91FCF71BF80998FCF70EF8DE
:10A780000B990C9A0A200A90FCF712F80A98FCF729
:10A7900005F80B990C9A17200D90FCF709F80D9805
:10A7A000FBF7FCFF1AB080BD80B582B040F6B03038
:10A7B000C2F20000019043F20001C4F20101016005
:10A7C0004FF48271416000218160C160016101220A
:10A7D00042614FF4007282611822C26101624162DB
:10A7E00081620A21C162FCF75FFD18B1FFE7FAF749
:10A7F00055F8FFE702B080BD80B588B00021009118
:10A80000079106910591049103910291019140F6FF
:10A810000840C2F2000044F20042C4F201020260A9
:10A820004160816041F28732C26001618161FDF760
:10A83000F5FE18B1FFE7FAF731F8FFE740F60840F8
:10A84000C2F20000FEF776FA18B1FFE7FAF726F831
:10A85000FFE760200190002202920392059240F6E9
:10A860000840C2F2000001A9FEF7C2F918B1FFE7E3
:10A87000FAF714F8FFE740F60840C2F20000FEF7CE
:10A8800051F908B080BD000080B58EB00021009164
:10A890000D910C910B910A910991089107910691E4
:10A8A0000591049103910291019140F65040C2F24A
:10A8B000000040F60002C4F20002026041608160C4
:10A8C00045F20722C26001618161FDF7A7FE18B160
:10A8D000FFE7F9F7E3FFFFE74FF480500A9040F6F7
:10A8E0005040C2F200000AA9FDF748FF18B1FFE787
:10A8F000F9F7D4FFFFE740F65040C2F20000FEF740
:10A9000019FA18B1FFE7F9F7C9FFFFE7002008902F
:10A91000099040F65040C2F2000008A9FDF7ECFD96
:10A9200018B1FFE7F9F7BAFFFFE7602001900020B8
:10A9300002900390059040F65040C2F2000001A939
:10A940000822FEF755F918B1FFE7F9F7A7FFFFE76F
:10A9500040F65040C2F20000FEF7E4F80EB080BDB1
:10A9600080B582B000210191009140F69840C2F27A
:10A97000000041F20042C4F20002026040F247329D
:10A980004260816040F2E732C2608161FDF746FEBD
:10A9900018B1FFE7F9F782FFFFE700200090019070
:10A9A00040F69840C2F200006946FDF7A5FD18B1D7
:10A9B000FFE7F9F773FFFFE702B080BD80B582B013
:10A9C00040F6E040C2F20000019041F20001C4F202
:10A9D000010101604FF4E131416000218160C160FB
:10A9E00001610C2242618161C161FEF745FD18B130
:10A9F000FFE7F9F753FFFFE702B080BD80B582B0F3
:10AA000040F62850C2F20000019044F60001C4F262
:10AA10000001016048F2A061C0F201014160002123
:10AA20008160C1604FF4806202610C2242618161E9
:10AA3000C161FEF721FD18B1FFE7F9F72FFFFFE72E
:10AA400002B080BD80B582B040F67050C2F2000006
:10AA5000019041F20041C4F2010101604FF4E13183
:10AA6000416000218160C16001610C22426181610D
:10AA7000C161FEF701FD18B1FFE7F9F70FFFFFE72E
:10AA800002B080BDFFE7FEE780B58AB0099008916B
:10AA90000898417B807B40EA0120ADF81E000898B1
:10AAA000C17B007C40EA0120ADF81C000898417C85
:10AAB000807C40EA0120ADF81A0009980079FFF780
:10AAC00003FAADF8180009980079FFF7A3FA8DEDA5
:10AAD000050ABDF81E0000EE100AB8EEC00A9FED90
:10AAE0006D1A80EE010A9FED6C1A20EE010A8DEDC1
:10AAF000040ABDF91C0000EE100AB8EEC00A8DED84
:10AB0000030ABDF91A00BDF91810484300EE100AF7
:10AB1000B8EEC00A9FED611A80EE010A8DED020ABF
:10AB200009988079C00700284CD0FFE7BDF81E00C7
:10AB30000999B1F84010401A01900198B0F5805F72
:10AB400005DDFFE70999486C013848640AE001987F
:10AB500010F5805F05DAFFE70999486C0130486419
:10AB6000FFE7FFE7BDF81E000999A1F8400004982F
:10AB70000090099890ED110AB8EEC00A9FED461AB0
:10AB800020EE010A9DED001A30EE010A9DED051A36
:10AB900080EE010A80ED120A0999886C88609DEDAB
:10ABA000030A9DED051A80EE010A099880ED030A5B
:10ABB0009DED020A9DED051A20EE010A099880ED2F
:10ABC000040A13E0099900204864BDF81E10099A90
:10ABD000A2F840100999886404980999886003983C
:10ABE0000999C860029809990861FFE7099890F8E7
:10ABF0002800C007002842D0FFE7FFE7099890ED42
:10AC0000020AB5EE400AF1EE10FA0ADAFFE70998F7
:10AC100090ED020A9FED201A30EE010A80ED020A43
:10AC2000ECE7FFE7099890ED020A9FED1B1AB4EEDE
:10AC3000410AF1EE10FA0ADBFFE7099890ED020AEB
:10AC40009FED171A30EE010A80ED020AEAE7099833
:10AC500090ED021A9FED100A30EE410A80ED020AD3
:10AC6000099890ED030AB1EE400A80ED030A0998B5
:10AC700090ED040AB1EE400A80ED040AFFE708985F
:10AC8000C07C00EE100AB8EE400A099880ED050A73
:10AC90000AB080BD00000046DB0FC94000008046BE
:10ACA000DB0FC9C0FFE7FEE788B007900691059269
:10ACB000079800F0070004900498C0F107000528E9
:10ACC00003D3FFE70420019004E00498C0F10700DB
:10ACD0000190FFE70198039004980430062803D8F8
:10ACE000FFE70020009003E0049803380090FFE79E
:10ACF0000098029006980399012202FA01F10139A5
:10AD00000840029B984005999A40013A1140084337
:10AD100008B0704780B590B00E908DED0D0ACDED66
:10AD20000C0A8DED0B1ACDED0A1A002028B9FFE7A9
:10AD30000D9801F0D3FF58B943E00D9809F03CF9A4
:10AD400041EC100B51EC100B01F0ACFFC8B3FFE766
:10AD5000002028B9FFE70C9801F0C0FF58B930E097
:10AD60000C9809F029F941EC100B51EC100B01F093
:10AD700099FF30B3FFE7002028B9FFE70B9801F0F7
:10AD8000ADFF58B91DE00B9809F016F941EC100B16
:10AD900051EC100B01F086FF98B1FFE7002028B9B5
:10ADA000FFE70A9801F09AFF78B90AE00A9809F0DB
:10ADB00003F941EC100B51EC100B01F073FF20B9BB
:10ADC000FFE70E9880690F9016E19DED0D0ADDED0D
:10ADD0000C0A0E98406890ED071AF9F7FBFB8DED11
:10ADE000090A9DED090A0E98406890ED001A20EEC0
:10ADF000010A8DED080A0E98406890ED000A9DED5D
:10AE00000C1A20EE010A8DED070A0E981C309DEDFC
:10AE1000070AFEF7CFFD8DED060A0E980078014671
:10AE2000019110B3FFE70198012804D0FFE70198D2
:10AE3000022817D01CE09DED060A0E9890ED021A2C
:10AE400090ED052A30EE420A9DED0A2AB4EE412A21
:10AE5000F1EE10FAC8BFB0EE421A80EE010A8DED95
:10AE6000050A05E00B98059002E000200590FFE739
:10AE700009980E99086106980E994861002028B932
:10AE8000FFE7059801F02AFF70B90AE0059809F07C
:10AE900093F841EC100B51EC100B01F003FF18B9C3
:10AEA000FFE700200590FFE79DED080A0E98406837
:10AEB00090ED011A90ED032A20EE010A9DED051A8E
:10AEC00021EE021A30EE410A8DED040A0E9890ED43
:10AED000030A9DED081A9DED0A2A21EE021A30EEB2
:10AEE000010A8DED030A9DED030A0E98406890ED6E
:10AEF000021A20EE010A8DED020A0E98406890EDCC
:10AF0000020A9FED3F1AB4EE410AF1EE10FA39DD64
:10AF1000FFE7002028B9FFE7039801F0DFFE58B9EA
:10AF20002FE0039809F048F841EC100B51EC100B9E
:10AF300001F0B8FE28B3FFE79DED040A9DED021A6B
:10AF400030EE010AB0EEC00A0E98406890ED051A86
:10AF5000B4EE410AF1EE10FA12DCFFE79DED030AB0
:10AF6000B0EEC00A0E98406890ED041AB4EE410AA3
:10AF7000F1EE10FA04DCFFE703980E99C860FFE7D2
:10AF8000FFE7FFE79DED021A9DED040A30EE010A8E
:10AF90008DED040A002028B9FFE7049801F09EFE19
:10AFA00058B925E0049809F007F841EC100B51EC72
:10AFB000100B01F077FED8B1FFE70E98406890EDD6
:10AFC000050A9FED0F1AB4EE410AF1EE10FA0BDDFF
:10AFD000FFE79DED040A0E984068D0ED050AF6F7EC
:10AFE0008FFD8DED040AFFE704980E998861FFE755
:10AFF0000E9880690F90FFE79DED0F0A10B080BD9D
:10B00000BD37863580B586B004908DF80F108DED74
:10B01000020A0192049820B9FFE7FF208DF817007B
:10B02000B7E0002030B9FFE70198406801F056FE14
:10B0300080B90BE00198406808F0BEFF41EC100BAE
:10B0400051EC100B01F02EFE20B9FFE7FF208DF828
:10B0500017009EE0002030B9FFE70198806801F0FA
:10B060003DFE80B90BE00198806808F0A5FF41EC37
:10B07000100B51EC100B01F015FE20B9FFE7FF207B
:10B080008DF8170085E0002030B9FFE70198C0680F
:10B0900001F024FE80B90BE00198C06808F08CFF35
:10B0A00041EC100B51EC100B01F0FCFD20B9FFE757
:10B0B000FF208DF817006CE0002030B9FFE7019801
:10B0C000006901F00BFE80B90BE00198006908F0FF
:10B0D00073FF41EC100B51EC100B01F0E3FD20B9B4
:10B0E000FFE7FF208DF8170053E0002030B9FFE79D
:10B0F0000198406901F0F2FD80B90BE001984069C8
:10B1000008F05AFF41EC100B51EC100B01F0CAFD96
:10B1100020B9FFE7FF208DF817003AE00198049965
:10B1200048609DED021AB7EE000A80EE010A8DED2F
:10B13000000A002028B9FFE7009801F0CFFD58B9B8
:10B140000EE0009808F038FF41EC100B51EC100BAA
:10B1500001F0A8FD20B1FFE700980499886003E0A2
:10B16000FF208DF8170014E0049901F11C009DEDFB
:10B17000020A4968D1ED060AFEF778FC9DF80F0037
:10B1800004990870049800F009F800208DF8170061
:10B19000FFE79DF9170006B080BD000080B584B0C0
:10B1A0000290029820B9FFE7FF208DF80F0013E00E
:10B1B000029900200190C8600299086102994861D3
:10B1C0000299886102981C309FED050AFEF7ECFC9D
:10B1D00001988DF80F00FFE79DF90F0004B080BDC6
:10B1E000000000000000000000000000000000005F
:10B1F000EFF30980BFF36F8F154B1A681EF0100F25
:10B2000008BF20ED108A20E9F04F10602DE90900F9
:10B210004FF0500080F31188BFF34F8FBFF36F8F53
:10B2200004F00CFD4FF0000080F31188BDE8090028
:10B2300019680868B0E8F04F1EF0100F08BFB0ECB6
:10B24000108A80F30988BFF36F8F704700BF00BF7B
:10B25000540F002083B002900191ADF8022040F617
:10B260002850C2F200000268516941F0400151616A
:10B270000168C86840F01000C86040F69020C2F233
:10B2800000000168086820F001000860FFE740F650
:10B290009020C2F2000000680068C00750B1FFE7CC
:10B2A00040F69020C2F200000168086820F001001A
:10B2B0000860ECE740F69020C2F20000026844F615
:10B2C0000401C4F20001916002990268D160019901
:10B2D00002681161BDF802100268516002681168CD
:10B2E00041F4802111600168086840F001000860A5
:10B2F00003B0704780B582B001900198806B0090D8
:10B3000000980168486820F0030048600099486D83
:10B3100040F0100048650099012081F85100009824
:10B32000FBF798FF02B080BD80B582B00190019814
:10B33000806B00900098FCF71FFB02B080BD0000FE
:10B3400080B582B001900198806B00900098FDF765
:10B3500045F802B080BD000080B582B00190019830
:10B36000806B00900098FDF78DF802B080BD000062
:10B3700080B584B003900398806B0290FBF770F95E
:10B38000019003980068006800F48070B0F5807F39
:10B3900039D0FFE702980168486820F02000486033
:10B3A0000298806868B9FFE702984068B0F5827F2C
:10B3B00007D1FFE702980168486820F00300486061
:10B3C00006E002980168486820F001004860FFE745
:10B3D0000298019A642100F0B5F820B1FFE70299C4
:10B3E00020204865FFE702990020C88702990120C4
:10B3F00081F851000298406D20B1FFE70298FBF7F9
:10B4000029FF04E0FFE70298FCF78CFAFFE704B09D
:10B4100080BD000080B584B003900398806B0290DB
:10B42000FBF71EF9019003980068006800F4807033
:10B43000B0F5807F3BD0FFE702980168486820F0B4
:10B440002000486002980168486820F002004860C7
:10B450000298019A642100F0E7F830B1FFE7029901
:10B46000486D40F020004865FFE70298806870B999
:10B47000FFE7FFE70020009002980068C068009096
:10B4800002980068806800900098FFE7FFE7029943
:10B490000020C8860299012081F851000298406D71
:10B4A00020B1FFE70298FBF7D5FE04E0FFE7029822
:10B4B000FCF770FFFFE704B080BD000080B584B0EA
:10B4C00003900398806B0290FBF7CAF801900398F1
:10B4D0000068006800F48070B0F5807F2BD0FFE733
:10B4E00002980168486820F0200048600298019A9C
:10B4F000642100F099F830B1FFE70299486D40F0FF
:10B5000020004865FFE702980168486820F00300C2
:10B51000486002990020C8860299C88702990120D4
:10B5200081F851000298406D20B1FFE70298FBF7C7
:10B5300091FE04E0FFE70298FCF77AFFFFE704B012
:10B5400080BD000080B586B00490039102920498FB
:10B550004068B0F5827F13D1FFE704988068B0F5AA
:10B56000004F06D0FFE704988068B0F5806F07D1E0
:10B57000FFE704980168086820F040000860FFE7D2
:10B5800004984068B0F5827F31D1FFE70498806865
:10B59000B0F5806F15D0FFE70498039B02996A46C7
:10B5A00011608021002200F0BDF848B1FFE7049946
:10B5B000486D40F02000486503208DF817002FE00B
:10B5C00014E00498039B02996A461160012100224D
:10B5D00000F0A8F848B1FFE70499486D40F020005A
:10B5E000486503208DF817001AE0FFE714E004987F
:10B5F000039B02996A4611600121002200F092F833
:10B6000048B1FFE70499486D40F0200048650320E9
:10B610008DF8170004E0FFE700208DF81700FFE722
:10B620009DF8170006B080BD80B586B004900391E8
:10B6300002920498039B02996A461160022101223A
:10B6400000F070F848B1FFE70499486D40F0200021
:10B65000486503208DF8170048E040F20000C2F270
:10B66000000000684AF6AB21CAF6AA21A0FB01102F
:10B6700000094DF68361C4F21B31A0FB0110800C60
:10B680004FF47A714843019004984068B0F5827F86
:10B6900015D1FFE70498039B02996A461160802147
:10B6A000002200F03FF848B1FFE70499486D40F0F0
:10B6B0002000486503208DF8170017E012E0FFE72F
:10B6C000019808B9FFE70CE0019801380190FFE705
:10B6D000049800688068C1B20020B0EBD11FEFD1A0
:10B6E000FFE7FFE700208DF81700FFE79DF8170040
:10B6F00006B080BD82B000900098006843F200015F
:10B70000C4F20101884204D1FFE700208DF8070050
:10B7100003E002208DF80700FFE79DF8070002B064
:10B720007047000080B58AB0DDF830C008900791FE
:10B730008DF81B20059305980190FAF791FF0246BA
:10B7400001980C99891A08440390FAF789FF02902E
:10B75000039840F20001C2F200010968C1F3CB3145
:10B7600048430490FFE708980068806807990840FC
:10B77000401AB0FA80F040099DF81B1088425FD053
:10B78000FFE705980130002859D0FFE7FAF768FF76
:10B790000299401A0399884204D2FFE703980028CF
:10B7A00042D1FFE708980168486820F0E00048604F
:10B7B00008984068B0F5827F13D1FFE70898806849
:10B7C000B0F5004F06D0FFE708988068B0F5806FAD
:10B7D00007D1FFE708980168086820F0400008607A
:10B7E000FFE70898806AB0F5005F0FD1FFE7FFE739
:10B7F00008980168086820F40050086008980168FB
:10B80000086840F400500860FFE7FFE7089901204E
:10B8100081F85100FFE70899002081F85000FFE708
:10B8200003208DF827000FE0049818B9FFE70020E7
:10B83000039003E0049801380490FFE7FFE792E7E4
:10B8400000208DF82700FFE79DF827000AB080BD93
:10B85000074B19680868B0E8F04F80F30988BFF318
:10B860006F8F4FF0000080F31188704700BF00BF5A
:10B87000540F002080B56FF00400002101F0C0FAE1
:10B8800080BD000080B582B0019002F08BF902F01B
:10B890003FFA02B080BD000080B582B000900098F1
:10B8A0000138B0F1807F03D3FFE70120019019E058
:10B8B000009801384EF21401CEF2000108604FF0FA
:10B8C000FF300F2101F07AFA4EF21801CEF200019A
:10B8D000002008604EF21002CEF200020721116033
:10B8E0000190FFE7019802B080BD000080B5FAF733
:10B8F000BDFE05F097FB012803D0FFE704F0AEFA88
:10B90000FFE780BD80B594B008A83021F4F771FD41
:10B91000002007900690059004900390FFE7002018
:10B92000029043F64000C4F20200016841F08051E9
:10B930000160006800F0805002900298FFE7FFE786
:10B940000020019047F20000C4F20000016841F4B9
:10B9500080410160006800F4804001900198FFE799
:10B96000012008904FF48030099002200E904FF48F
:10B9700080010F9106211091A821119112900420AD
:10B98000139008A8FBF706F918B1FFE7F8F786FF50
:10B99000FFE70F20039002200490002005904FF451
:10B9A000A05006904FF48050079003A80521FAF7A5
:10B9B00021FF18B1FFE7F8F771FFFFE714B080BD72
:10B9C0004EF68851CEF20001086840F4700008601D
:10B9D0007047000080B540F69840C2F20000FCF7C6
:10B9E00093FF80BD83B0029001910298006800909F
:10B9F00002980021C4F20101884225D0FFE7029895
:10BA0000B0F1804F20D0FFE7029840F20041C4F22D
:10BA10000001884218D0FFE7029840F60001C4F206
:10BA20000001884210D0FFE7029840F60041C4F2BE
:10BA30000001884208D0FFE7029840F20041C4F2BA
:10BA4000010188420AD1FFE7009820F070000090C1
:10BA500001984168009808430090FFE70298002190
:10BA6000C4F20101884255D0FFE70298B0F1804F3F
:10BA700050D0FFE7029840F20041C4F20001884232
:10BA800048D0FFE7029840F60001C4F20001884266
:10BA900040D0FFE7029840F60041C4F2000188421E
:10BAA00038D0FFE7029840F20041C4F20101884219
:10BAB00030D0FFE7029844F20001C4F2010188424D
:10BAC00028D0FFE7029844F20041C4F20101884205
:10BAD00020D0FFE7029844F60001C4F20101884239
:10BAE00018D0FFE7029841F60001C4F20001884235
:10BAF00010D0FFE7029841F60041C4F200018842ED
:10BB000008D0FFE7029842F20001C4F20001884227
:10BB10000AD1FFE7009820F4407000900198C168B6
:10BB2000009808430090FFE7009820F080000199FA
:10BB3000496908430090019880680299C862019899
:10BB400000680299886202980021C4F201018842CB
:10BB500008D0FFE7029840F20041C4F20101884298
:10BB600005D1FFE70198006902990863FFE7029990
:10BB7000086840F0040008600299012048610098BC
:10BB80000299086003B0704784B00390029101925B
:10BB9000029800F01F01012088400090009A03994C
:10BBA000086A904308620198029901F01F0100FAA7
:10BBB00001F20399086A1043086204B0704700005C
:10BBC00085B00490039102920193049880680090DC
:10BBD000009820F47F40009003980299019A41EA6E
:10BBE000022101430098084300900098049988605E
:10BBF00005B0704783B00290019102988068009070
:10BC0000009820F07000009001980099084340F0DF
:10BC10000700009000980299886003B07047000008
:10BC200085B0049003910498006A01900499086A11
:10BC300020F0010008620498406800900498806930
:10BC40000290029820F070000290029820F0030009
:10BC5000029003980168029808430290019820F02E
:10BC600002000190039881680198084301900498AC
:10BC70000021C4F20101884208D0FFE7049840F295
:10BC80000041C4F2010188420ED1FFE7019820F083
:10BC9000080001900398C168019808430190019839
:10BCA00020F004000190FFE704980021C4F2010194
:10BCB000884208D0FFE7049840F20041C4F2010135
:10BCC000884213D1FFE7009820F48070009000981C
:10BCD00020F4007000900398416900980843009098
:10BCE00003988169009808430090FFE70098049941
:10BCF00048600298049988610398406804994863F1
:10BD000001980499086205B07047000085B004905E
:10BD100003910498006A01900499086A20F01000C9
:10BD20000862049840680090049880690290029824
:10BD300020F4E0400290029820F4407002900398B2
:10BD40000168029840EA01200290019820F020004A
:10BD5000019003988168019840EA011001900498CD
:10BD60000021C4F20101884208D0FFE7049840F2A4
:10BD70000041C4F2010188420FD1FFE7019820F091
:10BD8000800001900398C168019840EA0110019079
:10BD9000019820F040000190FFE704980021C4F2D0
:10BDA0000101884208D0FFE7049840F20041C4F244
:10BDB0000101884215D1FFE7009820F480600090CF
:10BDC000009820F40060009003984169009840EAD0
:10BDD0008100009003988169009840EA81000090FA
:10BDE000FFE70098049948600298049988610398D5
:10BDF00040680499886301980499086205B0704707
:10BE000085B0049003910498006A01900499086A2F
:10BE100020F4807008620498406800900498C0691B
:10BE20000290029820F070000290029820F0030027
:10BE3000029003980168029808430290019820F448
:10BE40000070019003988168019840EA01200190F8
:10BE500004980021C4F20101884208D0FFE7049849
:10BE600040F20041C4F2010188420FD1FFE701987E
:10BE700020F4006001900398C168019840EA012015
:10BE80000190019820F480600190FFE70498002160
:10BE9000C4F20101884208D0FFE7049840F2004153
:10BEA000C4F20101884215D1FFE7009820F48050C8
:10BEB0000090009820F40050009003984169009889
:10BEC00040EA0110009003988169009840EA01104F
:10BED0000090FFE700980499486002980499C861AF
:10BEE000039840680499C86301980499086205B0F2
:10BEF0007047000085B0049003910498006A019097
:10BF00000499086A20F48050086204984068009000
:10BF10000498C0690290029820F4E04002900298D0
:10BF200020F44070029003980168029840EA0120D2
:10BF30000290019820F400500190039881680198C4
:10BF400040EA0130019004980021C4F201018842C6
:10BF500008D0FFE7049840F20041C4F20101884292
:10BF60000BD1FFE7009820F48040009003984169CE
:10BF7000009840EA81100090FFE70098049948601B
:10BF800002980499C861039840680499086401986C
:10BF90000499086205B0704785B00490039102923D
:10BFA0000498006A00900499086A20F00100086271
:10BFB000049880690190019820F0F00001900299A6
:10BFC000019840EA01100190009820F00A000090CA
:10BFD000039900980843009001980499886100989B
:10BFE0000499086205B0704785B0049003910292ED
:10BFF0000498006A00900499086A20F01000086212
:10C00000049880690190019820F470400190029991
:10C01000019840EA01300190009820F0A0000090C3
:10C020000399009840EA01100090019804998861F2
:10C0300000980499086205B07047000080B586B08A
:10C04000059001F0BBF94CF23910C0F6000044F243
:10C05000D032C0F601020021029101F0ABFD02993D
:10C0600041F22C42C2F20002049210604CF2B12064
:10C07000C0F6000044F2F432C0F6010201F09AFD6D
:10C080000299049A50604CF28940C0F6000044F2D4
:10C090001842C0F6010201F08DFD0299049A9060E9
:10C0A0004CF20960C0F6000044F23C42C0F60102C6
:10C0B00001F080FD0299049AD0604CF26160C0F6F4
:10C0C000000044F26042C0F6010201F073FD029AE2
:10C0D00004990861022003900A2101F05DFA029A96
:10C0E000049B014603985961242101F055FA029AF4
:10C0F000049B0146039899610C21019101F04CFACF
:10C100000199029ADDF810C003460398CCF8283054
:10C1100001F042FA029A049B0146039859621821E1
:10C1200001F03AFA0499C86101F09EF901F03AFD74
:10C1300001F0EEFD06B080BD80B58CB00B9001F033
:10C1400015F907F041FB41EC100B9FED531B53EC2D
:10C15000112B51EC100B07F02DF941EC100B51ECA9
:10C16000100B07F0EDFA0A900020089001F07AF821
:10C1700001F0E8F8099041F22C40C2F2000000F111
:10C18000580140F2A820C2F200000790F5F738FDF0
:10C190000798F5F70DFD40F28020C2F2000040F64E
:10C1A0000861C2F20001F4F777FA089940F6C85026
:10C1B000C2F2000040F2D802C2F200029FED380A3B
:10C1C000FEF720FF0120F6F7EFFDFFE70A99099837
:10C1D00008440990F5F704FFF5F7D2FCF5F7E0FC09
:10C1E000F5F7F8FCF5F704FD01F0E8F840F2A820B7
:10C1F000C2F200000690F5F7C7FD0698F5F73EFE7F
:10C20000069800F1100100F11C02029240F2802019
:10C21000C2F20000019040F60863C2F20003F4F796
:10C220007DFB019940F6BC50C2F200000390F4F788
:10C2300085F941F22C40C2F200000590406A01F0FD
:10C240008DFA02990598406A002304931A4601F07A
:10C2500023FA0598806A01F081FA0399049B0598F6
:10C26000806A1A4601F018FA01F0FEF80698D0ED3F
:10C270000A0A40F6C850C2F200009FED0A0ADFED3C
:10C280000A1AB0EE611AFEF745FD0120F6F7ECFC44
:10C29000099801F001F899E70000000000407F4094
:10C2A0000000FA43000020420000000000000000EF
:10C2B000B0B588B0079001F059F807F085FA41EC65
:10C2C000100B9FED6F1B53EC112B51EC100B07F073
:10C2D00071F841EC100B51EC100B07F031FA06909D
:10C2E000002000F0BFFF01F02DF8059002F0F8FDEE
:10C2F000FFE7069905980844059041F2F830C2F22C
:10C300000000007838B1FFE741F2F831C2F20001D5
:10C3100000200870FFE741F2D433C2F20003039318
:10C3200018685A68D3F808C0D3F80CE01C695D6936
:10C3300040F61861C2F2000104914D610C61C1F830
:10C340000CE0C1F808C04A6008609869DA691B6AA5
:10C350000B62CA61886141F22C40C2F20000806920
:10C3600000231A4601F098F908B9FFE7FFE740F605
:10C370001860C2F20000B0F9100001460291B0F559
:10C38000B07F0BD0FFE70298B0F5806F0FD0FFE7CA
:10C39000029840F29F61884212D01AE040F60411E0
:10C3A000C2F2000100200871012008601AE040F686
:10C3B0000411C2F20001012008710220086011E09E
:10C3C00040F60411C2F20001022008710320086047
:10C3D00008E040F60411C2F20001042008600020C9
:10C3E0000871FFE740F61860C2F20000B0F91200D1
:10C3F00001460191B0F5B07F0BD0FFE70198B0F591
:10C40000806F0ED0FFE7019840F29F61884210D004
:10C4100018E040F60411C2F200014FF07E5048616E
:10C4200010E040F60411C2F200014FF07F50486165
:10C4300008E040F60411C2F200010020C4F2A0009E
:10C440004861FFE740F61860C2F20000C26840F69B
:10C450000411C2F200018A608268CA600068086143
:10C4600041F22C40C2F20000C06900231A4601F0DC
:10C4700013F908B9FFE7FFE7059800F00DFF38E76B
:10C480000000000000407F4080B58AB0099000F0B5
:10C490006DFF07F099F941EC100B9FED571B53EC22
:10C4A000112B51EC100B06F085FF41EC100B51ECF9
:10C4B000100B07F045F90890002000F0D3FE00F0C3
:10C4C00041FF0790F8F7D4F8014640F21030C2F26D
:10C4D00000009FED4B0A00F0D3FCFFE70899079896
:10C4E0000844079041F22C40C2F20000806A40F2FA
:10C4F0001031C2F2000101F20C4100231A4600F093
:10C50000EBFF38B9FFE740F60011C2F2000101204D
:10C510000860FFE741F22C40C2F20000406A40F29E
:10C520001031C2F2000101F57D7100231A4600F0BE
:10C53000D3FF38B9FFE740F60011C2F20001022034
:10C540000860FFE741F22C40C2F20000806940F62B
:10C550003C61C2F2000100231A4600F0BDFF38B969
:10C56000FFE740F60011C2F2000103200860FFE778
:10C5700041F22C40C2F20000C06940F2F021C2F248
:10C58000000100231A4600F0A7FFA8B9FFE740F614
:10C590000011C2F200010520086040F21030C2F222
:10C5A00000000090F7F768FF009840F2F021C2F217
:10C5B0000001F6F7F3FD14E040F60011C2F20001AD
:10C5C00006200860002006900590049003900290D9
:10C5D000019040F21030C2F2000001A9F6F7DEFD32
:10C5E000FFE740F21030C2F20000F6F745FF07986F
:10C5F00000F052FE72E700BF0000000000407F40E4
:10C600000000FA430000000080B584B0039000F001
:10C61000ADFE07F0D9F841EC100B9FED0F1B53EC6A
:10C62000112B51EC100B06F0C5FE41EC100B51EC38
:10C63000100B07F085F80290002000F013FE00F0C8
:10C6400081FE0190FFE7029901980844019001984A
:10C6500000F022FEF7E700BF0000000000407F402E
:10C6600080B584B0039000F081FE07F0ADF841EC96
:10C67000100B9FED0F1B53EC112B51EC100B06F020
:10C6800099FE41EC100B51EC100B07F059F8029099
:10C69000002000F0E7FD00F055FE0190FFE7029951
:10C6A000019808440190019800F0F6FDF7E700BFFB
:10C6B0000000000000407F4080B582B001900198EA
:10C6C000806B009000990020C8850098FCF77CFCE6
:10C6D00002B080BD84B00390FFE7FFE703980068D5
:10C6E00050E8030F20F490700290FFE7029903983E
:10C6F000026842E803100028F0D1FFE7FFE7FFE7F8
:10C70000FFE70398006850E8050F20F00100019052
:10C71000FFE701990398026842E805100028F0D16C
:10C72000FFE7FFE70398006B012814D1FFE7FFE75D
:10C73000FFE70398006850E8030F20F01000009016
:10C74000FFE700990398026842E803100028F0D13F
:10C75000FFE7FFE7FFE70399202081F842000399F4
:10C760000020086304B0704780B582B00190019842
:10C770000168C86820F04000C8600199202081F855
:10C7800041000198FDF7AEF8002002B080BD000026
:10C7900082B000900098006844F60001C4F20001E5
:10C7A000884204D1FFE700208DF8070010E00098D0
:10C7B000006841F20041C4F20101884204D1FFE760
:10C7C00001208DF8070003E003208DF80700FFE744
:10C7D0009DF8070002B0704780B586B00490002035
:10C7E00003900290049890F84200222840F0A08024
:10C7F000FFE704988068B0F5805F13D1FFE70498E5
:10C80000006978B9FFE70498806A0290049800688C
:10C8100040686FF35F20029908800499886A0230AB
:10C82000886223E00498806A039004988068B0F5D9
:10C83000805F08D0FFE70498806850B9FFE704984C
:10C84000006930B9FFE704980068406803990870F0
:10C8500007E004980068406800F07F0003990870C2
:10C86000FFE70499886A01308862FFE70499C88D60
:10C870000138C8850004002856D1FFE704980168F4
:10C88000C86820F02000C86004980168C86820F4D7
:10C890008070C86004980168486920F00100486110
:10C8A0000499202081F842000499002048630498EC
:10C8B000006B012830D1FFE7049900200863FFE7EF
:10C8C000FFE70498006850E8030F20F01000019083
:10C8D000FFE701990498026842E803100028F0D1AC
:10C8E000FFE7FFE7049800680068C00600280ED53F
:10C8F000FFE7FFE7002000900498006800680090C0
:10C9000004980068406800900098FFE7FFE70498EB
:10C91000818DFCF753FB03E00498FCF7B9FFFFE7B8
:10C9200000208DF8170007E000208DF8170003E0C5
:10C9300002208DF81700FFE79DF8170006B080BDB4
:10C9400080B586B0059005980068006920F44050D5
:10C95000059A1168D26810430861059988680B69C7
:10C960004A69C96918431043084304900598006850
:10C97000C06849F20C618843049908430599096825
:10C98000C86005980068406920F44070059A1168F5
:10C990009269104348610598006841F20001C4F2B1
:10C9A0000101884209D0FFE70598006841F2004183
:10C9B000C4F20101884204D1FFE7FAF765F8039059
:10C9C00003E0FAF74FF80390FFE70598C069B0F568
:10C9D000004F29D1FFE703981921A0FB0101059A17
:10C9E0001368029353685A00DB0FF3F73DFC02997A
:10C9F000864648F21F53C5F2EB13AEFB03204209F3
:10CA000010014FF0640C02FB1CEC322202EBCC0252
:10CA1000A2FB0332F82303EA521300EB4300C2F3F4
:10CA200042121044886026E003981921A0FB0101FE
:10CA3000059A1368019353689A009B0FF3F714FC4F
:10CA40000199844648F21F52C5F2EB12ACFB02304A
:10CA50004309642003FB10CC322000EB0C10A0FB38
:10CA60000202F02000EA521000EB0310C2F343125E
:10CA700010448860FFE706B080BD000083B00190DD
:10CA8000019890F8410021283AD1FFE70198806889
:10CA9000B0F5805F13D1FFE70198006978B9FFE72F
:10CAA0000198006A0090009800886FF35F20019958
:10CAB000096848600199086A0230086208E0019A32
:10CAC000106A411C11620078019909684860FFE70B
:10CAD0000199C88C0138C884000468B9FFE701983F
:10CAE0000168C86820F08000C86001980168C868C3
:10CAF00040F04000C860FFE700208DF80B0003E025
:10CB000002208DF80B00FFE79DF80B0003B0704783
:10CB100080B540F6E040C2F20000FCF77FFA80BD2D
:10CB200080B582B040F62850C2F20000006800686C
:10CB30008006002801D5FFE792E044F60000C4F229
:10CB400000000068C006002840F18980FFE7FFE789
:10CB50000020019040F62850C2F2000001680968E8
:10CB600001910068406801900198FFE740F690202D
:10CB7000C2F20000006800680003002835D4FFE717
:10CB800040F69021C2F200010A68106820F001000E
:10CB9000106008684068C0F1320241F2CC40C2F235
:10CBA000000002800B6832225A600B681A6842F457
:10CBB00000221A600A68116841F0010111600088C2
:10CBC000192811D1FFE741F2F930C2F2000041F219
:10CBD000D431C2F2000102F08FF941F2F831C2F211
:10CBE000000101200870FFE738E040F69021C2F212
:10CBF00000010A68106820F00100106008684068B1
:10CC0000C0F1320241F2CC40C2F2000002800B6857
:10CC100032225A6046F22803C4F202031A6822F450
:10CC200000221A600A68116841F001011160008851
:10CC3000192812D1FFE741F2F930C2F20000193091
:10CC400041F2D431C2F2000102F056F941F2F8315A
:10CC5000C2F2000101200870FFE7FFE7FFE7FFE7EE
:10CC600002B080BD80B582B040F67050C2F20000C4
:10CC70000190FCF7D3F90198F6F70CFA02B080BDE9
:10CC8000FFE7FEE782B041EC100B8DED000B019841
:10CC9000C0F30A5040F2FF71401A18BF012002B0E1
:10CCA0007047000082B041EC100B8DED000B019835
:10CCB000C0F30A5040F2FF71401A18BF012002B0C1
:10CCC0007047000081B000EE100A00900098C0F399
:10CCD000C750FF3818BF012001B0704781B000EE87
:10CCE000100A00900098C0F3C750FF3818BF012009
:10CCF00001B0704784B041EC100B8DED020B039A2C
:10CD000000200021CFF6E071B1EB420F019006D177
:10CD1000FFE70298B0FA80F040090190FFE7019820
:10CD200000F0010004B0704781B000EE100A0090DE
:10CD300000994FF0807000EB4100B0FA80F040099C
:10CD400001B0704781B08DF803009DF90300002801
:10CD500012D4FFE79DF9031001F01F02012090405B
:10CD60004A094EF28011CEF2000141F82200BFF3D1
:10CD70004F8FBFF36F8FFFE701B0704781B08DF821
:10CD800003009DF9030000280ED4FFE79DF903106E
:10CD900001F01F02012090404A094EF20011CEF22C
:10CDA000000141F82200FFE701B070474EF60C5039
:10CDB000CEF200000068C0F30220704782B08DF808
:10CDC000070000919DF9070000280AD4FFE70098AA
:10CDD00000019DF907104EF20042CEF20002885485
:10CDE0000BE0009800019DF8071001F00F014EF6CE
:10CDF0001452CEF200028854FFE702B070470000E0
:10CE000082B08DF8070000919DF9070000280AD430
:10CE1000FFE7009800019DF907104EF20042CEF2A4
:10CE2000000288540BE0009800019DF8071001F003
:10CE30000F014EF61452CEF200028854FFE702B002
:10CE40007047000083B00290029800F00700009045
:10CE50004EF60C51CEF200010868019001984FF691
:10CE6000FF02104001900198009A40EA022000223F
:10CE7000C0F2FA52104301900198086003B0704765
:10CE800080B590B00E900D918DED0C0A0E9858B1B2
:10CE9000FFE70D9840B1FFE79DED0C0AB5EE400AA3
:10CEA000F1EE10FA04DCFFE7FF208DF83F00FFE011
:10CEB0000D980E99C1F828040E990020039008736C
:10CEC000F5F7D0FA03980B90FFE70B9803280EDCD8
:10CED000FFE70E98D0F828040B9900EBC1006030F2
:10CEE000FDF7C0F8FFE70B9801300B90EDE700204D
:10CEF0000A90FFE70A9803280EDCFFE70E98D0F8A7
:10CF000028040A9900EBC1008030FDF7ABF8FFE779
:10CF10000A9801300A90EDE744F2A843C0F60103F5
:10CF2000186859689A68DB68099308920791069017
:10CF30000E990698079A089BDDF824C0C1F824C40E
:10CF4000C1F82034C1F81C24C1F818040020059051
:10CF5000FFE70598032816DCFFE70E990598C0EB5C
:10CF6000001001EB800000F538709DED0C0AD1F83F
:10CF7000281401F140020021FEF744F8FFE705986C
:10CF800001300590E5E700200490FFE704980328AE
:10CF900025DCFFE70E990498C0EB001001EB800040
:10CFA00000F5F8709DED0C0AD1F8282400210291BB
:10CFB000FEF728F802990E9A0498C0EB001002EBD5
:10CFC000800000F580709DED0C0AD2F828242032F4
:10CFD000FEF718F8FFE7049801300490D6E70E98A2
:10CFE00000F24C409DED0C0AF3EE040ACDED010A6F
:10CFF000FCF73CFDDDED010A0E9800F26C409DED62
:10D000000C0AFCF733FDDDED010A0E9800F28C40AE
:10D010009DED0C0AFCF72AFDDDED010A0E9800F2E9
:10D02000AC409DED0C0AFCF721FDDDED010A0E98E8
:10D0300000F2CC409DED0C0AFCF718FDDDED010A75
:10D040000E9800F2EC409DED0C0AFCF70FFDDDEDB3
:10D05000010A0E9800F20C509DED0C0AFCF706FD3B
:10D06000DDED010A0E9800F22C509DED0C0AFCF744
:10D07000FDFCDDED010A0E9800F24C509DED0C0A0E
:10D08000FCF7F4FCDDED010A0E9800F26C509DED0A
:10D090000C0AFCF7EBFCDDED010A0E9800F28C5057
:10D0A0009DED0C0AFCF7E2FC00208DF83F00FFE745
:10D0B0009DF93F0010B080BD82B08DED010ACDED2D
:10D0C000000A01980099C90F61F3DF7001909DED8E
:10D0D000010A02B07047000080B588B0069006983B
:10D0E0000190019858B9FFE74FF0500080F3118884
:10D0F000BFF36F8FBFF34F8F0790FFE7FEE70198F5
:10D1000040F65471C2F200010968884204D1FFE779
:10D1100000208DF8170056E002F054F9019840699C
:10D12000049040F65C70C2F200000068039040F684
:10D130006470C2F200000068029002F06FF9049877
:10D140000399884205D0FFE704980299884204D1E8
:10D15000FFE702208DF8170034E0049845F68001BF
:10D16000C2F20001884218D1FFE70198806A78B9BD
:10D17000FFE7019890F85800012804D1FFE702204A
:10D180008DF8170003E003208DF81700FFE703E098
:10D1900002208DF81700FFE713E0049845F694018C
:10D1A000C2F20001884203D0FFE7049820B9FFE7EC
:10D1B00004208DF8170003E001208DF81700FFE729
:10D1C000FFE7FFE7FFE79DF8170008B080BD00000C
:10D1D00080B582B000200190F9F756FAFEF792FB75
:10D1E000FDF7EEF9FDF76EF9FDF71CF9FDF742F9D1
:10D1F000FDF704FCFDF726FCFDF7D6FAFDF7DEFB94
:10D20000FDF742FBFDF7ACFBFDF7F6FA00F0B2F8D4
:10D21000FDF7B6F900F0FEF8FFE7FEE785B08DED0B
:10D22000040ACDED030A8DED021ACDED011A8DED44
:10D23000002A9DED040A9DED033A30EE430A9DED70
:10D24000002A9DED011A32EE412A20EE020A9DEDE0
:10D25000022A32EE432A80EE020A30EE010A05B0BD
:10D260007047000080B584B00290EFF30580039012
:10D27000039820B1FFE76FF00500019009E000205E
:10D280000190029820B1FFE7029802F015FAFFE73B
:10D29000FFE7019804B080BD80B586B00490EFF33D
:10D2A00005800590059820B1FFE76FF0050001901B
:10D2B0001BE00020019003F0D1FE03900498039935
:10D2C000401A0290029858B1FFE702990020B0EB93
:10D2D000D17F05D1FFE7029903A802F025FA03E008
:10D2E0006FF003000190FFE7FFE7019806B080BDF3
:10D2F00080B582B003F096FE0146009158B1FFE779
:10D30000009801280AD0FFE70098022807D1FFE71C
:10D310000220019012E0032001900FE0FFE740F2AD
:10D320001420C2F200000068012803D1FFE70120A9
:10D33000019002E000200190FFE7FFE7019802B0B2
:10D3400080BD000080B582B0EFF3058001900198A8
:10D3500020B1FFE703F08CFE009003E003F07EFEB7
:10D360000090FFE7009802B080BD00004FF47A7093
:10D370007047000082B0EFF305800190019820B162
:10D38000FFE76FF00500009014E040F21420C2F2B5
:10D390000000006848B9FFE740F21421C2F2000122
:10D3A000012008600020009003E04FF0FF30009063
:10D3B000FFE7FFE7009802B07047000080B584B037
:10D3C000EFF305800390039820B1FFE76FF00500AD
:10D3D00002901BE003F026FE0146019140B1FFE7F9
:10D3E000019801280CD0FFE70198022803D008E03B
:10D3F0000120029009E002F019FC0020029004E0F4
:10D40000FFE74FF0FF300290FFE7FFE7029804B01C
:10D4100080BD000080B582B0EFF3058001900198D7
:10D4200020B1FFE76FF00500009019E040F21420F2
:10D43000C2F20000006801280DD1FFE7FEF71AFADA
:10D4400040F21421C2F200010220086002F07EFBCB
:10D450000020009003E04FF0FF300090FFE7FFE76F
:10D46000009802B080BD000080B584B0EFF3058065
:10D470000390039820B1FFE76FF00500029027E0CA
:10D4800003F0D0FD0146019140B1FFE7019801286A
:10D4900018D0FFE70198022811D014E00120029073
:10D4A00004F0AAF8012809D0FFE703F0BBFD20B97A
:10D4B000FFE74FF0FF300290FFE7FFE707E00020B3
:10D4C000029004E0FFE74FF0FF300290FFE7FFE734
:10D4D000029804B080BD000080B588B00690059128
:10D4E000049203930698029000200190EFF30580C8
:10D4F0000790079868B3FFE7029830B1FFE70598F7
:10D5000018B1FFE7039820B1FFE76FF00300019027
:10D510001EE000200090029805996A4603F0EAF8A0
:10D52000012804D0FFE76FF0020001900FE000989F
:10D5300060B1FFE74EF60451CEF200014FF080508B
:10D540000860BFF34F8FBFF36F8FFFE7FFE7FFE781
:10D550001FE0029818B1FFE7059820B9FFE76FF0C8
:10D560000300019014E002980599039A02F0D4FF99
:10D5700001280CD0FFE7039820B1FFE76FF001000E
:10D58000019003E06FF002000190FFE7FFE7FFE783
:10D59000FFE7019808B080BD80B588B0069005917E
:10D5A000049200200390EFF305800790079800286D
:10D5B0006ED1FFE7069800286AD0FFE7059800289B
:10D5C00066D0FFE74FF0FF300290049868B3FFE7A2
:10D5D00004988068A0B1FFE70498C06850280FD372
:10D5E000FFE70498006958B1FFE70498406906997D
:10D5F000059A5143884203D3FFE70120029013E0CC
:10D600000498806878B9FFE70498C06858B9FFE7C4
:10D610000498006938B9FFE70498406918B9FFE732
:10D6200000200290FFE7FFE702E000200290FFE702
:10D63000029801280ED1FFE706980599049A93688D
:10D640001269EE464FF0000CCEF800C002F08CFCE0
:10D6500003900AE0029838B9FFE70698059900227E
:10D6600002F048FC0390FFE7FFE7039878B1FFE77B
:10D67000049820B1FFE704980068019002E00020C0
:10D680000190FFE70398019901F0BAFFFFE7FFE778
:10D69000039808B080BD000080B588B00690059161
:10D6A0008DF8132003930698029000200190EFF369
:10D6B00005800790079868B3FFE7029830B1FFE74D
:10D6C000059818B1FFE7039820B1FFE76FF003005A
:10D6D00001901EE000230093029805996A4602F02B
:10D6E0003FFE012804D0FFE76FF0020001900FE039
:10D6F000009860B1FFE74EF60451CEF200014FF002
:10D7000080500860BFF34F8FBFF36F8FFFE7FFE7D5
:10D71000FFE720E0029818B1FFE7059820B9FFE77E
:10D720006FF00300019015E002980599039A002319
:10D7300002F000FD01280CD0FFE7039820B1FFE7BD
:10D740006FF00100019003E06FF002000190FFE72D
:10D75000FFE7FFE7FFE7019808B080BD80B584B020
:10D76000029002980190EFF305800390039820B196
:10D77000FFE76FF0050000900DE0019820B9FFE78A
:10D780006FF00300009005E000210091019802F085
:10D7900073FCFFE7FFE7009804B080BD80B586B05A
:10D7A00004900391049820F001000290049800F086
:10D7B0000100009000200190EFF30580059005988E
:10D7C00020B1FFE76FF00500019033E0029820B927
:10D7D000FFE76FF0030001902BE00098A0B1FFE796
:10D7E0000298039903F020F901280CD0FFE7039871
:10D7F00020B1FFE76FF00100019003E06FF002003D
:10D800000190FFE7FFE713E00298039902F0F6FFAB
:10D8100001280CD0FFE7039820B1FFE76FF001006B
:10D82000019003E06FF002000190FFE7FFE7FFE7E0
:10D83000FFE7FFE7019806B080BD000080B588B023
:10D84000069000200590EFF30580079007980028C8
:10D8500040F08580FFE7069820B1FFE70698406812
:10D86000049002E000200490FFE79DF81000C0073C
:10D8700018B1FFE70120039002E000200390FFE7CA
:10D88000049800F00800082868D0FFE74FF0FF3048
:10D8900002900698C8B1FFE70698806840B1FFE79C
:10D8A0000698C068502803D3FFE7012002900BE0E0
:10D8B0000698806838B9FFE70698C06818B9FFE78E
:10D8C00000200290FFE7FFE702E000200290FFE760
:10D8D0000298012812D1FFE7039838B1FFE70698B4
:10D8E0008168042002F0ECFA059006E00698816851
:10D8F000012002F0E5FA0590FFE711E0029870B907
:10D90000FFE7039828B1FFE7042002F0C5FA05906D
:10D9100004E0012002F0C0FA0590FFE7FFE7FFE70F
:10D92000059878B1FFE7069820B1FFE706980068F0
:10D93000019002E000200190FFE70598019901F0B5
:10D940005FFEFFE7059840B1FFE7039828B1FFE7C6
:10D95000059840F001000590FFE7FFE7FFE7059815
:10D9600008B080BD80B586B00490049820F0010016
:10D970000390049800F00100019000200290EFF362
:10D9800005800590059820B1FFE76FF00500029033
:10D9900024E0039820B9FFE76FF0030002901CE039
:10D9A000019858B1FFE7039802F080FD012804D0E8
:10D9B000FFE76FF002000290FFE70DE003980023FD
:10D9C00019461A4602F0B6FB012804D0FFE76FF0B3
:10D9D00002000290FFE7FFE7FFE7FFE7029806B0CB
:10D9E00080BD000080B58AB0089007910898069025
:10D9F000069830B1FFE79DF81F000006002804D507
:10DA0000FFE76FF0030005903BE04FF0FF3005901B
:10DA1000EFF305800990099820B3FFE700230393F3
:10DA2000049306980799EC4604AACCF8002001223A
:10DA300003F00CFA039A069869460A6005AB114692
:10DA400003F004FA049860B1FFE74EF60451CEF2F9
:10DA500000014FF080500860BFF34F8FBFF36F8F0E
:10DA6000FFE70DE00698079901220023029303F0D7
:10DA700031F9029A069805AB114603F02BF9FFE73E
:10DA8000FFE705980AB080BD80B58CB00A90099177
:10DA90000892EFF305800B900B9820B1FFE76FF031
:10DAA000050007907AE09DF82B000006002804D5B9
:10DAB000FFE76FF0030007906FE09DF824008007F8
:10DAC000002803D5FFE70020059002E00A980590A2
:10DAD000FFE7002007900898029003F0BFFA049037
:10DAE000FFE70599029B002006AA03F0B3FB019013
:10DAF000019801283FD1FFE70A990798084007904D
:10DB000006990798084307909DF82400C00780B144
:10DB1000FFE70A9907980840884201D1FFE73BE0F8
:10DB2000089820B9FFE76FF00200079034E0FFE7A4
:10DB30000EE00A980799084201D0FFE72CE0089808
:10DB400020B9FFE76FF00200079025E0FFE7FFE74D
:10DB500003F084FA0499401A0390039802998842CA
:10DB600003D9FFE70020029004E003990298401ACD
:10DB70000290FFE70BE0089820B9FFE76FF0020082
:10DB8000079003E06FF001000790FFE7FFE7FFE772
:10DB900001980028A5D1FFE7FFE7FFE707980CB041
:10DBA00080BD000080B582B003F032FA0190019888
:10DBB00002B080BDB0B58EB00B900A9109920020E2
:10DBC0000690EFF305800D900D98002840F09980A5
:10DBD000FFE70B98002800F09480FFE78020079073
:10DBE00018200590002008904FF0FF30049009980D
:10DBF00000284DD0FFE70998006820B1FFE7099899
:10DC000000680890FFE70998806920B1FFE709984C
:10DC100080690590FFE7059848B1FFE70598382827
:10DC200005D8FFE709980079C00718B1FFE7002081
:10DC30000C9069E00998406928B1FFE709984069AC
:10DC400080080790FFE70998806880B1FFE709988E
:10DC5000C0685C280BD3FFE70998006938B1FFE77B
:10DC60000998406918B1FFE7012004900FE0099876
:10DC7000806858B9FFE70998C06838B9FFE7099884
:10DC8000006918B9FFE700200490FFE7FFE702E012
:10DC900000200490FFE70498012817D1FFE70B98B4
:10DCA0000899079A0A9BDDF814C0DDF824E0DEF835
:10DCB0000850DEF81040EE46CEF80850CEF804408A
:10DCC000CEF800C002F09EFF069019E00498B0B9AB
:10DCD000FFE70B980899BDF81C200A9BDDF814C0DB
:10DCE000EE4606ACCEF80440CEF800C002F03AFF93
:10DCF000012803D0FFE700200690FFE7FFE7FFE7DA
:10DD0000FFE706980C90FFE70C980EB0B0BD00003E
:10DD100080B586B0049004980390EFF305800590D9
:10DD2000059820B1FFE76FF0050002901CE0039812
:10DD300020B9FFE76FF00300029014E00398FFF7AB
:10DD4000CBF98DF807009DF80700042806D0FFE7FF
:10DD500000200290039801F071FD03E06FF00200D3
:10DD60000290FFE7FFE7FFE7029806B080BD0000E2
:10DD700080B584B00390029145F6A800C2F200007D
:10DD80000068009040F65470C2F200000068043051
:10DD900001F04AFA08B9FFE700E0FFE70398013015
:10DDA00080B9FFE7029868B1FFE740F65470C2F20D
:10DDB00000000068011D45F68000C2F2000001F07D
:10DDC000D9FA3DE00098039908440190019840F683
:10DDD0005471C2F2000109684860019800998842B4
:10DDE0000ED2FFE740F66470C2F20000006840F611
:10DDF0005471C2F200010968043101F085FA1EE095
:10DE000040F65C70C2F20000006840F65471C2F245
:10DE100000010968043101F077FA019845F60C0118
:10DE2000C2F200010968884207D2FFE7019845F66F
:10DE30000C01C2F20001086000E0FFE7FFE7FFE726
:10DE400004B080BD80B582B0019001F0BBFA45F20C
:10DE5000E001C2F2000108680130086040F6547029
:10DE6000C2F20000006898B9FFE7019840F65471CB
:10DE7000C2F20001086045F2E000C2F20000006852
:10DE8000012803D1FFE700F021FB00E0FFE71CE0E1
:10DE900045F67400C2F200000068A0B9FFE740F642
:10DEA0005470C2F200000068C06A0199C96A8842D1
:10DEB00007D8FFE7019840F65471C2F200010860EC
:10DEC00000E0FFE700E0FFE7FFE745F2EC00C2F209
:10DED00000000168013101600068019948640198FF
:10DEE000C06A45F2F001C2F200010968884208D90F
:10DEF000FFE70198C06A45F2F001C2F20001086034
:10DF0000FFE70199C86A00EB800240F66C70C2F22C
:10DF1000000000EB8200043101F02CFA01F07EFADF
:10DF200045F67400C2F200000068C8B1FFE740F691
:10DF30005470C2F200000068C06A0199C96A884240
:10DF40000CD2FFE74EF60451CEF200014FF08050A4
:10DF50000860BFF34F8FBFF36F8F00E0FFE700E073
:10DF6000FFE702B080BD000080B584B001F02AFA5E
:10DF700045F6AC00C2F200000068002840D1FFE77F
:10DF800045F2AC70C2F20000029001F09DF945F23A
:10DF9000C070C2F20000039001F096F90299039854
:10DFA00040F65872C2F20002116040F66871C2F287
:10DFB0000001086069460020086040F66062C2F215
:10DFC000000240F60073C2F200030A20102101F0A3
:10DFD000CBFF014645F6AC00C2F2000001600068CC
:10DFE00060B1FFE745F6AC00C2F20000006844F201
:10DFF000ED41C0F6010101F003FB00E0FFE700E0A6
:10E00000FFE701F00BFA04B080BD000080B582B0DC
:10E01000FFE745F2E400C2F20000006808B3FFE742
:10E0200001F0D0F945F69400C2F20000C068C06863
:10E0300001900198043001F0F7F845F2E001C2F2D6
:10E04000000108680138086045F2E401C2F20001ED
:10E0500008680138086001F0E1F9019800F08CF8D7
:10E06000D7E702B080BD000080B582B0019000917A
:10E070000198006CB8B1FFE70199C8680A6C1044B8
:10E08000C86001988168C068884204D3FFE701999D
:10E090000868C86000E0FFE70098019AD168126C38
:10E0A000F2F75AF9FFE702B080BD000080B586B0F4
:10E0B000059004910392002002900598806B0190D6
:10E0C0000598006C78B9FFE70598006848B9FFE744
:10E0D0000598806803F02AF902900599002088606D
:10E0E00000E0FFE741E00398B8B9FFE7059A04991B
:10E0F0005068126CF2F730F9059948680A6C1044C0
:10E100004860059948688968884204D3FFE7059903
:10E110000868486000E0FFE726E0059A0499D068A7
:10E12000126CF2F719F90599C8680A6C801AC86070
:10E1300005980168C068884206D2FFE7059988689B
:10E140000A6C801AC86000E0FFE70398022809D132
:10E15000FFE7019820B1FFE701980138019000E046
:10E16000FFE700E0FFE7FFE7FFE7019801300599CF
:10E170008863029806B080BD80B582B00090009898
:10E1800090F8590040B9FFE70098006B01F06CF976
:10E19000009801F069F91CE0009890F859000128F6
:10E1A00004D1FFE7009801F05FF911E0009890F8C2
:10E1B000590002280BD0FFE74FF0500080F3118880
:10E1C000BFF36F8FBFF34F8F0190FFE7FEE7FFE7CD
:10E1D000FFE702B080BD000082B001900198406A64
:10E1E00038B1FFE70198006B0068C0F1380000907B
:10E1F00002E000200090FFE7009802B070470000A6
:10E2000082B0019040F65870C2F2000000680068C9
:10E21000B0FA80F04009019908600198006848B997
:10E22000FFE740F65870C2F200000068C06800685E
:10E23000009002E000200090FFE7009802B07047D5
:10E2400084B04FF47050009041F2D440C2F200000C
:10E2500001909DF80400400788B1FFE7019807305E
:10E260000190019820F007000190019A41F2D441F9
:10E27000C2F200010098891A08440090FFE7019853
:10E280000290029945F67800C2F200000160002178
:10E2900041600298009A104401900198083801905A
:10E2A000019820F007000190019A40F66070C2F2D8
:10E2B00000000260026851600268116002990391D7
:10E2C0000199039A891A51600068039908600398BC
:10E2D000406845F60801C2F20001086003984068F2
:10E2E00045F60001C2F20001086045F2D471C2F2A5
:10E2F00000014FF00040086004B0704780B582B064
:10E300000190FFE7FFF782FE40F66C70C2F200005A
:10E31000006802280CD3FFE74EF60451CEF200014C
:10E320004FF080500860BFF34F8FBFF36F8F00E056
:10E33000FFE7E7E780B582B00190019868B1FFE799
:10E34000019800238360019803600198C3600198DD
:10E3500019461A4601F0EEFE00E0FFE702B080BD6C
:10E3600080B584B0DDF818C00390029101928DF859
:10E370000330029818B9FFE70698006003E001989F
:10E3800006990860FFE703980699C8630298069902
:10E3900008640698012101F06FFE9DF803000699BC
:10E3A00081F84C0004B080BD80B588B0DDF834C081
:10E3B000DDF830C0DDF82CC0DDF828C006900591EE
:10E3C000049203930C98006B04998900A522F2F73C
:10E3D00008F80C98006B049900EB81000438029057
:10E3E000029820F0070002909DF80800400758B1FD
:10E3F000FFE74FF0500080F31188BFF36F8FBFF33A
:10E400004F8F0790FFE7FEE70598F8B1FFE7002080
:10E410000190FFE701980F2813D8FFE70598019AAC
:10E42000805C0C99114481F8340005980199405C96
:10E4300008B9FFE705E0FFE7FFE701980130019029
:10E44000E8E70C99002081F8430004E00C990020D3
:10E4500081F83400FFE70A98382803D3FFE7372014
:10E460000A9000E0FFE70A980C99C8620A980C9994
:10E47000C8640C990020009008650C98043000F0E6
:10E480003BFF0C98183000F037FF00980C99096199
:10E490000A99C1F138010C9A91610C9949620C9961
:10E4A00048650C9981F8580002980699039A00F083
:10E4B000E7FC0C9908600B9820B1FFE70C980B99CA
:10E4C000086000E0FFE708B080BD000080B584B0C0
:10E4D00000200390FFE70398372810D8FFE7039840
:10E4E00000EB800140F66C70C2F2000000EB81008E
:10E4F00000F0EAFEFFE7039801300390EBE745F2F6
:10E50000D870C2F20000019000F0DEFE45F2EC701F
:10E51000C2F20000029000F0D7FE45F62000C2F2E1
:10E52000000000F0D1FE45F69400C2F2000000F0B9
:10E53000CBFE45F68000C2F2000000F0C5FE019956
:10E54000029840F65C72C2F20002116040F66471FB
:10E55000C2F20001086004B080BD000083B00290E8
:10E5600045F67800C2F200000190FFE701980068CC
:10E570000299884205D2FFE7FFE701980068019001
:10E58000F4E70198009000980199496808440299BD
:10E59000884209D1FFE7029842680199486810440F
:10E5A00048600198029000E0FFE702980090009810
:10E5B00002994968084401990968884220D1FFE717
:10E5C0000198006840F66071C2F200010968884253
:10E5D0000DD0FFE70198006842680299486810442E
:10E5E00048600198006800680299086007E040F6FA
:10E5F0006070C2F20000006802990860FFE704E062
:10E600000198006802990860FFE701980299884222
:10E6100004D0FFE702980199086000E0FFE703B02B
:10E620007047000080B586B0059004910392029374
:10E6300000200190049805994860059800610498AD
:10E640000399884216D8FFE703980299401A059962
:10E650008969884203D3FFE70120019009E040F671
:10E660006870C2F2000000680599043100F04CFEA9
:10E67000FFE717E003980299884208D2FFE7049861
:10E680000299884203D3FFE70120019009E040F698
:10E690005870C2F2000000680599043100F034FEA1
:10E6A000FFE7FFE7019806B080BD000080B582B0AB
:10E6B000019000F087FE0198806B18B9FFE70120F8
:10E6C000009002E000200090FFE700F0A7FE009815
:10E6D00002B080BD80B582B0019000F073FE019859
:10E6E000806B0199C96B884203D1FFE7012000903C
:10E6F00002E000200090FFE700F090FE009802B0DA
:10E7000080BD000008480068006880F308884FF06A
:10E71000000080F3148862B661B6BFF34F8FBFF379
:10E720006F8F00DF00BF00BF08ED00E080B586B04E
:10E730000490039140F65870C2F200000068C0686F
:10E74000C06801900198043000F06EFD019890F8C7
:10E7500028004007002823D5FFE70198049B816922
:10E760001944039AFFF75EFFC0B1FFE70198049ACE
:10E77000694600230B60194603F04CF8029002989A
:10E7800058B9FFE74FF0500080F31188BFF36F8F47
:10E79000BFF34F8F0590FFE7FEE700E0FFE707E0DC
:10E7A000019991F8280000F0FE0081F82800FFE7A9
:10E7B0000198016A884706B080BD000080B58EB020
:10E7C000FFE745F6AC00C2F20000006807A900228E
:10E7D00001F0A2FE002800F0B880FFE70798B0F132
:10E7E000FF3F17DCFFE707A804300290029858B9F2
:10E7F000FFE74FF0500080F31188BFF36F8FBFF336
:10E800004F8F0B90FFE7FEE702990A684868896816
:10E81000904700E0FFE70798002800F19580FFE7A8
:10E82000099806900698406928B1FFE706980430D9
:10E8300000F0FAFC00E0FFE705A800F0FBF8039009
:10E8400007980190092800F27D800199DFE801F026
:10E850000505053D456605053D45069991F82800E5
:10E8600040F0010081F828000698089B816919444E
:10E87000039AFFF7D7FE30B3FFE70698016A88478F
:10E88000069890F82800400700281AD5FFE7069858
:10E89000089982690A44694600230B60194602F010
:10E8A000B9FF0490049858B9FFE74FF0500080F387
:10E8B0001188BFF36F8FBFF34F8F0C90FFE7FEE718
:10E8C00000E0FFE700E0FFE73DE0069991F828004F
:10E8D00000F0FE0081F8280035E0069991F8280044
:10E8E00040F0010081F82800089806998861069890
:10E8F000806958B9FFE74FF0500080F31188BFF3EB
:10E900006F8FBFF34F8F0D90FFE7FEE70698039BD5
:10E91000816919441A46FFF785FE14E0069890F8BD
:10E9200028008007002804D4FFE7069800F09CFD2B
:10E9300007E0069991F8280000F0FE0081F8280011
:10E94000FFE700E0FFE7FFE73BE70EB080BD000018
:10E9500080B584B00390029101F068F9684600F038
:10E9600069F801900098D8BBFFE7029860B9FFE70B
:10E9700003980199884207D8FFE702F03DFE03980B
:10E980000199FFF7D3FE2AE0029858B1FFE740F65D
:10E990006870C2F2000000680068B0FA80F04009B8
:10E9A0000290FFE745F6AC00C2F200000068039950
:10E9B000019A891A029A00F04DFE02F01DFE60B91C
:10E9C000FFE74EF60451CEF200014FF08050086090
:10E9D000BFF34F8FBFF36F8F00E0FFE7FFE702E069
:10E9E00002F00AFEFFE704B080BD000081B040F6EF
:10E9F0005C70C2F200000068006840B9FFE745F6AD
:10EA00000C01C2F200014FF0FF3008600FE040F649
:10EA10005C70C2F200000068C068C0680090009896
:10EA2000406845F60C01C2F200010860FFE701B042
:10EA30007047000080B582B0019002F00FFB00909B
:10EA4000009840F65071C2F200010968884206D26F
:10EA5000FFE700F011F801990120086003E0019937
:10EA600000200860FFE7009840F65071C2F20001F4
:10EA70000860009802B080BD80B588B0FFE740F61E
:10EA80005870C2F200000068006800284ED0FFE70E
:10EA900040F65870C2F200000168C9680968069122
:10EAA0000068C068C06803900398043000F0BCFBA5
:10EAB0000398016A8847039890F8280040070028C7
:10EAC00032D5FFE7069803998969084405900598AF
:10EAD000069988420FD9FFE7059803994860039883
:10EAE000006140F65870C2F20000006803990431DA
:10EAF00000F00AFC17E00398069A694600230B60B1
:10EB0000194602F087FE0290029858B9FFE74FF0CD
:10EB1000500080F31188BFF36F8FBFF34F8F0790C2
:10EB2000FFE7FEE7FFE700E0FFE7A8E740F65872DF
:10EB3000C2F200021068049040F66871C2F200014F
:10EB4000086810600498086008B080BD83B0002099
:10EB5000009040F20010C2F200000068013058B18D
:10EB6000FFE74FF0500080F31188BFF36F8FBFF3C2
:10EB70004F8F0190FFE7FEE74FF0500080F31188C0
:10EB8000BFF36F8FBFF34F8F0290FFE7009808B974
:10EB9000FFE7FBE703B0704780B584B00390FFE761
:10EBA00001A8FFF72DFB029002980199FFF7D0FE14
:10EBB000FFF704FEF4E7000080B582B0019000F09A
:10EBC00001FC019890F845008DF80300FFE79DF9DE
:10EBD0000300012816DBFFE70198406A58B1FFE700
:10EBE0000198243002F0A0FC18B1FFE700F0C0FE4D
:10EBF00000E0FFE700E005E09DF8030001388DF834
:10EC00000300E4E70199FF2081F8450000F006FCCD
:10EC100000F0D8FB019890F844008DF80200FFE75F
:10EC20009DF90200012816DBFFE70198006980B119
:10EC3000FFE70198103002F077FC18B1FFE700F011
:10EC400097FE00E0FFE79DF8020001388DF8020012
:10EC500000E000E0E4E70199FF2081F8440000F0C3
:10EC6000DDFB02B080BD000080B58AB006900020B8
:10EC7000029000F0DBFF40F66070C2F20000006816
:10EC800018B9FFE7FFF7DCFA00E0FFE7069845F266
:10EC9000D471C2F200010968084240F0C580FFE764
:10ECA000069800B3FFE70698083006909DF8180014
:10ECB0004007B0B1FFE7069820F007000830069043
:10ECC0009DF81800400758B1FFE74FF0500080F35F
:10ECD0001188BFF36F8FBFF34F8F0790FFE7FEE7F9
:10ECE00000E0FFE700E0FFE70698002800F09A80C8
:10ECF000FFE7069845F60001C2F200010968884264
:10ED000000F29080FFE745F67800C2F20000049020
:10ED100000680590FFE705984168069A0020914237
:10ED2000019007D2FFE705980068002818BF01206E
:10ED30000190FFE70198C00730B1FFE70598049004
:10ED4000059800680590E6E7059840F66071C2F204
:10ED500000010968884263D0FFE704980068083022
:10ED60000290059800680499086005984068069923
:10ED7000401A112821D3FFE705980699084403900B
:10ED80009DF80C00400758B1FFE74FF0500080F3AA
:10ED90001188BFF36F8FBFF34F8F0890FFE7FEE737
:10EDA000059840680699401A0399486006980599A5
:10EDB00048600398FFF7D2FB00E0FFE70598426840
:10EDC00045F60000C2F200000168891A016000687F
:10EDD00045F60801C2F20001096888420BD2FFE73C
:10EDE00045F60000C2F20000006845F60801C2F2D4
:10EDF0000001086000E0FFE745F2D470C2F20000B5
:10EE00000268059948681043486005990020086029
:10EE100045F61401C2F2000108680130086000E004
:10EE2000FFE700E0FFE700E0FFE702F0E5FB9DF809
:10EE30000800400758B1FFE74FF0500080F31188F9
:10EE4000BFF36F8FBFF34F8F0990FFE7FEE7029884
:10EE50000AB080BD40F65470C2F20000006848B1AC
:10EE6000FFE740F65470C2F200000168086D0130FF
:10EE70000865FFE740F65470C2F200000068704772
:10EE800083B0029001910092029804380290029996
:10EE90004FF080700860029804380290019820F0CA
:10EEA00001000299086002980438029002994EF617
:10EEB0004D30C0F6000008600298143802900098A7
:10EEC0000299086002980438029002996FF00200DB
:10EED0000860029820380290029803B07047000042
:10EEE00080B541F2F930C2F2000000F11901192297
:10EEF000FCF7B0F980BD000080B586B005900491A4
:10EF0000059818B1FFE7049808B9FFE77EE1059876
:10EF100040780599897840EA01206FF3DF2000EE00
:10EF2000100AB8EEC00A049880ED000A05988078AF
:10EF3000C0080599C97840EA41106FF3DF2000EE60
:10EF4000100AB8EEC00A049880ED030A0598C0784C
:10EF500080090599097940EA81000599497940EAD3
:10EF600081206FF3DF2000EE100AB8EEC00A04988B
:10EF700080ED010A0598407940080599897940EAB1
:10EF8000C1106FF3DF2000EE100AB8EEC00A04983B
:10EF900080ED020A0598807900090599C97940EA4F
:10EFA00001106FF3DF20049988830598C079C009A8
:10EFB0000599097A40EA41000599497A40EA4120D9
:10EFC0006FF3DF20049908820598407A800805993C
:10EFD000897A40EA81106FF3DF200499488305980D
:10EFE000807A40090599C97A40EAC10004990883EA
:10EFF0000598007B0599497B40EA01206FF3DF20EB
:10F000000499C8820598407BC0080599897B40EA2D
:10F0100041106FF3DF20049988820598807B800976
:10F020000599C97B40EA81000599097C40EA812065
:10F030006FF3DF20049948820598007C4008059909
:10F04000497C40EAC1106FF3DF200499C88304981B
:10F0500090ED010ADFED720ACDED000A9FED711A05
:10F060008DED011AFFEE001ACDED021AB7EE002A5F
:10F070008DED032AFEF7D2F8DDED000A9DED011AB1
:10F08000DDED021A9DED032A049880ED010A049833
:10F0900090ED000AFEF7C2F8DDED000A9DED011AC1
:10F0A000DDED021A9DED032A049880ED000A049814
:10F0B00090ED020AFEF7B2F8DDED000A9DED011AAF
:10F0C000DDED021A9DED032A049880ED020A0498F2
:10F0D00090ED030AFEF7A2F8049880ED030A049865
:10F0E000006804F069FF41EC100B9FED491B53ECE5
:10F0F000112B51EC100B04F0A6FFA0B9FFE7049808
:10F10000006804F059FF41EC100B9FED431B53ECDA
:10F11000112B51EC100B04F08FFF20B9FFE704997D
:10F1200000200860FFE70498406804F045FF41ECC8
:10F13000100B9FED371B53EC112B51EC100B04F00F
:10F1400082FFA0B9FFE70498406804F035FF41EC66
:10F15000100B9FED311B53EC112B51EC100B04F0F5
:10F1600064FF20B9FFE7049900204860FFE7049896
:10F17000806804F021FF41EC100B9FED251B53EC40
:10F18000112B51EC100B04F05EFFA0B9FFE70498BF
:10F19000806804F011FF41EC100B9FED1F1B53EC36
:10F1A000112B51EC100B04F040FF20B9FFE704993C
:10F1B00000208860FFE70498C06804F0FDFE41EC81
:10F1C000100B9FED131B53EC112B51EC100B04F0A3
:10F1D0003AFFA0B9FFE70498C06804F0EDFE41ECE7
:10F1E000100B9FED0D1B53EC112B51EC100B04F089
:10F1F0001CFF20B9FFE704990020C860FFE741F237
:10F20000F831C2F2000101200870FFE706B080BDAE
:10F210007B14AE47E17A84BF7B14AE47E17A843F2A
:10F220000000B04300E0D34482B00190019800692F
:10F2300000900198416880688860019948688968F1
:10F240004860009840680199884205D1FFE701981D
:10F2500080680099486000E0FFE70199002008619C
:10F2600000990868013808600098006802B070478B
:10F2700083B0029001910092029945F2F420C2F20B
:10F2800000000860019945F2F400C2F20000086035
:10F2900000998020086003B07047000083B002909E
:10F2A00001910092029945F25070C2F2000008608C
:10F2B000019945F25030C2F20000086000994FF405
:10F2C0008070086003B0704781B00090009901F130
:10F2D0000800486000994FF0FF308860009901F104
:10F2E0000800C860009901F1080008610099002039
:10F2F000086001B07047000081B0009000990020C4
:10F30000086101B07047000084B003900291029838
:10F31000006800900098013020B9FFE70398006969
:10F32000019010E0039808300190FFE701984068D1
:10F3300000680099884205D8FFE7FFE70198406818
:10F340000190F3E7FFE7019840680299486002984E
:10F350004168886001980299886002980199486024
:10F36000039802990861039908680130086004B0A5
:10F370007047000083B002900191029840680090AD
:10F380000098019948600098806801998860019808
:10F3900000998968486001980099886002980199ED
:10F3A0000861029908680130086003B070470000E6
:10F3B000DFF80C00016841F470010160704700BF84
:10F3C00088ED00E082B04FF0500080F31188BFF369
:10F3D0006F8FBFF34F8F009040F20010C2F2000019
:10F3E0000168013101600068012814D1FFE74EF681
:10F3F0000450CEF200000068000658B1FFE74FF05D
:10F40000500080F31188BFF36F8FBFF34F8F0190CF
:10F41000FFE7FEE7FFE702B07047000082B040F26E
:10F420000010C2F20000006858B9FFE74FF050002A
:10F4300080F31188BFF36F8FBFF34F8F0090FFE70A
:10F44000FEE740F20010C2F20000016801390160DD
:10F45000006830B9FFE700200190019880F311881F
:10F46000FFE702B07047000080B586B003900398B4
:10F470000290039800285CD0FFE7029808380290B9
:10F48000029801900198406845F2D471C2F20001DF
:10F49000096808420BD1FFE74FF0500080F3118854
:10F4A000BFF36F8FBFF34F8F0490FFE7FEE7019824
:10F4B000006858B1FFE74FF0500080F31188BFF3A8
:10F4C0006F8FBFF34F8F0590FFE7FEE7019840680D
:10F4D00045F2D471C2F200010968084227D0FFE763
:10F4E0000198006808BBFFE745F2D470C2F2000043
:10F4F0000268019948689043486000F097FB0198C2
:10F50000426845F60001C2F2000108681044086034
:10F510000198FFF723F845F61801C2F200010868C8
:10F520000130086002F068F800E0FFE700E0FFE764
:10F53000FFE706B080BD00004EF21001CEF20001E0
:10F54000002008604EF21802CEF20002106040F275
:10F550000000C2F20000006844F6D352C1F2620219
:10F56000A0FB02024FF0FF3000EB92104EF21402AB
:10F57000CEF20002106007200860704784B0EFF3FD
:10F5800005800190019810281ED3FFE701984EF2E4
:10F59000F031CEF20001405C8DF803009DF80300CD
:10F5A00045F2D401C2F20001097888420BDAFFE784
:10F5B0004FF0500080F31188BFF36F8FBFF34F8F70
:10F5C0000290FFE7FEE7FFE74EF60C50CEF2000098
:10F5D000006800F4E06045F2D801C2F20001096859
:10F5E00088420BD9FFE74FF0500080F31188BFF33A
:10F5F0006F8FBFF34F8F0390FFE7FEE704B07047B4
:10F6000083B00290019100200090FFE70098072846
:10F610001DD8FFE7009945F63400C2F2000050F80B
:10F62000310070B9FFE70198009A45F63401C2F243
:10F63000000141F832000298009A01EBC2014860D3
:10F6400005E0FFE7FFE7009801300090DEE703B038
:10F650007047000080B584B0039002910192039836
:10F660000090FFF7AFFE009890F94400013028B9F0
:10F67000FFE70099002081F84400FFE7009890F927
:10F680004500013028B9FFE70099002081F84500C6
:10F69000FFE7FFF7C3FE0098806B38B9FFE70098DB
:10F6A00024300299019A00F08DF900E0FFE70098FC
:10F6B000FFF782FA04B080BD80B584B002900020CC
:10F6C00001900298E0B1FFE745F2E800C2F20000C5
:10F6D000006858B1FFE74FF0500080F31188BFF386
:10F6E0006F8FBFF34F8F0390FFE7FEE700F09EFAA6
:10F6F00002980021FEF73CFB01F07EFF019000E044
:10F70000FFE7019860B9FFE74EF60451CEF2000121
:10F710004FF080500860BFF34F8FBFF36F8F00E052
:10F72000FFE704B080BD000080B58AB00690059167
:10F7300000200290069858B9FFE74FF0500080F380
:10F740001188BFF36F8FBFF34F8F0790FFE7FEE77E
:10F75000059858B9FFE74FF0500080F31188BFF3C8
:10F760006F8FBFF34F8F0890FFE7FEE745F2E80089
:10F77000C2F20000006858B1FFE74FF0500080F37C
:10F780001188BFF36F8FBFF34F8F0990FFE7FEE73C
:10F7900000F04CFA45F6A800C2F2000000680190A3
:10F7A000069800680599084404900198069909682C
:10F7B000884210D2FFE7049806990968884208D267
:10F7C000FFE704980199884203D9FFE701200290DE
:10F7D00000E0FFE70FE0049806990968884205D326
:10F7E000FFE704980199884203D9FFE701200290BE
:10F7F00000E0FFE7FFE7049806990860029838B137
:10F80000FFE704980199401A0021FEF7B1FA00E0E1
:10F81000FFE701F0F1FE0390039860B9FFE74EF6B1
:10F820000451CEF200014FF080500860BFF34F8FBB
:10F83000BFF36F8F00E0FFE70AB080BD80B584B0F2
:10F840000290FFF7BFFD029838B9FFE740F6547009
:10F85000C2F200000068009002E002980090FFE70A
:10F860000098019001980430FFF7DEFC08B9FFE72B
:10F8700000E0FFE70198806A28B1FFE7019818309F
:10F88000FFF7D2FC00E0FFE745F2EC01C2F2000115
:10F89000086801300860019840F65471C2F2000116
:10F8A0000968884210D1FFE70198011D45F69400D0
:10F8B000C2F20000FFF75EFD45F2E401C2F2000172
:10F8C0000868013008600CE045F2E001C2F2000176
:10F8D0000868013808600198FEF74EFCFFF786F8CB
:10F8E000FFE7FFF79BFD45F67400C2F200000068D9
:10F8F00048B3FFE7019840F65471C2F2000109686D
:10F9000088421ED1FFE745F2E800C2F2000000681D
:10F9100058B1FFE74FF0500080F31188BFF36F8FAD
:10F92000BFF34F8F0390FFE7FEE74EF60451CEF290
:10F9300000014FF080500860BFF34F8FBFF36F8F0F
:10F9400000E0FFE7FFE704B080BD000081B0009059
:10F9500045F61000C2F2000000680099086045F604
:10F96000A800C2F2000000680099486001B070472A
:10F9700045F6B401C2F200010120086070470000A2
:10F9800080B584B002900191029858B9FFE74FF01A
:10F99000500080F31188BFF36F8FBFF34F8F039038
:10F9A000FFE7FEE7029840F65471C2F200010968D1
:10F9B0001831FFF7A9FC01980121FEF7D9F904B02D
:10F9C00080BD000080B584B0029001910092029841
:10F9D00058B9FFE74FF0500080F31188BFF36F8FE5
:10F9E000BFF34F8F0390FFE7FEE7029840F6547194
:10F9F000C2F2000109681831FFF7BCFC009820B181
:10FA0000FFE74FF0FF300190FFE701980099FEF704
:10FA1000AFF904B080BD000080B588B005900491B6
:10FA200005980390012000900598002800F08B8035
:10FA3000FFE70398006D58B9FFE74FF0500080F3DF
:10FA40001188BFF36F8FBFF34F8F0690FFE7FEE77C
:10FA50000398C06C0499884203D2FFE70498019090
:10FA600003E00398C06C0190FFE70398C06A019916
:10FA7000884266D0FFE70398006D01285FD1FFE759
:10FA8000039840F65471C2F20001096888420BD114
:10FA9000FFE74FF0500080F31188BFF36F8FBFF383
:10FAA0004F8F0790FFE7FEE70398C06A0290019826
:10FAB0000399C8620398C07E0006002806D4FFE7B9
:10FAC0000198C0F138000399886100E0FFE70398CE
:10FAD0004069029901EB810240F66C71C2F20001AB
:10FAE00001EB8201884228D1FFE703980430FFF739
:10FAF0009BFB08B9FFE700E0FFE70398C06A45F207
:10FB0000F001C2F200010968884208D9FFE70398B2
:10FB1000C06A45F2F001C2F200010860FFE70399F4
:10FB2000C86A00EB800240F66C70C2F2000000EB85
:10FB300082000431FFF71EFC00E0FFE700E0FFE772
:10FB400000E0FFE700E0FFE708B080BD80B58AB0C5
:10FB5000002003900690059006A805A904AAFFF7C7
:10FB600087FB039B049A0599DDF818C06846C0F826
:10FB700008C0416003604EF2FD20C0F6000044F270
:10FB8000E841C0F6010101F03DF8014645F60400E8
:10FB9000C2F200000160006818B1FFE70120079081
:10FBA00002E000200790FFE70798012804D1FFE753
:10FBB00001F0E6FD079000E0FFE70798012823D158
:10FBC000FFE74FF0500080F31188BFF36F8FBFF352
:10FBD0004F8F089045F60C01C2F200014FF0FF3044
:10FBE000086045F67401C2F200010120086045F684
:10FBF000A801C2F200010020086000F083F808B1FB
:10FC0000FFE700E0FFE70FE00798013058B9FFE792
:10FC10004FF0500080F31188BFF36F8FBFF34F8F09
:10FC20000990FFE7FEE7FFE70AB080BD45F2E80173
:10FC3000C2F20001086801300860704783B045F2E5
:10FC4000E800C2F20000006838B1FFE745F6B401F1
:10FC5000C2F200010120086051E045F6B401C2F291
:10FC600000010020086045F2F000C2F200000068C8
:10FC70000190FFE7019800EB800140F66C70C2F242
:10FC8000000050F8210090B9FFE7019858B9FFE74C
:10FC90004FF0500080F31188BFF36F8FBFF34F8F89
:10FCA0000290FFE7FEE7019801380190E2E7019832
:10FCB00000EB800140F66C70C2F2000000EB8100A6
:10FCC0000090009948684068486000994868083189
:10FCD000884205D1FFE70099486840684860FFE71F
:10FCE00000984068C06840F65471C2F20001086094
:10FCF000019845F2F001C2F200010860FFE703B08D
:10FD00007047000080B588B04EF60050CEF200007B
:10FD100000684CF27121C4F20F1188420BD1FFE749
:10FD20004FF0500080F31188BFF36F8FBFF34F8FF8
:10FD30000590FFE7FEE74EF60050CEF200000068A7
:10FD40004CF27021C4F20F1188420BD1FFE74FF043
:10FD5000500080F31188BFF36F8FBFF34F8F069071
:10FD6000FFE7FEE74EF20040CEF20000039001787C
:10FD70000491FF21017000788DF80B009DF80B00B5
:10FD800000F0500045F2D401C2F20001087045F2C3
:10FD9000D801C2F2000107200860FFE79DF80B00C0
:10FDA000000600280DD5FFE745F2D801C2F2000198
:10FDB0000868013808609DF80B0040008DF80B00C2
:10FDC000ECE745F2D800C2F20000006803280BD02F
:10FDD000FFE74FF0500080F31188BFF36F8FBFF340
:10FDE0004F8F0790FFE7FEE745F2D801C2F200010E
:10FDF000086800020860086800F4E0600860049881
:10FE00004EF20041CEF2000108704EF62051CEF2C3
:10FE10000001086840F470000860086840F0704015
:10FE20000860FFF789FB40F20011C2F200010020D8
:10FE300001900860FFF7BCFA4EF63471CEF2000173
:10FE4000086840F040400860FEF75CFCFFF7F6FEF3
:10FE5000FEF77CFE019808B080BD000080B582B03E
:10FE60004FF0500080F31188BFF36F8FBFF34F8FB7
:10FE7000009001F00DF940B1FFE74EF60451CEF2CB
:10FE800000014FF080500860FFE7002001900198CA
:10FE900080F3118802B080BD80B584B08DF80F006A
:10FEA00001200190002100919DF80F2000F022F820
:10FEB00002900298FEF73EFA029804B080BD00005E
:10FEC00080B586B08DF817000491012002900022C1
:10FED00001929DF81710049BEC46CCF800101146D7
:10FEE00000F042F803900398FEF724FA039806B056
:10FEF00080BD000080B588B0069005918DF8132074
:10FF0000069858B9FFE74FF0500080F31188BFF30F
:10FF10006F8FBFF34F8F0790FFE7FEE706980599B5
:10FF20004843029002985030FEF79EFE03900398DB
:10FF3000B0B1FFE703980190019850300190039908
:10FF4000002081F8460006980599019A9DF8133023
:10FF5000DDF80CC0EE46CEF800C0FEF701FA00E076
:10FF6000FFE7039808B080BD80B590B08446129832
:10FF7000CDF828C00991089207938DF81B000A98C4
:10FF800058B9FFE74FF0500080F31188BFF36F8F2F
:10FF9000BFF34F8F0B90FFE7FEE7079858B9FFE7D5
:10FFA0004FF0500080F31188BFF36F8FBFF34F8F76
:10FFB0000C90FFE7FEE708990020039031B1FFE7BE
:10FFC0000998B0FA80F040090390FFE70398C00752
:10FFD00058B1FFE74FF0500080F31188BFF36F8FE7
:10FFE000BFF34F8F0D90FFE7FEE7089900200290C6
:10FFF00031B9FFE70998002818BF01200290FFE7F8
:020000040801F1
:100000000298C00758B1FFE74FF0500080F3118805
:10001000BFF36F8FBFF34F8F0E90FFE7FEE75020C7
:100020000490049850280BD0FFE74FF0500080F365
:100030001188BFF36F8FBFF34F8F0F90FFE7FEE77D
:10004000049807980590059888B1FFE70599012065
:1000500081F846000A980999089A9DF81B30DDF846
:1000600014C0EE46CEF800C0FEF77AF900E0FFE7D4
:10007000059810B080BD000080B584B00290019159
:1000800002980090009858B9FFE74FF0500080F3B5
:100090001188BFF36F8FBFF34F8F0390FFE7FEE729
:1000A000FFF790F900990B68C86B0A6C00FB0230EF
:1000B000886000990020886300990868486000996A
:1000C0000B68C86B0A6C013800FB0230C8600099ED
:1000D000FF2081F84400009981F845000198D0B9CB
:1000E000FFE700980069A0B1FFE70098103001F029
:1000F0001BFA60B1FFE74EF60451CEF200014FF05B
:1001000080500860BFF34F8FBFF36F8F00E0FFE7B1
:1001100000E0FFE708E000981030FFF7D5F80098FE
:100120002430FFF7D1F8FFE7FFF778F9012004B09A
:1001300080BD000080B592B00C900B910A9209939B
:10014000002008900C980490049858B9FFE74FF0ED
:10015000500080F31188BFF36F8FBFF34F8F0E9065
:10016000FFE7FEE70B990020039039B9FFE70498F9
:10017000006C002818BF01200390FFE70398C00718
:1001800058B1FFE74FF0500080F31188BFF36F8F35
:10019000BFF34F8F0F90FFE7FEE709990020022978
:1001A000029007D1FFE70498C06B013818BF012007
:1001B0000290FFE70298C00758B1FFE74FF05000E8
:1001C00080F31188BFF36F8FBFF34F8F1090FFE75D
:1001D000FEE700F027FF01460020019031B9FFE75C
:1001E0000A98002818BF01200190FFE70198C00776
:1001F00058B1FFE74FF0500080F31188BFF36F8FC5
:10020000BFF34F8F1190FFE7FEE7FFE7FFF7DAF844
:100210000498806B0499C96B884204D3FFE709985E
:10022000022834D1FFE704980B99099AFDF73EFFA5
:1002300007900498406AA0B1FFE70498243001F0C9
:1002400073F960B1FFE74EF60451CEF200014FF0B2
:1002500080500860BFF34F8FBFF36F8F00E0FFE760
:1002600010E0079860B1FFE74EF60451CEF20001AE
:100270004FF080500860BFF34F8FBFF36F8F00E0E7
:10028000FFE7FFE7FFF7CAF801200D9065E00A9845
:1002900028B9FFE7FFF7C2F800200D905DE008984D
:1002A00030B9FFE705A8FFF751FB0120089000E0F7
:1002B000FFE7FFE7FFE7FFF7B1F8FFF7B7FCFFF74E
:1002C00081F8049890F94400013028B9FFE70499B7
:1002D000002081F84400FFE7049890F945000130C0
:1002E00028B9FFE70499002081F84500FFE7FFF7F0
:1002F00095F805A80AA900F0CFFB28BBFFE70498F2
:10030000FEF7E8F9C8B1FFE7049810300A99FFF743
:1003100037FB0498FEF750FC01F06EF960B9FFE777
:100320004EF60451CEF200014FF080500860BFF34A
:100330004F8FBFF36F8FFFE705E00498FEF73CFC9B
:1003400001F05AF9FFE707E00498FEF735FC01F0E9
:1003500053F900200D9000E058E70D9812B080BDD1
:1003600080B592B00B900A91099208930B98059072
:10037000059858B9FFE74FF0500080F31188BFF39C
:100380006F8FBFF34F8F0C90FFE7FEE70A990020B5
:10039000029039B9FFE70598006C002818BF0120CA
:1003A0000290FFE70298C00758B1FFE74FF05000F6
:1003B00080F31188BFF36F8FBFF34F8F0D90FFE76E
:1003C000FEE7089900200229019007D1FFE7059870
:1003D000C06B013818BF01200190FFE70198C007EA
:1003E00058B1FFE74FF0500080F31188BFF36F8FD3
:1003F000BFF34F8F0E90FFE7FEE7FFF7BFF8EFF375
:1004000011814FF0500080F31188BFF36F8FBFF35D
:100410004F8F10910F90109806900598806B05995A
:10042000C96B884204D3FFE70898022833D1FFE75D
:10043000059890F845008DF813000598806B03909F
:1004400005980A99089AFDF731FE9DF913000130CD
:10045000B8B9FFE70598406A88B1FFE705982430EE
:1004600001F062F848B1FFE7099820B1FFE7099968
:100470000120086000E0FFE700E0FFE700E0FFE7A1
:1004800006E09DF813000130059981F84500FFE76B
:100490000120079002E000200790FFE706981190E6
:1004A000119880F31188079812B080BD80B586B08E
:1004B000049004980290029858B9FFE74FF050005A
:1004C00080F31188BFF36F8FBFF34F8F0590FFE765
:1004D000FEE702988068019000F09AFD01460198BD
:1004E000884213D1FFE70299C8680138C8600298B2
:1004F000C06838B9FFE70298002319461A46FFF78B
:1005000019FE00E0FFE70120039002E000200390C5
:10051000FFE7039806B080BD80B58EB009900891C2
:1005200007920020069009980390039858B9FFE7B6
:100530004FF0500080F31188BFF36F8FBFF34F8FE0
:100540000B90FFE7FEE708990020019039B9FFE71B
:100550000398006C002818BF01200190FFE7019864
:10056000C00758B1FFE74FF0500080F31188BFF388
:100570006F8FBFF34F8F0C90FFE7FEE700F052FD47
:1005800001460020009031B9FFE70798002818BF06
:1005900001200090FFE70098C00758B1FFE74FF037
:1005A000500080F31188BFF36F8FBFF34F8F0D9012
:1005B000FFE7FEE7FFE7FEF705FF0398806B029079
:1005C000029830B3FFE703980899FDF74DFD0298B4
:1005D00001380399886303980069A0B1FFE7039885
:1005E000103000F0A1FF60B1FFE74EF60451CEF2EB
:1005F00000014FF080500860BFF34F8FBFF36F8F43
:1006000000E0FFE700E0FFE7FEF708FF01200A90A7
:100610006DE0079828B9FFE7FEF700FF00200A9079
:1006200065E0069830B9FFE704A8FFF78FF90120CD
:10063000069000E0FFE7FFE7FFE7FEF7EFFEFFF7BA
:10064000F5FAFEF7BFFE039890F94400013028B98F
:10065000FFE70399002081F84400FFE7039890F931
:100660004500013028B9FFE70399002081F84500D3
:10067000FFE7FEF7D3FE04A807A900F00DFA30BB90
:10068000FFE70398FEF712F8D0B1FFE70398243094
:100690000799FFF775F90398FEF78EFA00F0ACFFA3
:1006A00060B9FFE74EF60451CEF200014FF08050E2
:1006B0000860BFF34F8FBFF36F8F00E0FFE705E0E7
:1006C0000398FEF779FA00F097FFFFE70EE0039832
:1006D000FEF772FA00F090FF0398FDF7E7FF18B1FC
:1006E000FFE700200A9002E0FFE7FFE763E70A98D0
:1006F0000EB080BD80B58EB0089007910692089824
:100700000390039858B9FFE74FF0500080F3118829
:10071000BFF36F8FBFF34F8F0990FFE7FEE7079995
:100720000020009039B9FFE70398006C002818BF3B
:1007300001200090FFE70098C00758B1FFE74FF095
:10074000500080F31188BFF36F8FBFF34F8F0A9073
:10075000FFE7FEE7FEF712FFEFF311814FF05000C5
:1007600080F31188BFF36F8FBFF34F8F0C910B9005
:100770000C9804900398806B0290029898B3FFE75E
:10078000039890F844008DF8070003980799FDF747
:100790006BFC02980138039988639DF907000130CA
:1007A000B8B9FFE70398006988B1FFE703981030F4
:1007B00000F0BAFE48B1FFE7069820B1FFE70699BE
:1007C0000120086000E0FFE700E0FFE700E0FFE74E
:1007D00006E09DF807000130039981F84400FFE727
:1007E0000120059002E000200590FFE704980D909D
:1007F0000D9880F3118805980EB080BD80B590B03B
:100800000A900991002008900A9905910490059892
:1008100058B9FFE74FF0500080F31188BFF36F8F96
:10082000BFF34F8F0C90FFE7FEE70598006C58B1BF
:10083000FFE74FF0500080F31188BFF36F8FBFF3D5
:100840004F8F0D90FFE7FEE700F0ECFB0146002024
:10085000019031B9FFE70998002818BF01200190E5
:10086000FFE70198C00758B1FFE74FF0500080F351
:100870001188BFF36F8FBFF34F8F0E90FFE7FEE736
:10088000FFE7FEF79FFD0598806B0390039860B328
:10089000FFE703980138059988630598006828B92F
:1008A000FFE7FEF7D7FA0599886000E0FFE70598B3
:1008B0000069A0B1FFE70598103000F035FE60B187
:1008C000FFE74EF60451CEF200014FF08050086071
:1008D000BFF34F8FBFF36F8F00E0FFE700E0FFE74C
:1008E000FEF79CFD01200B909BE0099898B9FFE76B
:1008F000049858B1FFE74FF0500080F31188BFF320
:100900006F8FBFF34F8F0F90FFE7FEE7FEF786FD77
:1009100000200B9085E0089830B9FFE706A8FFF7A4
:1009200015F80120089000E0FFE7FFE7FFE7FEF77A
:1009300075FDFFF77BF9FEF745FD059890F944003A
:10094000013028B9FFE70599002081F84400FFE74E
:10095000059890F94500013028B9FFE70599002076
:1009600081F84500FFE7FEF759FD06A809A900F048
:1009700093F8A8BBFFE70598FDF798FE48B3FFE79B
:100980000598006850B9FFE7FEF71CFD05988068E0
:1009900000F042FD0490FEF741FD00E0FFE70598FE
:1009A00024300999FEF7ECFF0598FEF705F900F0F1
:1009B00023FE60B9FFE74EF60451CEF200014FF07E
:1009C00080500860BFF34F8FBFF36F8F00E0FFE7E9
:1009D00005E00598FEF7F0F800F00EFEFFE71FE0D7
:1009E0000598FEF7E9F800F007FE0598FDF75EFEB2
:1009F000A0B1FFE7049870B1FFE7FEF7E3FC0598AC
:100A0000FDF7EAFB0290059880680299FFF704F869
:100A1000FEF704FDFFE700200B9002E0FFE7FFE791
:100A20002FE70B9810B080BD80B586B0049003917D
:100A300004980190019858B9FFE74FF0500080F3F7
:100A40001188BFF36F8FBFF34F8F0590FFE7FEE76D
:100A500001988068009000F0DBFA01460098884217
:100A600007D1FFE70199C8680130C86001200290F2
:100A70000EE001980399FFF7C1FE0290029828B199
:100A8000FFE70199C8680130C86000E0FFE7FFE7B1
:100A9000029806B080BD000080B588B00590049132
:100AA000059858B9FFE74FF0500080F31188BFF365
:100AB0006F8FBFF34F8F0690FFE7FEE7049858B99A
:100AC000FFE74FF0500080F31188BFF36F8FBFF343
:100AD0004F8F0790FFE7FEE7FEF774FC45F6A8008E
:100AE000C2F2000000680290029805994968401A15
:100AF000019004980068013018B9FFE700200390C6
:100B00002BE045F61000C2F2000000680599096864
:100B1000884209D0FFE7029805994968884203D3C3
:100B2000FFE70120039017E00198049909688842C3
:100B30000BD2FFE7019A04990868801A08600598AB
:100B4000FEF704FF0020039005E0049900200860F0
:100B500001200390FFE7FFE7FFE7FEF75FFC039844
:100B600008B080BD70B58CB0DDF844C0DDF840C081
:100B70000B900A91ADF826200893BDF8260080005E
:100B8000FEF772F80590059880B1FFE75C20FEF74C
:100B90006BF80790079820B1FFE70598079908635D
:100BA00003E00598FEF760FCFFE702E000200790F5
:100BB000FFE70798F0B1FFE70798002680F8596033
:100BC0000B980A99BDF82620089BDDF840C0119CBF
:100BD000079DEE46CEF80C60CEF80850CEF80440E3
:100BE000CEF800C0FDF7E0FB0798FDF72BF90120D8
:100BF000069003E04FF0FF300690FFE706980CB038
:100C000070BD0000B0B58EB0DDF850C0DDF84CC04E
:100C1000DDF848C00A90099108920793139858B9D3
:100C2000FFE74FF0500080F31188BFF36F8FBFF3E1
:100C30004F8F0B90FFE7FEE7149858B9FFE74FF08E
:100C4000500080F31188BFF36F8FBFF34F8F0C906C
:100C5000FFE7FEE75C20049004985C280BD0FFE7D8
:100C60004FF0500080F31188BFF36F8FBFF34F8FA9
:100C70000D90FFE7FEE70498149820B3FFE7139860
:100C800008B3FFE71498069013980699086306992D
:100C9000022081F859000A980999089A079BDDF803
:100CA00048C0069CEE460025CEF80C50CEF8084011
:100CB00005ACCEF80440CEF800C0FDF775FB0698F1
:100CC000FDF7C0F802E000200590FFE705980EB0A0
:100CD000B0BD000080B58CB0089007918DF81B2046
:100CE000059301200390089858B9FFE74FF0500092
:100CF00080F31188BFF36F8FBFF34F8F0990FFE729
:100D0000FEE708980490FEF75DFB059828B1FFE721
:100D10000498406D05990860FFE7049890F8580022
:100D20008DF80B000499022081F858009DF81B00F3
:100D300001460191042822D80199DFE801F01F0340
:100D4000090E1200079A0499486D1043486527E080
:100D50000499486D0130486522E007980499486578
:100D60001EE09DF80B00022804D0FFE707980499C5
:100D7000486502E000200390FFE711E010E00498CE
:100D8000406D013058B1FFE74FF0500080F31188FB
:100D9000BFF36F8FBFF34F8F0A90FFE7FEE7FFE7C8
:100DA0009DF80B0001284BD1FFE704980430FEF7B3
:100DB0003BFA0498C06A45F2F001C2F200010968EA
:100DC000884208D9FFE70498C06A45F2F001C2F2F0
:100DD00000010860FFE70499C86A00EB800240F652
:100DE0006C70C2F2000000EB82000431FEF7C2FA20
:100DF0000498806A58B1FFE74FF0500080F31188E3
:100E0000BFF36F8FBFF34F8F0B90FFE7FEE70498A0
:100E1000C06A40F65471C2F200010968C96A88428A
:100E20000CD9FFE74EF60451CEF200014FF080508E
:100E30000860BFF34F8FBFF36F8F00E0FFE700E064
:100E4000FFE7FEF7EBFA03980CB080BD80B590B0D9
:100E5000DDF848C0099008918DF81F200693012005
:100E60000390099858B9FFE74FF0500080F31188BC
:100E7000BFF36F8FBFF34F8F0A90FFE7FEE7FEF7D8
:100E80007DFB09980590EFF311814FF0500080F33E
:100E90001188BFF36F8FBFF34F8F0C910B900C989D
:100EA0000290069828B1FFE70598406D0699086002
:100EB000FFE7059890F858008DF813000599022077
:100EC00081F858009DF81F0001460191042822D89E
:100ED0000199DFE801F01F03090E1200089A059935
:100EE000486D1043486527E00599486D0130486515
:100EF00022E00898059948651EE09DF81300022835
:100F000004D0FFE708980599486502E000200390A7
:100F1000FFE711E010E00598406D013058B1FFE7A0
:100F20004FF0500080F31188BFF36F8FBFF34F8FE6
:100F30000D90FFE7FEE7FFE79DF8130001285FD162
:100F4000FFE70598806A58B1FFE74FF0500080F343
:100F50001188BFF36F8FBFF34F8F0E90FFE7FEE74F
:100F600045F2E800C2F20000006820BBFFE70598E8
:100F70000430FEF759F90598C06A45F2F001C2F253
:100F800000010968884208D9FFE70598C06A45F260
:100F9000F001C2F200010860FFE70599C86A00EBA2
:100FA000800240F66C70C2F2000000EB8200043157
:100FB000FEF7E0F909E0059800F1180145F6200078
:100FC000C2F20000FEF7D6F9FFE70598C06A40F6C6
:100FD0005471C2F200010968C96A88420ED9FFE75C
:100FE000129820B1FFE7129901200860FFE745F64B
:100FF000B401C2F200010120086000E0FFE7FFE752
:1010000002980F900F9880F31188039810B080BD5C
:1010100081B040F65470C2F2000000680090009861
:1010200001B0704781B045F67400C2F2000000685C
:1010300018B9FFE7012000900DE045F2E800C2F288
:101040000000006818B9FFE70220009002E00020CD
:101050000090FFE7FFE7009801B0704781B045F6C8
:10106000A800C2F2000000680090009801B070472C
:1010700080B582B0FEF782FA0020009045F6A80005
:10108000C2F2000000680190019802B080BD00002B
:1010900080B586B00020029045F2E800C2F2000060
:1010A0000068002840F0CB80FFE745F6A801C2F2B7
:1010B000000108680130019001980860019858BB50
:1010C000FFE740F65C70C2F200000068006858B1AB
:1010D000FFE74FF0500080F31188BFF36F8FBFF32D
:1010E0004F8F0590FFE7FEE740F65C72C2F2000208
:1010F0001068009040F66471C2F200010868106048
:101100000098086045F61001C2F20001086801303D
:101110000860FDF76BFC00E0FFE7019845F60C0165
:10112000C2F200010968884268D3FFE7FFE740F692
:101130005C70C2F200000068006840B9FFE745F645
:101140000C01C2F200014FF0FF30086055E040F69C
:101150005C70C2F200000068C068C0680490049827
:101160004068039001980399884207D2FFE70398EB
:1011700045F60C01C2F2000108603EE0FFE704986A
:101180000430FEF751F80498806A28B1FFE704980C
:101190001830FEF749F800E0FFE70498C06A45F20E
:1011A000F001C2F200010968884208D9FFE70498FB
:1011B000C06A45F2F001C2F200010860FFE704993D
:1011C000C86A00EB800240F66C70C2F2000000EBCF
:1011D00082000431FEF7CEF80498C06A40F65471DC
:1011E000C2F200010968C96A884203D3FFE70120FF
:1011F000029000E0FFE7FFE799E7FFE740F6547051
:10120000C2F200000068C06A00EB800140F66C701A
:10121000C2F2000050F82100022803D3FFE70120AA
:10122000029000E0FFE745F6B400C2F2000000685B
:1012300018B1FFE70120029000E0FFE707E045F664
:101240001C01C2F20001086801300860FFE7029843
:1012500006B080BD80B586B00590049103920293DC
:10126000FEF7B0F840F65470C2F20000006890F843
:101270005800022822D0FFE7059B40F65470C2F2C6
:1012800000000268516D994351650168012081F8A1
:101290005800029880B1FFE702980121FCF768FD31
:1012A0004EF60451CEF200014FF080500860BFF3BB
:1012B0004F8FBFF36F8F00E0FFE700E0FFE7FEF71F
:1012C000ADF8FEF77FF8039848B1FFE740F6547099
:1012D000C2F200000068406D03990860FFE740F625
:1012E0005470C2F20000006890F85800022803D041
:1012F000FFE7002001900BE0049A40F65470C2F220
:1013000000000168486D9043486501200190FFE7A7
:1013100040F65470C2F200000168002081F85800C5
:10132000FEF77CF8019806B080BD000080B586B05D
:10133000039003980290002001900398002867D042
:10134000FFE7029840F65471C2F200010968884232
:101350000BD0FFE74FF0500080F31188BFF36F8F81
:10136000BFF34F8F0490FFE7FEE70298006D58B976
:10137000FFE74FF0500080F31188BFF36F8FBFF38A
:101380004F8F0590FFE7FEE70299086D0138086569
:101390000299C86AC96C884238D0FFE70298006D8C
:1013A00090BBFFE702980430FDF73EFF08B9FFE766
:1013B00000E0FFE70299C86CC8620299C86AC0F1F0
:1013C000380088610298C06A45F2F001C2F200015B
:1013D0000968884208D9FFE70298C06A45F2F0011F
:1013E000C2F200010860FFE70299C86A00EB8002C0
:1013F00040F66C70C2F2000000EB82000431FDF791
:10140000B9FF0120019000E0FFE700E0FFE700E006
:10141000FFE7019806B080BD80B584B003900398C3
:101420000290002001900398002878D0FFE70298EE
:10143000C06A40F65471C2F200010968C96A884264
:101440005CD2FFE70298C07E000600280BD4FFE7BD
:1014500040F65470C2F200000068C06AC0F1380063
:101460000299886100E0FFE702994869C96A01EBC7
:10147000810240F66C71C2F2000101EB82018842E8
:1014800030D1FFE702980430FDF7CEFE08B9FFE740
:1014900000E0FFE740F65470C2F200000068C06A46
:1014A0000299C8620298C06A45F2F001C2F20001D6
:1014B0000968884208D9FFE70298C06A45F2F0013E
:1014C000C2F200010860FFE70299C86A00EB8002DF
:1014D00040F66C70C2F2000000EB82000431FDF7B0
:1014E00049FF08E040F65470C2F200000068C06A8C
:1014F0000299C862FFE7012001900FE00298C06CDA
:1015000040F65471C2F200010968C96A884203D2E8
:10151000FFE70120019000E0FFE7FFE700E0FFE7C1
:10152000019804B080BD000080B584B0029002989C
:10153000C068C0680190019858B9FFE74FF05000AB
:1015400080F31188BFF36F8FBFF34F8F0390FFE7D6
:10155000FEE701981830FDF767FE45F2E800C2F299
:101560000000006820BBFFE701980430FDF75CFE37
:101570000198C06A45F2F001C2F200010968884290
:1015800008D9FFE70198C06A45F2F001C2F20001F4
:101590000860FFE70199C86A00EB800240F66C70B2
:1015A000C2F2000000EB82000431FDF7E3FE09E027
:1015B000019800F1180145F62000C2F20000FDF785
:1015C000D9FEFFE70198C06A40F65471C2F20001EB
:1015D0000968C96A884208D9FFE70120009045F6EA
:1015E000B401C2F20001086002E000200090FFE7B1
:1015F000009804B080BD000080B584B00020029047
:10160000019045F2E800C2F20000006858B9FFE717
:101610004FF0500080F31188BFF36F8FBFF34F8FEF
:101620000390FFE7FEE7FDF7CDFE45F2E800C2F2CA
:1016300000000168013901600068002840F09980CD
:10164000FFE745F2E000C2F200000068002800F069
:101650008F80FFE7FFE745F62000C2F20000006838
:10166000002842D0FFE745F62000C2F20000C06823
:10167000C068029002981830FDF7D6FD0298043039
:10168000FDF7D2FD0298C06A45F2F001C2F20001F6
:101690000968884208D9FFE70298C06A45F2F0015C
:1016A000C2F200010860FFE70299C86A00EB8002FD
:1016B00040F66C70C2F2000000EB82000431FDF7CE
:1016C00059FE0298C06A40F65471C2F200010968DE
:1016D000C96A884207D3FFE745F6B401C2F20001A8
:1016E0000120086000E0FFE7B5E7029818B1FFE7C6
:1016F000FDF77CF9FFE745F61C00C2F20000006828
:1017000000900098E0B1FFE7FFE7FFF7C1FC38B1B8
:10171000FFE745F6B401C2F200010120086000E0D5
:10172000FFE7009801380090FFE700980028ECD10F
:10173000FFE745F61C01C2F200010020086000E04E
:10174000FFE745F6B400C2F20000006870B1FFE7A1
:10175000012001904EF60451CEF200014FF080506E
:101760000860BFF34F8FBFF36F8F00E0FFE7FFE725
:1017700000E0FFE7FDF752FE019804B080BD0000D5
:1017800080B58AB000200890FCF7EEFB45F6AC006F
:10179000C2F20000006858B3FFE7002004900790F1
:1017A000069007A806A905AAFDF778FD049B059AEF
:1017B0000698DDF81CC06946C1F808C048600220E0
:1017C00008604EF69930C0F6000044F2F241C0F6CF
:1017D0000101FFF717FA014645F6B000C2F200001A
:1017E0000160006818B1FFE701200890FFE700E002
:1017F000FFE7089858B9FFE74FF0500080F31188D1
:10180000BFF36F8FBFF34F8F0990FFE7FEE7089894
:101810000AB080BD80B58AB0DDF830C0089007916D
:101820000692059300200490089858B9FFE74FF0FE
:10183000500080F31188BFF36F8FBFF34F8F099073
:10184000FFE7FEE745F6AC00C2F200000068A8B36F
:10185000FFE7079800900698019008980290079873
:1018600005281EDCFFE7FFF7DDFB02280CD1FFE7B0
:1018700045F6AC00C2F2000000680C9A69460023ED
:10188000FEF758FC04900BE045F6AC00C2F20000F5
:101890000068694600231A46FEF74CFC0490FFE7F7
:1018A0000BE045F6AC00C2F200000068059A6946FC
:1018B0000023FEF755FD0490FFE700E0FFE70498E2
:1018C0000AB080BD03B401984100009850EAC120DD
:1018D00018BF04204A0D18BF40F0010040F2FF720B
:1018E000B2EB515F08BF40F00200012808BF05209D
:1018F00002B070474100080218BF04200A0E18BF4A
:1019000040F001004FF07F4232EA010108BF40F091
:101910000200012808BF05207047000010B54FF0F5
:101920000E402DED028BB0EE408A18EE104A00EB0F
:101930004400B0F1506F4AD84FF0FC40B0EB440F78
:1019400022D2B0EEC80AF7EE000A30EEC00AF6EE78
:10195000000A60EE208A18EE900A01F019FC01EEF0
:10196000100A14F0004F1DBFDFED2D0A9FED2D0A68
:10197000B1EE411ADFED2C0A08BF9FED2C0AF8EEFC
:10198000001A21EE218A05E0DFED290A68EE088AB7
:10199000B0EE600A9FED271ADFED271A30EE080A35
:1019A00048EE811A9FED251A08EEA11ADFED241AE0
:1019B00048EE811A9FED231A08EEA11A68EE281A44
:1019C000BDEC028B01EE810A30EE200A10BD4FF013
:1019D000E440B0EB440F0CD918EE100AFFF78AFF71
:1019E000042808BF01F00EFBB0EE480ABDEC028BE4
:1019F00010BD4FF07F40B0EB440F07D2B0EE480A65
:101A0000BDEC028BBDE8104001F0EEBA0120EEF70C
:101A10001FFDBDEC028BBDE8104001F0EBBA0000E9
:101A20000000C9BF22AAFDB90000C93F22AAFD39A2
:101A30000000000024FE1C3DC78AD83C1E67383DCC
:101A40001B93993DAFAA2A3E70B59B482DED020B22
:101A50002DED068B079D25F00044A04218DC974829
:101A6000844202DC0AD1069840B19DED060BBDEC24
:101A7000068B02B0BDE8704001F082BA002DCCBFE9
:101A80009FED8F0B9FED900BBDEC068B02B070BDF0
:101A90008F48A04215DD8F48A042D8BF4FF0FF34D9
:101AA00058DD9DED060B51EC100BFFF70BFF0428E2
:101AB00008BF01F089FA9DED060BBDEC068B02B064
:101AC00070BD9DED060B51EC100B01F055FBCDE9FF
:101AD000060181489FED828BA0423CDD8248A042F6
:101AE0001FDD00249FED82AB9DED060B53EC1A2BFE
:101AF00051EC100B01F0AAFB9DED060B41EC190B0C
:101B000053EC1A2B51EC100B01F0EAFE53EC182B9E
:101B100002F064F953EC192B01F04CFCCDE90601FD
:101B200049E09DED060B012453EC182B51EC100BF2
:101B300001F08CFB9DED060B41EC190B53EC182BBF
:101B400051EC100B02F04AF953EC192B01F032FC66
:101B5000CDE906012FE06848A0421FDD02249FED79
:101B6000689B9DED060B53EC192B51EC100B01F00B
:101B7000B7FE53EC182B01F069FB9DED060B41EC11
:101B8000180B53EC192B51EC100B02F027F953EC06
:101B9000182B01F00FFCCDE906010CE09DED060BC2
:101BA000032453EC102B9FED580B51EC100B01F05C
:101BB00001FCCDE906019DED060B53EC102B51EC19
:101BC000100B01F08DFE41EC180B53EC182B01F0BB
:101BD00087FE41EC190B4E480621B0EE490AF0EEA3
:101BE000690A784401F0B8F853EC182B51EC100B4B
:101BF00001F076FE41EC180B4648B0EE490AF0EED3
